:100000000000022085820000AD820000AF82000067
:10001000B1820000B3820000B58200000000000041
:10002000000000000000000000000000B782000097
:10003000B982000000000000BB820000BD82000009
:10004000BF8200008D58000049860000BD8100007D
:10005000B1810000BF820000BF820000BF820000AB
:1000600035390000BF820000BF820000BF8200005F
:10007000BF820000BF820000BF820000BF8200007C
:10008000BF820000CD860000BF820000BF8200005A
:10009000BF820000BF820000BF820000BF8200005C
:1000A000BF820000BF820000BF820000BF8200004C
:1000B000BF820000BF8200000000000000000000BE
:1000C000BF820000BF820000BF820000BF8200002C
:1000D000BF820000BF820000BF820000BF8200001C
:1000E000BF820000000000000000000000000000CF
:1000F00000000000BF82000000000000BF8200007E
:1001000000000000000000000000000000000000EF
:1001100000000000000000000000000000000000DF
:1001200000000000000000000000000000000000CF
:1001300000000000000000000000000000000000BF
:1001400000000000000000000000000000000000AF
:10015000000000000000000000000000000000009F
:10016000000000000000000000000000000000008F
:10017000000000000000000000000000000000007F
:10018000000000000000000000000000000000006F
:10019000000000000000000000000000000000005F
:1001A000000000000000000000000000000000004F
:1001B000000000000000000000000000000000003F
:1001C000000000000000000000000000000000002F
:1001D000000000000000000000000000000000001F
:1001E000000000000000000000000000000000000F
:1001F00000000000000000000000000000000000FF
:1002000010B5054C237833B9044B13B10448AFF350
:1002100000800123237010BD440200200000000074
:100220001CDD000008B5034B1BB103490348AFF3C5
:10023000008008BD00000000480200201CDD000016
:10024000154B002B08BF134B9D46A3F5803A0021A8
:100250008B460F461348144A121A0AF0CDFC0F4B76
:10026000002B00D098470E4B002B00D09847002061
:10027000002104000D000D48002802D00C48AFF307
:1002800000800AF071FC2000290008F035FA0AF01D
:1002900045FC00BF00000800000002200000000034
:1002A00000000000440200209490012000000000A3
:1002B0000000000010F0010310D104280CD90368DD
:1002C000C3F30F1343B1013B9B001A1DC1180979F9
:1002D00011B101339342F9D1184670470023FBE76F
:1002E000037883B11A0601D40130704703F0C003CC
:1002F000C02B08BF0130024610460132037803F0DC
:10030000C003802BF8D0704708B5002103780BB9E3
:10031000084608BDFFF7E4FF0131F7E738B50022D2
:1003200004460D46411C092003F038FE40B163002D
:10033000024643F0010342F8043F0023A34200DBDE
:1003400038BD55F8231042F8041F0133F6E70128A1
:1003500038B504DC1C20BDE8384001F021BA0D6836
:10036000EA0701D41120F6E74868C30706D4042839
:1003700004D9036803F00F03042B01D00E20EAE731
:1003800003F070FC6D10002D044603DDFFF7BCFF89
:10039000A84206DA1220DEE72046FFF7A1FF013D62
:1003A0000446012DF8D120787F2808DDDF280ADCFB
:1003B0006378800100F4F86003F03F0318434000C5
:1003C00040F0010038BDEF280ADC637800039B0190
:1003D00080B203F47C630343A07800F03F00EDE7B4
:1003E000F72810DC637880041B0303F47C3300F4EB
:1003F000E0101843E37803F03F030343A078800143
:1004000000F47C60DAE74FF0FF30D8E7486838B591
:10041000C3070D4606D4042804D9036803F00F026D
:10042000092A04D00B20BDE8384001F0B9B944686E
:10043000C3F30F1364105A1EA2420BD8032194FB7E
:10044000F1F16429A8BF64210329ACBF5918D91C54
:1004500003F0E0FD0368C3F30F13013B9C4208D295
:10046000A31C013464002A6840F8232044F00104EE
:100470004460002038BD01282DE9F84304DC1C202D
:10048000BDE8F84301F08CB902284E680CD08C68A6
:10049000E70709D56410012CB8BF0124F50705D57D
:1004A0004FF0FF30BDE8F8830124F7E7042EF7D9B9
:1004B00033680D6803F00F02042A30D1E80706D430
:1004C000042D04D92B6803F00F03042B01D00E2058
:1004D000D6E73046FFF7EEFEA042E1DB304603F000
:1004E000C1FB0646284603F0BDFB03780146002BFE
:1004F000D6D0601E30440AF04EFF01460028CFD00F
:10050000012433780BB18E4203D3640044F0010020
:10051000C8E73046FFF7E4FE01340646F1E7092A52
:1005200038D177687F10BC42BADCE90729D4042DA2
:1005300027D92B6803F00F03042B22D1284603F0A0
:1005400091FB804604F1010956F82900854203D148
:10055000600040F00100A5E7C2070ED404280CD9C2
:10056000036803F00F03042B07D103F07BFB014664
:1005700040460AF0D7FE0028C7D0B9454C46E1DD19
:100580008EE7631C56F82320AA42BED0BB421C460D
:10059000F7DD85E7032A83D1C3F30F17C3F3417354
:1005A000C3EB8707BC423FF77BAFEB0728D4042D92
:1005B00026D9286800F00F03032B17D1C0F30F13BF
:1005C000C0F3417005F10408C0EB83003F1A013C01
:1005D00040440336BC423FF763AF3219434683427F
:1005E00019460FD315D1601C4000B2E7042B07D188
:1005F000284603F037FB80462846FFF75BFEE5E719
:100600000F203DE712F8015F09788D4203F10103E5
:10061000E5D00134DEE7000001282DE9F0470E4661
:1006200004DC1C20BDE8F04701F0BAB80868C20736
:1006300006D4042804D9036803F00F03042B01D067
:100640000E20EFE74B6813F00109F9D1042BF7D91D
:100650001B6803F00F03042BF2D103F003FB0446E5
:10066000706803F0FFFA82460AF066FE804670B9B1
:100670002046FFF749FE05460122A918092003F08C
:100680008DFC354F386098B90020BDE8F0875146A1
:1006900020460AF080FE231A5D425D4120466F1C11
:1006A0000028E9D0514640440AF075FE3D46F6E781
:1006B0006B0043F001034360B8F1000F19D12046ED
:1006C000FFF70EFE4D45064601DC3868DDE7311BBD
:1006D000204603F0E4FC0028D6D009F102023B6872
:1006E00043F822003046FFF7FBFD09F101093446CB
:1006F000E8E7012D02D133688360C6E75146204602
:100700000AF049FE01268146B9F1000F14D0B54226
:10071000DBDBA9EB0401204603F0C1FC0028B3D0C9
:100720003B68013609EB080443F826005146204691
:100730000AF031FE8146E7E7B542C6DB20460AF003
:10074000FBFD0146204603F0AAFC00289CD00136A0
:100750003B6843F82600B8E7546D012008B503F064
:1007600065FA400040F0010008BDC30711D4042819
:100770000FD9026802F00F03032B0AD101F0030323
:10078000C3F104035B0703F0C04322F0C0421343EC
:1007900003607047002838B504DC1C20BDE83840F1
:1007A00000F0FEBF0C68E50701D40D20F6E7012834
:1007B0001CD04B68DA07F8D55B10FF2B01D913204A
:1007C000ECE71A0442EA03621A4342EA0322641085
:1007D00024EAE474E11C8910032003F0DFFB0546E2
:1007E00010B12146FFF7C1FF284638BD0022EEE7D1
:1007F00001282DE9F0470546884604DC1C20BDE8A9
:10080000F04700F0CDBF4C6814F0010701D10D2076
:10081000F5E7022802D08B68DA07F8D5D8F800602F
:10082000F30700F1A980042E40F2A680326864101C
:10083000012C02F00F03B8BF0124092B28D17668E0
:10084000022D4FEA660605D0D8F808305B109E42AC
:10085000A8BF1E46351B0135012225EAE575A918FA
:10086000092003F09BFB074648B16D00034645F0A5
:100870000105D8F8002043F8045FA64202DA3846A2
:10088000BDE8F087013452F8241043F8041FF4E760
:10089000042B43D1304603F0E5F9FFF735FD022D77
:1008A000824605D0D8F808305B109842A8BF9A4617
:1008B000A24504DA0020BDE8F04703F0E9BB30466A
:1008C00003F0D0F90546A74222DB304603F0CAF90F
:1008D000A94606462846FFF703FD0134A245054612
:1008E000F8DAA0EB0905284603F0D2FB07460028FA
:1008F000C5D003F0B7F90446D8F8000003F0B2F908
:10090000A9EB060101442A4620460AF051F9B6E750
:100910002846FFF7E5FC01370546D4E7032B2BD12A
:10092000C2F30F13022DC2F34172C2EB830205D052
:10093000D8F808305B109A42A8BF1A46A24206DADD
:10094000002211460320BDE8F04703F027BB151B2A
:100950000423291D002291FBF3F1032003F01EFB69
:10096000074600288BD001352946FFF7FEFEE11C23
:100970002A4631440430C8E7212040E70028F8B572
:1009800004DC1C20BDE8F84000F00ABF0C6814F03D
:10099000010711D06410FF2C01D91320F2E70022C7
:1009A0000121032003F0FAFA054618B10121FFF7EF
:1009B000DCFE04712846F8BD042CEED9256805F04C
:1009C0000F05042D19D12046FFF774FC3A46C11CCF
:1009D000064691FBF5F1032003F0E0FA05460028F6
:1009E000E8D03146FFF7C1FE204603F03BF932461E
:1009F0000146281D0AF0DCF8DCE7092D1DD16668E8
:100A000076100423F11C3A4691FBF3F1032003F026
:100A1000C5FA05460028CDD03146FFF7A6FE0434BE
:100A2000B742C7DA54F8043FDA0704D55B10FF2B4E
:100A3000B3D8EA1913710137F2E7032DADD125467A
:100A4000B8E77F2902DC017001307047B1F5006F13
:100A50000CDA03468A1162F03F0203F8022B01F020
:100A60003F0161F07F01417018467047B1F5803F4A
:100A70000FDA0B1363F01F030370C1F3851301F04A
:100A80003F0163F07F0361F07F01437081700330A9
:100A90007047B1F5883F0DDAF0230370902343705F
:100AA0008B1101F03F0163F07F0361F07F018370E0
:100AB000C1700430704700000028F7B50F4603DC12
:100AC0001C2000F06DFE0CE00A6812F001000AD054
:100AD0006C4651102046FFF7B4FF011B204603F07F
:100AE000DEFA044616E0042A3BD9136803F00F032C
:100AF000092B36D155681C496D100124AC420CDD20
:100B000003F0C6FA044628B13F6803F0ABF80126AB
:100B1000AE421DDD204603B0F0BD013452F8243052
:100B200013F0010601D12720CBE75B107F2B09DDF5
:100B3000B3F5006F08DBB3F5803F07DB8B42D4BF12
:100B4000042600263044D9E70226FBE70326F9E70E
:100B5000013657F82610CB07E5D54910FFF771FF8E
:100B6000D6E70B20ADE700BFFF0F010010B510F076
:100B7000010402D04410204610BD042812D9026896
:100B800002F00F02042A07D103F06CF80A22214672
:100B9000BDE810400AF094BC032A03D10A22214682
:100BA0000430F5E70D2000F0FBFDE4E710B5044646
:100BB00011F0010011D104290ED90B6803F00F03C5
:100BC000042B09D1084603F04DF8014620460AF0EF
:100BD000A9FBB0FA80F0400910BD0020FCE700003E
:100BE0000128F8B50D4604DC1C20BDE8F84000F0F3
:100BF000D7BD4E68F20706D4042E04D9336803F03B
:100C00000F02092A01D00B20EFE77468096864100D
:100C1000C3F30F13A34298BF03F1FF3411F0010790
:100C20000DD0481000283ADD844238DB06EB800303
:100C3000844218DD9A6843F8042F0130F8E71A4817
:100C4000FFF7B4FF40B10123BC4201DA0020F8BD38
:100C5000013746F82730F7E729681448FFF7A6FF61
:100C600050B1002CF2D00122631C013C944014438B
:100C700046F823207460E9E72868C30711D40428E4
:100C80000FD9036803F00F03042B0AD1FFF76EFF9F
:100C90000028C8D129680648FFF788FF08B112204C
:100CA000A3E71120A1E700BFB7C20000BBC200004C
:100CB000C0C20000002310B50B70C3070C4606D558
:100CC0000E4942102046BDE810400AF0EFBA28B99C
:100CD0000B492046BDE810400AF008BB042801D1AA
:100CE0000849F6E709D9036803F00F03042B04D180
:100CF00002F0B8FF04490246E4E710BD94CE0000BC
:100D0000C2C20000C8C20000CDC200002DE9F043FD
:100D100001288FB081460E4607DC1C2000F040FD04
:100D2000054628460FB0BDE8F0830B6813F00104B8
:100D300040F0A180042B40F2D5801B6803F00F0324
:100D4000092B40D1274656F8273013F0010806D169
:100D5000042B04D9186800F00F00092801D02220C4
:100D6000DCE75B680137B94504EB6304EBD1012292
:100D7000A11803F013F9054608B90025D1E764006E
:100D800044F001044460424600F1080456F8221081
:100D90004B6808685B10C0F30F10984298BF00F1D1
:100DA000FF3304310020834207DC013223EAE3737E
:100DB000BA4204EB8304E9DBB3E751F804CF44F80B
:100DC00020C00130EFE7032B40F08C80274656F817
:100DD000270010F00108C2D10428C0D9036803F02D
:100DE0000F02032A38D1C3F30F12C3F34173C3EBCD
:100DF00082031C440137B945E9D10423E11C0022D8
:100E000091FBF3F1032003F0C9F805460028B4D0A4
:100E10002146FFF7AAFC00F1040956F82840E10733
:100E200020D4042C1ED9206800F00F03032B19D105
:100E3000C0F30F13C0F34170C0EB830003344B4683
:100E4000A3EB0902824211DB08F101080028A8BFC8
:100E50008144B845E1DB64E7042A80D1FFF72AFA30
:100E60000444C7E72046FFF725FAE7E714F8012F07
:100E700003F8012BE4E700252C4656F82500C207AD
:100E800032D4042830D9036803F00F02042A32D187
:100E9000FFF710FA04440135A945EED1204603F0CE
:100EA000F7F8054600283FF468AF041DB04606EB8E
:100EB000890958F8046BF30728D4042E26D933681F
:100EC00003F00F02042A34D13046FFF7F3F9074646
:100ED000304602F0C7FE3A460146204609F068FE59
:100EE0003C4421E02546C8E701A9FFF7E3FE01A83D
:100EF0000AF022FACEE7032A7FF431AFC3F30F12D0
:100F0000C3F34173C3EB82031C44C4E701A9304619
:100F1000FFF7D0FE01A80AF00FFA01A90646024623
:100F2000204609F045FE3444C145C2D10023237058
:100F3000F7E6032AF8D1C3F30F17C3F34173C3EBEA
:100F400087073A46311DC8E72DE9F04F002893B0D6
:100F50000F4607DC1C2000F023FC0546284613B092
:100F6000BDE8F08F0D6815F0010806D1042D04D9F5
:100F70002B6803F00F03092B01D00B20EBE76E6801
:100F80007610002E03DC404603F082F8E5E70128E6
:100F900026D04868C20723D4042821D9036803F067
:100FA0000F03042B1CD102F05DFE044620460AF01C
:100FB000C3F90435731E8146009303FB00FB05EB68
:100FC000860A55F8040FC30771D404286FD9036843
:100FD00003F00F02042A05D1FFF76CF983440AE0FD
:100FE000384CE3E7032A69D1C3F30F12C3F341730B
:100FF000C3EB82039B44AA45E3D1584603F048F86B
:1010000005460028AAD0D7F800A0B9F1000F03D0F8
:10101000786802F027FE0446284602F023FE0AF113
:10102000040307460193019B53F804AF0193504614
:1010300002F018FE1AF001030146029302D1BAF140
:10104000040F04D805A95046FFF734FE05A9084649
:1010500003910AF071F9DDE9023183468BB9BAF1E7
:10106000040F0ED9DAF8000000F00F0CBCF1030FEA
:1010700001BFC0F30F13C0F341700AF10401C0EBCC
:10108000830B38465A4609F093FD5F44B9F1000FCF
:1010900008D0009B434505DD38464A46214609F005
:1010A00087FD4F4408F101084645BCD156E705A924
:1010B000FFF700FE05A80AF03FF98FE702F0D2FD26
:1010C000F9E700BFF9C70000021E10B513DD0B6879
:1010D00013F001041CBF5C1024EAE474012A00D060
:1010E0004A68611C092002F059FF18B1640044F0FD
:1010F0000104446010BD00240122F2E70A6838B5FB
:1011000012F0010436D1042A34D91368496803F077
:101110000F00092818D15068C3F30F134010834201
:1011200098BF03F1FF30151DA04205DC01330220FA
:10113000984205DB002038BD45F8041F0134F3E771
:1011400042F820100130F3E7032813D1C80704D474
:101150001320BDE8384000F023BB4910FF29F7D821
:101160000432C3F30F1302EB83039A42E2D202F874
:10117000011BFAE70B2000F013FBDBE72DE9F04140
:101180004E6816F00107884629D1042E27D9326807
:1011900002F00F03092B12D17068C2F30F12451031
:1011A000AA4200D8551ED8F8008018F0010F1AD0B6
:1011B0004FEA6804002C49DDA54220DA46E0042B02
:1011C00004D13046FFF776F80546ECE7032B08D14B
:1011D000C2F30F10C2F34172C2EB8005E3E70025B2
:1011E000E1E73D46DFE741463248FFF7DFFCA8B1C3
:1011F00009F0F4FF90FBF5F303FB1500441C002FEE
:1012000055D1042E53D9336803F00F03092B26D18F
:10121000013456F824402046BDE8F0814146264876
:10122000FFF7C4FCC8B9B8F1040F11D9D8F80030E1
:1012300003F00F03042B0BD14046FFF797FC041E6D
:10124000B9D141461D48FFF7B1FC08B1122000E0BA
:101250001120BDE8F04100F0A3BA2C46CFE7042BE3
:101260001DD1304602F0FEFC012C05460FDCFFF7D5
:1012700037F8461B304602F00BFF04460028CAD060
:1012800002F0F0FC3246294609F092FCC3E72B78C5
:10129000013C002BDAD02846FFF722F8E4E7032BC5
:1012A00005D13444E478640044F00104B3E70B2032
:1012B000CFE700BFB0C20000BBC20000C0C2000048
:1012C0002DE9F0414C6814F0010788462ED1042C1A
:1012D0002CD923688E6803F00F02092A13D16568A0
:1012E000C3F30F136D10AB4200D85D1ED8F8001089
:1012F0003448FFF75BFC68B3236803F00F03092B46
:101300001ED1012317E0032A10D1F20704D41320C1
:10131000BDE8F04100F044BA7710FF2FF7D8C3F3CF
:101320000F15C3F34173C3EB8505DFE70B20EFE730
:10133000013344F823609D42FADA0020BDE8F081D1
:10134000032BFAD1033401239D42F6DB04F8017F1D
:101350000133F9E7D8F8008018F0010F0ED04FEAFA
:101360006800002822DD854220DB236803F00F039C
:10137000092B21D1013044F82060DEE741461248B4
:10138000FFF714FCB0B9B8F1040F11D9D8F8003048
:1013900003F00F03042B0BD14046FFF7E7FB0028B7
:1013A000E0D141460948FFF701FC08B11220AFE740
:1013B0001120ADE72846D8E7032B04BF2418E770B7
:1013C000BBE700BFB7C20000BBC20000C0C2000044
:1013D000086808B5C3071BD4042819D9036803F0AB
:1013E0000F02092A01D1406808BD032A09D1C3F3BD
:1013F0000F12C3F34170C0EB8200400040F00100C7
:10140000F2E7042A04D102F02DFCFEF77DFFF4E799
:101410000120E9E7024A03480D2104F001BB00BFA7
:1014200048C2000040C200000020704704207047FE
:1014300001207047002002F02BBE002070470020E2
:101440007047002070470020704700207047002040
:101450007047002070470020704700207047000050
:10146000024A03480D2104F0DBBA00BF54C3000058
:10147000BCC300007047037883B11A0601D4013061
:10148000704703F0C003C02B08BF0130024610466E
:101490000132037803F0C003802BF8D070470000BE
:1014A000F8B511F0010506461446084626D1042970
:1014B0003FD90B6803F00F03042B3AD1D30714D4A0
:1014C000042A36D9136803F00F03042B31D102F03C
:1014D000C9FB0546204602F0C5FB0146284609F037
:1014E00021FF00282DDB1ED126E002F0BBFB2946A0
:1014F0000A2209F0E5FF0546601011E012F001072D
:1015000015D1042A15D9136803F00F03042B10D149
:1015100010464D1002F0A6FB0A22394609F0D0FF12
:1015200085420EDB08DD002E09DC00200CE04D10AA
:10153000E2E7064B0F221A700136022EF5D804207E
:1015400002E0701700F00400F8BD00BF8402002024
:101550002DE9F0412E4F06460024E500EB191B79DA
:10156000032B0BD00134FF2CF7D1304604F06CFA7A
:10157000002814BF04464FF0FF3445E0304609F020
:10158000DBFE31460246E0B204F0E6FA00283BD129
:10159000EB5959681A1D8842E4D052F8045FF02DC7
:1015A00000F10100F7D1800008301A18D107D9D412
:1015B000042AD7D91B5803F00F010429D2D1C3F351
:1015C0000F13013302EB8300C507CBD40428C9D91C
:1015D00052F8233003F00F03042BC3D102F042FB77
:1015E0004FF0030805460921284609F08EFE002821
:1015F000B8D0B8F1010800F10105F4D13146284610
:1016000009F0C9FE8542ADD12046BDE8F08100BF9A
:101610006886012010B510F0010402D04410204665
:1016200010BD042812D9026802F00F02042A07D163
:1016300002F018FB0A222146BDE8104009F040BF25
:10164000032A03D10A2221460430F5E7014B0D227B
:101650001A70E4E78402002010F0010210B516D1E0
:10166000042802D90268C2F30F1211F0010310D14D
:10167000042902D90B68C3F30F13934216D1043027
:1016800000EB83020331904205D301200BE00022DE
:10169000EBE70023F1E710F8014B11F8013F1CB90B
:1016A000B3FA83F0400910BD9C42ECD00020FAE769
:1016B0002DE9F74F804689469A46304F304E6AB141
:1016C00002233B70012333603368DFF8D0B000247D
:1016D000FC54444504DB03B0BDE8F08F3260F3E70F
:1016E00059F824003168C30707EB0105C1F54871BB
:1016F00005D5244A4310284609F0A4FD04E0C8B9E2
:10170000214A284609F09EFD1C4809F015FE30606C
:10171000BAF1000F0CD008F1FF33A34208DDB0F599
:10172000487F05D2431C20223A540022FA543360E9
:101730000134CEE7042801D1144AE2E71BD902683C
:1017400002F00F03042B06D1019102F08BFA104A2C
:1017500001990346CFE7092B03D143685A465B1032
:10176000C9E7032B08D1C2F30F13C2F34172C2EBD6
:101770008303084ABFE70123074ABCE7850200202C
:10178000A805002094CE0000C2C20000C8C200001C
:10179000C3D4000043C600004EC6000034C600009B
:1017A000014B1870002070478402002010B501F032
:1017B00097FF084C231D01461F22184609F0D6FD4D
:1017C00009F0BAFD04308008000140F004002060F8
:1017D000204610BD600200202DE9F04F85B000F1D9
:1017E000180104690291D0E90232824601EB8404B7
:1017F000BC4F4169029800EB8109397803EB8205FF
:1018000029BB53F82230B84A1E1203F07F03043577
:1018100052F82330904643F0010318479AF801002C
:1018200004F0CEFD00238AF8003021E03B7873B944
:101830002B681E1203F07F03043558F82330EAE7C3
:10184000029A231D9A1AD82A26DD1A233B70DAF849
:1018500008209AF8023039789AF80100AA1A9210F2
:1018600043EA022204F0B2FD00238AF800303B7004
:10187000DAF80830ED1A029BE41AA9EB0309AD105F
:10188000A4104FEAA903CAF80C50CAF81040CAF8CD
:10189000143005B0BDE8F08F22461C463B78166038
:1018A000002BD4D12B681E1203F07F03043558F8A7
:1018B0002330B0E7029A231D9A1AD82A02DD1A2390
:1018C0003B70C4E721461C462B680B603B782A1D01
:1018D0000BB11546BBE76B681E1203F07F0308359A
:1018E00058F8233097E7029A231D9A1AD82A02DD66
:1018F0001A233B70ABE722461C463B7805EB860675
:101900001660002BA3D12B681E1203F07F03043551
:1019100058F823307FE7029A231D9A1AD82A02DD4D
:101920001A233B7093E722461C46704B53F826302F
:1019300013603B78002B8AD12B681E1203F07F03C3
:10194000043558F8233066E7684B54F8042D43F803
:1019500026203B78002B7FF47AAF2B681E1203F011
:101960007F03043558F8233055E7DFF880B15BF882
:101970002600FFF74FFE3A785AB9009054F8040D4C
:10198000FFF748FE009B1844400040F001004BF870
:1019900026003B78002B7FF45AAF2B681E1203F011
:1019A0007F03043558F8233035E7029B221DD31AF4
:1019B000D82B02DD1A233B7049E7029B21464B4599
:1019C00034BF59F80C3C01230B603B781446002BC4
:1019D0007FF43DAF2B681E1203F07F03043558F8E7
:1019E000233018E7029B221DD31AD82B02DD1A23BD
:1019F0003B702CE7029B4B4518D259F80C3C06F182
:101A000080465B10C3EB8373033E334459F82330A5
:101A100023603B781446002B7FF419AF2B681E120D
:101A200003F07F03043558F82330F4E618233B70A5
:101A30000023EDE7029B4B4518D259F80C3C54F8B3
:101A4000042D5B1006F18046C3EB8373033E3344E1
:101A500049F823203B78002B7FF4F9AE2B681E1247
:101A600003F07F03043558F82330D4E618233B7085
:101A7000F0E7029B4B4529D259F80C3C06F1804611
:101A80005B10033EC3EB8373334459F82300FFF725
:101A9000C1FD834654F8040DFFF7BCFD59F80C3C1A
:101AA0005B10C3EB837358441E44400040F00100B8
:101AB00049F826003B78002B7FF4C9AE2B681E1234
:101AC00003F07F03043558F82330A4E618233B7055
:101AD000F0E7029A231D9A1AD82A09DD1A233B70CF
:101AE000B5E600BF8402002034C40000608E0120EF
:101AF00022461C4659F8263013603B78002B7FF4B1
:101B0000A6AE2B681E1203F07F03043558F823306D
:101B100081E654F8043D49F826303B78002B7FF4E9
:101B200096AE2B681E1203F07F03043558F823305D
:101B300071E659F826004FEA600B54F8040DFFF7E0
:101B400069FD584440003B7840F0010049F8260008
:101B5000002B7FF47CAE2B681E1203F07F0304354C
:101B600058F8233057E6029BA4EB8604A3420BD817
:101B70003B78002B7FF46BAE2B681E1203F07F03C3
:101B8000043558F8233046E6C24802F05BF83B784B
:101B9000002B7FF45CAE2B681E1203F07F0304352C
:101BA00058F8233037E6002E05EB8605FFF660AEC9
:101BB0003B78002B7FF44BAE2B681E1203F07F03A3
:101BC000043558F8233026E654F8043D042B04D19C
:101BD000002E05EB8605FFF64BAE3B78002B7FF41D
:101BE00036AE2B681E1203F07F03043558F82330FD
:101BF00011E654F8043D042B04D0002E05EB8605B5
:101C0000FFF636AE3B78002B7FF421AE2B681E1218
:101C100003F07F03043558F82330FCE554F8040C36
:101C2000C307A4F1040B0BD54010013800280ADBD0
:101C3000400040F0010005EB8605CBF8000017E6F8
:101C4000FFF7E8FCF1E73B780BB15C46FFE52B685A
:101C50001E1203F07F035C4658F823300435DAE5A2
:101C6000730003F4FF7343F001032360DAF80830D4
:101C7000EB1A9D109AF8023043EA05235B0043F00B
:101C800001036360029BA9EB030322465B1043F050
:101C90000103361293608AF802607F4B3A78F6B2FD
:101CA0000C4653F83630CAF808301AB103F108056B
:101CB0008946CCE503F10C059B681E1203F07F03F7
:101CC000894658F82330A6E5029B54F8046C4B452E
:101CD0002FD1F70720D4042E17D9336803F00F0350
:101CE000042B13D1304601F0BDFF09F025FBB0F500
:101CF000487F28BF4FF448700630643003F05EFF21
:101D000070B9043DDDF80890B2E507D0002E14BF8D
:101D10004FF400700720F0E70A20EEE70720ECE719
:101D200031469AF8010004F068FB00238AF800307D
:101D3000E8E759F80C3C58495A106FF00303534335
:101D40000C3B09EB030449F8036059F8083C5A10AE
:101D50008AF80220D2B2C3F3552351F83220CAF8D0
:101D6000082059F8041C4FEA6109029901EB89091E
:101D70003978043402EB830500297FF468AD52F80A
:101D800023301E1203F07F03043558F8233042E558
:101D900054F8040CFFF73EFC1E288346A4EB86048F
:101DA00025DC00280BDC3B78002B7FF450AD2B6842
:101DB0001E1203F07F03043558F823302BE501F0A1
:101DC00079FCABF1030B354E834401F073FCA0EBBF
:101DD0000B00B042F9D83B78002B7FF438AD2B686C
:101DE0001E1203F07F03043558F8233013E5012356
:101DF0008AF8003001F05EFC0A385844CAF8040042
:101E000036E554F8040CFFF705FCA4EB8604061E27
:101E10000BDC3B78002B7FF41AAD2B681E1203F00D
:101E20007F03043558F82330F5E41D4B9E4202DD54
:101E30001D233B700BE501238AF8003001F03AFCCA
:101E40004FF47A7303FB06000A38D7E700233046C5
:101E5000A4EB8604134E1A462146FFF729FC31688D
:101E6000114802F01CF9114B316818600E4804F05B
:101E700081F931680C4804F0C5FA3B78002B7FF4F7
:101E8000E6AC2B681E1203F07F03043558F82330AC
:101E9000C1E400BF60C60000688601203F420F0019
:101EA00080EE3600A80500208502002008000020F2
:101EB0003B78A4EB8604002B7FF4C9AC2B681E1280
:101EC00003F07F03043558F82330A4E4504603F0B0
:101ED000D9FE3B78002B7FF4BAAC2B681E1203F0BE
:101EE0007F03043558F8233095E454F8043C002B64
:101EF00044D154F80C0C10F0010B1ED04FEA600BCB
:101F00004FEA4B0343F0010344F8083CBBF1000FD8
:101F100040F388804FEA4B0343F0010354F80C0C64
:101F200044F8043C54F8083CC107CBEB63032AD5C2
:101F300001335B0043F0010330E004281BD9036840
:101F400003F00F02092A01D14068D7E7042A09D11A
:101F500001F088FE0378002BD2D0FFF78CFA0BF14A
:101F6000010BF7E7032A06D1C3F30F1BC3F3417339
:101F7000C3EB8B0BC4E719233B7068E44FEA630B98
:101F80000BF1FF3BC2E7042849D9026802F00F02B7
:101F9000092A11D103F1020B50F82B3049F82630F1
:101FA0003B78002B7FF453AC2B681E1203F07F03A9
:101FB000043558F823302EE4042A2BD1039309EB7F
:101FC0008603009301F04EFE039B83465E1C012EA8
:101FD00012DC5846FFF74FFAA0EB0B06304602F032
:101FE00057F8034670B1039001F03CFE3246594663
:101FF00008F0DEFD039B05E09BF80030013E23B9AD
:1020000012223A70009A1360CAE75846FFF733FA73
:102010008346DCE7032A02D11844037989E71923B0
:102020003B7014E40435BBE7029A04EB86039B1A69
:10203000D82B11DC0122002E06F1FF3310DC3B7897
:10204000002B7FF404AC2B681E1203F07F030435D1
:1020500058F82330FFF7DFBB1A233B70FFF7F7BBBD
:1020600022601E460434E6E7029A231D9B1AD82BF1
:1020700003DD1A233B70FFF7EABB029B4B452AD2D4
:1020800054F8040CFFF7C6FA002821DD59F80C3C7F
:102090005B1083421CDBC3EB8373184400F1804068
:1020A0000438A4EB860359F820201A606FF003006F
:1020B0003B7800FB06440434002B7FF4C8AB2B684C
:1020C0001E1203F07F03043558F82330FFF7A3BB3B
:1020D00020233B70EAE71823FBE7C04B1A68A4EB08
:1020E00086036FF003001A603B7800FB064404345B
:1020F000002B7FF4ACAB2B681E1203F07F0304357A
:1021000058F82330FFF787BB54F8043C042B3B7886
:10211000A4F1040204BF05EB8605224613B1144660
:10212000FFF795BB2B681E1203F07F03144658F887
:1021300023300435FFF76FBB54F8043D042B1CBF5C
:10214000002323603B781CBF05EB86050434002B7D
:102150007FF47DAB2B681E1203F07F03043558F823
:102160002330FFF758BB002EA4EB860115DC1C239F
:102170003B7000226FF003003B780A6000FB0644CE
:102180000434002B7FF463AB2B681E1203F07F0333
:10219000043558F82330FFF73EBB0B684FF0000CB6
:1021A0005B1051F82C0010F0010202D10D233B709E
:1021B000E0E7401083420CF1010CA8BF03466645DE
:1021C000EFDC5B0043F00102D4E7002EA4EB8601B4
:1021D00015DC1C233B7000226FF003003B780A6083
:1021E00000FB06440434002B7FF431AB2B681E1235
:1021F00003F07F03043558F82330FFF70CBB0B685E
:102200004FF0000C5B1051F82C0010F0010202D1CD
:102210000D233B70E0E7401083420CF1010CB8BF86
:1022200003466645EFDC5B0043F00102D4E754F857
:10223000081C11F0010F4FEA86031ED054F8042C3D
:10224000D0071AD55210B2EB610FA4EB0303D4BF31
:10225000002204221A606FF003003B7800FB064462
:102260000434002B7FF4F3AA2B681E1203F07F03C3
:10227000043558F82330FFF7CEBA54F8042C6FF029
:102280000100A4EB030BFFF70BF9CBF80000E2E72A
:1022900054F8081C11F0010F4FEA86031ED054F8C1
:1022A000042CD0071AD55210B2EB610FA4EB030334
:1022B000B4BF002204221A606FF003003B7800FBD9
:1022C00006440434002B7FF4C2AA2B681E1203F0CC
:1022D0007F03043558F82330FFF79DBA54F8042CD7
:1022E0004FF0FF30A4EB030BFFF7DAF8CBF8000058
:1022F000E2E754E9020181424FEA860314D1E31A6E
:1023000004221A606FF003003B7800FB064404349B
:10231000002B7FF49CAA2B681E1203F07F03043568
:1023200058F82330FFF777BA0428A4EB030B01D841
:10233000002315E0C307FBD4036803F00F03042B4D
:10234000F6D1CB07F4D40429F2D90B6803F00F03BC
:10235000042BEDD1FFF780F900280CBF00230423E4
:10236000CBF80030CEE754E9020181424FEA860300
:1023700014D1E31A00221A606FF003003B7800FBCF
:1023800006440434002B7FF462AA2B681E1203F06B
:102390007F03043558F82330FFF73DBA0428A4EB37
:1023A000030B01D8042315E0C307FBD4036803F033
:1023B0000F03042BF6D1CB07F4D40429F2D90B6810
:1023C00003F00F03042BEDD1FFF746F900280CBFF3
:1023D00004230023CBF80030CEE700BF0800002024
:1023E00054F8081C11F0010F4FEA86031ED054F870
:1023F000042CD0071AD55210B2EB610FA4EB0303E3
:10240000CCBF002204221A606FF003003B7800FB6F
:1024100006440434002B7FF41AAA2B681E1203F022
:102420007F03043558F82330FFF7F5B954F8042C2E
:102430000120A4EB030BFFF733F8CBF80000E3E730
:1024400054F8081C11F0010F4FEA86031ED054F80F
:10245000042CD0071AD55210B2EB610FA4EB030382
:10246000ACBF002204221A606FF003003B7800FB2F
:1024700006440434002B7FF4EAA92B681E1203F0F3
:102480007F03043558F82330FFF7C5B954F8042CFE
:102490000220A4EB030BFFF703F8CBF80000E3E7FF
:1024A00054F8043C042BA4EB860314BF042200223E
:1024B0001A606FF003003B7800FB06440434002BE5
:1024C0007FF4C5A92B681E1203F07F03043558F86A
:1024D0002330FFF7A0B954F8080CFFF79BF88346A8
:1024E00054F8040CFFF796F85844A4EB8603400018
:1024F00040F0010018606FF003003B7800FB0644D9
:102500000434002B7FF4A3A92B681E1203F07F0371
:10251000043558F82330FFF77EB954F8080CFFF75C
:1025200079F8834654F8040CFFF774F8ABEB00001D
:10253000A4EB8603400040F0010018606FF0030038
:102540003B7800FB06440434002B7FF480A92B6801
:102550001E1203F07F03043558F82330FFF75BB9F0
:1025600054F8080CFFF756F8834654F8040CFFF7AC
:1025700051F800FB0BF0A4EB8603400040F0010093
:1025800018606FF003003B7800FB06440434002B16
:102590007FF45DA92B681E1203F07F03043558F801
:1025A0002330FFF738B954F8040CFFF733F88346AB
:1025B000B8B91F233B70A4EB86036FF00300C3F888
:1025C00000B03B7800FB06440434002B7FF43FA9A5
:1025D0002B681E1203F07F03043558F82330FFF7F1
:1025E0001AB954F8080CFFF715F890FBFBFB4FEAFB
:1025F0004B0B4BF0010BDEE754F8040CFFF70AF825
:102600008346B8B91F233B70A4EB86036FF0030029
:10261000C3F800B03B7800FB06440434002B7FF481
:1026200016A92B681E1203F07F03043558F82330D7
:10263000FFF7F1B854F8080CFEF7ECFF90FBFBF342
:1026400003FB1B0B4FEA4B0B4BF0010BDCE754F881
:10265000040CFEF7DFFF0028B8BF4042A4EB86035E
:10266000400040F0010018606FF003003B7800FB71
:1026700006440434002B7FF4EAA82B681E1203F0F2
:102680007F03043558F82330FFF7C5B8012EA4EBBB
:10269000860B32D1DBF80000FEF7BCFF02460028B3
:1026A000B4BF4FF0FF330123934202DC11461A46B8
:1026B0000B4601339B1A0392009308F08FFD009B99
:1026C000039A90FBF3F101FB130313445B0043F007
:1026D0000103CBF800306FF003003B7800FB0644A9
:1026E0000434002B7FF4B3A82B681E1203F07F0381
:1026F000043558F82330FFF78EB8022E0BD1DBF8E3
:102700000000FEF787FF0090DBF80400FEF782FF71
:10271000009B0246C8E764230122CAE7A4EB860BAC
:102720005946304601F050FE3B78CBF800006FF080
:10273000030000FB06440434002B7FF488A82B68B8
:102740001E1203F07F03043558F82330FFF763B8F7
:1027500054F8080CFEF75EFF834654F8040CFEF7AD
:1027600059FF0BEA0000A4EB8603400040F0010093
:1027700018606FF003003B7800FB06440434002B24
:102780007FF465A82B681E1203F07F03043558F808
:102790002330FFF740B854F8080CFEF73BFF8346A0
:1027A00054F8040CFEF736FF4BEA0000A4EB860356
:1027B000400040F0010018606FF003003B7800FB20
:1027C00006440434002B7FF442A82B681E1203F049
:1027D0007F03043558F82330FFF71DB854F8080C70
:1027E000FEF718FF834654F8040CFEF713FF8BEA3C
:1027F0000000A4EB8603400040F0010018606FF079
:1028000003003B7800FB06440434002B7FF41FA830
:102810002B681E1203F07F03043558F82330FEF7AF
:10282000FABF54F8040CFEF7F5FEC043A4EB860390
:10283000400040F0010018606FF003003B7800FB9F
:1028400006440434002B7FF402A82B681E1203F008
:102850007F03043558F82330FEF7DDBF54F8080C29
:10286000FEF7D8FE834654F8040CFEF7D3FE0BFAAD
:1028700000F0A4EB8603400040F0010018606FF008
:1028800003003B7800FB06440434002B7EF4DFAFEA
:102890002B681E1203F07F03043558F82330FEF72F
:1028A000BABF54F8080CFEF7B5FE834654F8040C82
:1028B000FEF7B0FE4BFA00F0A4EB8603400040F0B8
:1028C000010018606FF003003B7800FB06440434FD
:1028D000002B7EF4BCAF2B681E1203F07F0304357F
:1028E00058F82330FEF797BF54F80C0CFEF792FE11
:1028F000834654F8080CFEF78DFE8BFB002354F83A
:10290000040CCDE90023FEF785FEDDE90023C0F1CC
:10291000200CB0F1200103FA0CFC22FA00F040EA8E
:102920000C005CBF43FA01F10843A4EB860E4000A3
:1029300040F00100CEF800003B786FF0030000FB90
:1029400006440434002B7EF482AF2B681E1203F081
:102950007F03043558F82330FEF75DBFA4EB860BE8
:1029600059463046FEF7B0FB3B78CBF800006FF0DD
:10297000030000FB06440434002B7EF468AF2B6890
:102980001E1203F07F03043558F82330FEF743BFCF
:10299000A4EB860421463046FEF7B0FB3B78002BC3
:1029A0007EF455AF2B681E1203F07F03043558F8F0
:1029B0002330FEF730BFA4EB860B59463046FEF7B6
:1029C000DDFB3B78CBF800006FF0030000FB064412
:1029D0000434002B7EF43BAF2B681E1203F07F0300
:1029E000043558F82330FEF716BFA4EB86042146C1
:1029F0003046FEF765FC3B78002B7EF428AF2B6851
:102A00001E1203F07F03043558F82330FEF703BF8E
:102A1000A4EB860B59463046FEF7DAFC3B78CBF840
:102A200000006FF0030000FB06440434002B7EF42A
:102A30000EAF2B681E1203F07F03043558F82330C5
:102A4000FEF7E9BE54F8040C01F00CF954F8083C08
:102A5000DA072AD4042B0CD91B6803F00F03013BBF
:102A6000082B10D8DFE803F0052127230F0F0F0FE5
:102A70002500CC4908F056FCA4EB8603002814BFBF
:102A8000002204221A606FF003003B7800FB06442A
:102A90000434002B7EF4DBAE2B681E1203F07F03A0
:102AA000043558F82330FEF7B6BEBF49E2E7BF4908
:102AB000E0E7BF49DEE7BF49DCE7029B261DF31ACA
:102AC000D82B03DD1A233B70FEF7C1BE00F0FAFDE0
:102AD0002346400040F0010018603B783446002B4C
:102AE0007EF4B5AE2B681E1203F07F03043558F850
:102AF0002330FEF790BE029B261DF31AD82B03DD70
:102B00001A233B70FEF7A3BE00F0D4FDAA4B224669
:102B100003EA40003B7840F0010034461060002B8F
:102B20007EF495AE2B681E1203F07F03043558F82F
:102B30002330FEF770BE029B261DF31AD82B03DD4F
:102B40001A233B70FEF783BE00F0BCFD9B4B1B6855
:102B500098423DBFC3F5830303F63713C018C01A6C
:102B60004000234640F0010018603B783446002BBB
:102B70007EF46DAE2B681E1203F07F03043558F807
:102B80002330FEF748BE00F09DFD8C4B18603B786B
:102B9000A4EB8604002B7EF45AAE2B681E1203F0C1
:102BA0007F03043558F82330FEF735BE00F096FD5C
:102BB000B30068B9E41A3B78002B7EF448AE2B686A
:102BC0001E1203F07F03043558F82330FEF723BEAE
:102BD000304627467A4EE41A01231A462146FEF76C
:102BE00067FD3068643002F0E9FF18B9043D3C46E7
:102BF000FEF73EBE9AF801203168724803F015FCDA
:102C000001238AF8003000F055FD6F4A33681268DE
:102C1000063302FB0300FFF7F1B800F05FFDB300DD
:102C200068B9E41A3B78002B7EF411AE2B681E12B3
:102C300003F07F03043558F82330FEF7ECBD30462F
:102C400027465F4EE41A002201232146FEF730FD9D
:102C50003068643002F0B2FF0028C7D0594803F052
:102C600075F9CDE7FEF7A2FDA4EB860B3B78CBF818
:102C700000006FF0030000FB06440434002B7EF4D8
:102C8000E6AD2B681E1203F07F03043558F823309D
:102C9000FEF7C1BD3B78A4EB8604002B7EF4D7ADD4
:102CA0002B681E1203F07F03043558F82330FEF71B
:102CB000B2BDA4EB860B584600F03DFD3B78CBF847
:102CC00000006FF0030000FB06440434002B7EF488
:102CD000BEAD2B681E1203F07F03043558F8233075
:102CE000FEF799BDA4EB860B584600F026FD3B7815
:102CF000CBF800006FF0030000FB06440434002B07
:102D00007EF4A5AD2B681E1203F07F03043558F83E
:102D10002330FEF780BDA4EB860B5946304600F009
:102D200089FC3B78CBF800006FF0030000FB064401
:102D30000434002B7EF48BAD2B681E1203F07F034E
:102D4000043558F82330FEF766BDA4EB8604204610
:102D500000F0F6FC3B78002B7EF479AD2B681E1258
:102D600003F07F03043558F82330FEF754BDA4EB7D
:102D7000860B5946304600F0D1FB3B78CBF800007B
:102D80006FF0030000FB06440434002B7EF45FADBB
:102D90002B681E1203F07F03043558F82330FEF72A
:102DA0003ABD00BF70C6000078C600007FC60000B4
:102DB00086C600008BC60000FEFFFF7FB005002026
:102DC000A80500208502002004000020A4EB860452
:102DD000204600F09BFD3B78002B7EF438AD2B683D
:102DE0001E1203F07F03043558F82330FEF713BD9D
:102DF0000121304600F058FD3B78002B7EF427ADD2
:102E00002B681E1203F07F03043558F82330FEF7B9
:102E100002BD0021304600F047FD3B78002B7EF4D8
:102E200016AD2B681E1203F07F03043558F82330CB
:102E3000FEF7F1BCA4EB860B584600F0EDFC3B78A6
:102E4000CBF800006FF0030000FB06440434002BB5
:102E50007EF4FDAC2B681E1203F07F03043558F896
:102E60002330FEF7D8BCA4EB860B584600F0E8FCF4
:102E70003B78CBF800006FF0030000FB06440434FD
:102E8000002B7EF4E4AC2B681E1203F07F030435A4
:102E900058F82330FEF7BFBCA4EB8604204600F0B0
:102EA0009DFC3B78002B7EF4D2AC2B681E1203F005
:102EB0007F03043558F82330FEF7ADBCA4EB86043D
:102EC000204603F02FFF3B78002B7EF4C0AC2B682C
:102ED0001E1203F07F03043558F82330FEF79BBC25
:102EE000A4EB860B584603F0F3FF3B78CBF80000C9
:102EF0006FF0030000FB06440434002B7EF4A7AC03
:102F00002B681E1203F07F03043558F82330FEF7B8
:102F100082BCA4EB8604204603F054FE3B78002BD1
:102F20007EF495AC2B681E1203F07F03043558F82D
:102F30002330FEF770BCA4EB860B584603F05EFE10
:102F40003B78CBF800006FF0030000FB064404342C
:102F5000002B7EF47CAC2B681E1203F07F0304353B
:102F600058F82330FEF757BCA4EB860421463046C0
:102F700001F090FD3B78002B7EF469AC2B681E12AB
:102F800003F07F03043558F82330FEF744BCA4EB6C
:102F900086042146304601F07DFB3B78002B7EF411
:102FA00056AC2B681E1203F07F03043558F823300B
:102FB000FEF731BCA4EB86042146304601F024FC28
:102FC0003B78002B7EF443AC2B681E1203F07F038A
:102FD000043558F82330FEF71EBCA4EB86042146C6
:102FE000304601F037FC3B78002B7EF430AC2B6888
:102FF0001E1203F07F03043558F82330FEF70BBC94
:10300000A4EB860B5946304604F076F83B78CBF8B3
:1030100000006FF0030000FB06440434002B7EF434
:1030200016AC2B681E1203F07F03043558F82330CA
:10303000FEF7F1BBA4EB860B5946304604F064F86A
:103040003B78CBF800006FF0030000FB064404342B
:10305000002B7EF4FCAB2B681E1203F07F030435BB
:1030600058F82330FEF7D7BBA4EB860B5946304601
:1030700004F052F83B78CBF800006FF0030000FB3F
:1030800006440434002B7EF4E2AB2B681E1203F0DE
:103090007F03043558F82330FEF7BDBBA4EB860B45
:1030A0005946304603F04CFC3B78CBF800006FF0FB
:1030B000030000FB06440434002B7EF4C8AB2B68ED
:1030C0001E1203F07F03043558F82330FEF7A3BB2C
:1030D000A4EB86042146304601F060FC3B78002BCF
:1030E0007EF4B5AB2B681E1203F07F03043558F84D
:1030F0002330FEF790BBA4EB86042146304601F056
:10310000D1FB3B78002B7EF4A2AB2B681E1203F0A0
:103110007F03043558F82330FEF77DBBA4EB860B04
:103120005946304601F038FB3B78CBF800006FF091
:10313000030000FB06440434002B7EF488AB2B68AC
:103140001E1203F07F03043558F82330FEF763BBEB
:10315000A4EB86042146304601F0E2FA3B78002BCE
:103160007EF475AB2B681E1203F07F03043558F80C
:103170002330FEF750BB002E7CDD012E54F804BC3A
:103180003CD11BF0010F46D1BBF1040F43D9DBF852
:10319000003003F00F03042B3DD1584600F062FDD0
:1031A000FEF7D6F903465A1CA4EB860462D0022E21
:1031B00041D11BF0010F37D1BBF1040F34D9DBF83B
:1031C000002002F00F02092A2ED1DBF80400261F8E
:1031D000C0F347000122824220DD04EB8004FF2B74
:1031E0002BD840EA0326029B04F10C01CB1AD82B02
:1031F0007EF736AD1A233B70FEF729BB022E0AD1AB
:1032000054F8080CC10706D4042804D9036803F055
:103210000F03042BC2D04FF0FF33C4E701325BF839
:10322000221046F8041FD6E70B233B7000232360CF
:103230000434FEF70CBB0020D1E7029AA21AA4EBDB
:10324000800B9210CAF81020594698472E4A002346
:1032500013603B78CBF800000BF10404002B7EF4E4
:10326000F6AA2B681E1203F07F03043558F82330AA
:10327000FEF7D1BA002323603B78221D13B1144618
:10328000FEF7E5BA2B681E1203F07F03144658F8C8
:1032900023300435FEF7BFBA029BE31A9B10A4EB60
:1032A0008604CAF810302146304602F08FFE3B7883
:1032B000002B7EF4CCAA2B681E1203F07F0304358A
:1032C00058F82330FEF7A7BA029BE31A9B10A4EB31
:1032D000860BCAF810305946304602F077FE3B782C
:1032E000CBF800006FF0030000FB06440434002B11
:1032F0007EF4ADAA2B681E1203F07F03043558F844
:103300002330FEF788BA00BF546D01202DE9F84F35
:10331000224D0023002B03F1FF3706DA01F0D0FB2A
:1033200002F064FF03F0E0F819270026DFF8788048
:103330003046D8F80020B24215DD2B68184C013316
:103340009342A8BF00232B60D5F80090F02303FB25
:1033500009F304EB030AE35CA346EBB1022B04D1AF
:103360005046FEF739FA3B46D4E7012B0ED108B997
:1033700000F0A0F9F02303FB09F39B440949DBF8B3
:103380000420821A8A429CBF0222E254F02303FBEB
:1033900009F3E35C022BE3D00136CAE7000000200A
:1033A000087D01203F420F00AC0500200A4B4FF47E
:1033B00080721A60094B01211964D3F84025053247
:1033C000C3F84825C3F84C254FF44022C3F8042322
:1033D000034B1970704700BF00E100E0008000401F
:1033E000D705002004207047F8B5D1E9004514F056
:1033F00001002DD015F001002AD064101C2C3CD8FF
:103400001F4F6D1041F288363B5DAE42A8BF2E467D
:10341000012B05D00121204605F004FB01233B557B
:10342000184B1B780BB9FFF7C1FF002D4FF00003BD
:10343000154A0EDC154940F2DC50FF25D65CB4423B
:1034400004BF21F81300D5540133042BF6D1042016
:10345000F8BDD15C8C4203D10C4A22F81360F6E728
:103460000133042BF5D10023D15CFF2901D1D454C1
:10347000F2E70133042BF7D1E9E70020E8E700BFCA
:10348000B8050020D70500201C0000200E000020F9
:1034900070B5D1E9004514F001001BD015F0010012
:1034A00018D064101D2C28BF1B24154E335D012B32
:1034B00005D00121204605F0B5FA01233355114B03
:1034C0006D10A5F110029A420F4B04D94FF0FF3254
:1034D0001A60042070BD1C600C4B0D4890FBF5F089
:1034E00018800C4B1B780BB9FFF760FF0A4B0122C9
:1034F0009A64D3F848251044C3F84805E9E700BFAB
:10350000B805002090860100180000200C00002063
:1035100020A10700D70500200080004070B50C688E
:10352000E30704D40D20FEF73BF9012070BD6410C1
:103530001C2C14D8012814DD4B68042B14BF002563
:1035400002250A4E335DAB4204D02946204605F0E1
:1035500069FA3555204605F0ABFA012803D0002062
:10356000E4E70025EDE70420E0E700BFB805002010
:1035700070B50D680128CCBF4C68012415F001001E
:1035800042D014F001003FD06D10002D05DC1F4B20
:103590000122C3F80825002036E064101C2CFAD85C
:1035A0001B4E335D012B05D00121204605F03AFA70
:1035B000012333550A22174B93FBF5F3053393FB95
:1035C000F2F3154A154952F824201548120242F028
:1035D0000312C1F810250D4AC2F81005C2F81415DF
:1035E0000121C2F80415A2F5A83210690020C2F822
:1035F00010054FF6FF708342A8BF0346C2F840355E
:103600000420C2F80012116070BD00BF00F001403C
:10361000B805002000B4C40480D800000060004059
:1036200040A10040002802DC1C20FEF7B9B80120B0
:1036300070470000F8B50B68DA0707460D4604D45A
:103640000D20FEF7ADF8012007E05B10062B05D139
:1036500003F0E6FA400040F00100F8BDF3D80C4A50
:103660000C4E52F82340335D2BB10021204605F06B
:10367000D9F900233355012F06DD6B68042B03D1E4
:103680000221204605F0CEF9204605F0D5F8E1E705
:1036900000C70000B805002004207047002802DCA5
:1036A0001C20FEF77DB80B68DB0701D40D20F8E77E
:1036B00000207047024B01221A64D3F8400570477E
:1036C00000800040044B01221A64D3F840054FF4F7
:1036D0007A73B0FBF3F07047008000400120704720
:1036E000004870471CC700001D20704770B5054D8D
:1036F0002B5C8B4204460E4602D005F093F92E5502
:1037000070BD00BFB805002070B50024084D2646E6
:10371000635D012B08D10021204605F0ADF90021A1
:10372000204605F07FF9665501341D2CF0D170BD9F
:10373000B805002070470F2070473B2070470000FD
:1037400070B50468E20702D54568EB0704D40D2084
:10375000BDE87040FEF724B864101C2C2FD8184E1A
:10376000335D012B18D00121204605F05BF90123C0
:103770001B2C335510D1134BDA6E134B202AB8BFD4
:103780004FF0A04302F01F0203EB8203D3F800279F
:1037900042F44072C3F800270C4BD3F8082132B131
:1037A000D3F81821002AFBD00022C3F81821A5F372
:1037B0004A0120468910BDE8704005F0E1B870BDAF
:1037C000B805002080D800000003005000C0014070
:1037D00008B50846FFF7B4FF002008BD13B50A4A34
:1037E000044692E8030022686B46042A83E803003B
:1037F00019464FF0020003D101F006F802B010BDE7
:1038000001F028F8FAE700BF98C6000008B508469E
:10381000FFF7E4FF002008BD10B5084C63792BB119
:103820000021052005F0FEF800236371052005F056
:103830003FF900280CBF0420002010BDB80500206F
:1038400010B5084CE37A2BB100210B2005F0EAF803
:103850000023E3720B2005F02BF900280CBF042095
:10386000002010BDB805002010B50B4A0B4C0C48C9
:103870000C490023C2F80035A2F5C832C2F8103551
:103880000122626042604A60C4F80035C0F8003529
:10389000C1F8003510BD00BF00F0014000C001407C
:1038A00000100240002002401C2870B504460D465E
:1038B00025D8134E335C012B04D0012105F0B2F85A
:1038C000012333551C2C12D1FFF7CEFF0D4B1A6F7D
:1038D0000D4B202AB8BF4FF0A04302F01F0203EBAC
:1038E0008203D3F8002742F44072C3F80027291C52
:1038F000204618BF0121BDE8704005F0BDB870BD7D
:10390000B805002080D80000000300500368D907E4
:1039100002D40D20FDF744BF41680A1F51425141B6
:103920005810FFF7C1BF08B50846FFF7EFFF0020AA
:1039300008BD0000F8B5324CD4F84831ABB10023D3
:10394000D4F84855C4F848312E4B186800280CDBD1
:103950002D4A1178B1FA81F14909117005F08CF8FE
:103960002A4B1B882B44C4F84835254BD3F84C21EF
:10397000002A37D00021264ED3F84C45C3F84C110D
:103980003378244D33B12B68032B03D8224AD05C03
:1039900005F072F82B68204F01335A4202F00302FF
:1039A00003F0030358BF53422B600022042B194637
:1039B00019D00133F81810F8010CFF2801D10122A9
:1039C000F4E702B12960012105F056F801233370B4
:1039D0002A68124B33F8122004F10C031344084AEE
:1039E000C2F84C35F8BD4FF0FF3304F58C44044A5F
:1039F0002B605C3400233370C2F84C45F2E700BF03
:103A00000080004018000020D60500200C00002097
:103A1000D5050020B40500201C0000200E00002069
:103A2000094B0A4940F2DC521A805A809A80DA80A7
:103A3000074A00231370074AFF20087048708870F7
:103A4000C8701360704700BF0E0000201C000020EB
:103A5000D5050020B4050020024B4FF0FF321A605C
:103A6000704700BF18000020024A03480C2101F0F3
:103A7000D7BF00BFA0C60000CBCF000038B54FF4C1
:103A8000E131284804F09CFC274B012200211A61F7
:103A9000C3F804150321C3F808150421C3F8101551
:103AA0001A604FF080430221C3F818159A604FF056
:103AB0001023D3F80C32DB070FD51C4BC3F80425B9
:103AC000D3F80024002AFBD04FF010226FF0010140
:103AD000C2F80C120022C3F80425082004F094FE5A
:103AE000134A0023FF21995401331D2BFBD1114BA5
:103AF000114D01221A600020104A04230146146867
:103B0000002CFCD02C681160013B44EA0020F6D167
:103B10000B4B01221A6004F0ADFDBDE8384001F006
:103B20006BB800BF887C01200080004000E00140AD
:103B3000B805002000D0004008D5004000D100406A
:103B400004D00040F8B506460948094F0C4604F079
:103B500077FC8442A8BF04463546AB1B9C4205DD7A
:103B6000384604F073FC05F8010BF6E72046F8BD73
:103B7000887C01200146014804F027BC887C012094
:103B800010B5054C204604F02DFC20464FF4E131E1
:103B9000BDE8104004F014BC887C0120C3070CD49D
:103BA000064B1B68834208D8054B1B68984204D813
:103BB00050F8043C002B18BF18467047E005002061
:103BC000DC0500200B4908B50122002341F8232021
:103BD0000133642BFAD1084B1A60084B084A184687
:103BE000002107F009F8074B40F8043F064B186026
:103BF00008BD00BF608E012008000020E405002001
:103C000070670100A09D0500D8050020034B044A01
:103C10001A60044B044A1A60FFF7D4BFE005002085
:103C2000E4050020DC050020546D0120044B1B68D6
:103C30001868C0F30F10023820EAE070704700BF28
:103C4000D805002000B59BB00246054901A807F041
:103C50002DFB01A802F097F902F046FCFCE700BF3B
:103C6000E9C70000C30713D4042802D812D00B48B8
:103C70007047036803F00F03042B01D10430704731
:103C8000092B09D0064A0748032B18BF1046704776
:103C9000054870470548704705487047C2C2000094
:103CA000D4C70000DDC70000C3C70000C8C20000C1
:103CB000CDC70000064B074900201A6843F8040CE2
:103CC000C2F30F12023203EB82038B42F5D370472B
:103CD000E8050020546D01202F4B304A1868304B06
:103CE0002DE9F0411C682F4D136803F00F010729DF
:103CF00028D81368C3F30F13023302EB8302AA42DE
:103D0000F2D32949002251F82200FFF747FF41F87A
:103D100022000132642AF6D1244A1068FFF73EFFE0
:103D20001060234A106810B1FFF738FF1060214B74
:103D3000214C1E680021F0274FF03C08B14214DBF3
:103D4000BDE8F081C3F30F1302EB83039A42D0D096
:103D50001968CE0707D4884205D28C4203D351F8A4
:103D6000041C01B11960043BF0E707FB01F31A19C9
:103D70001B5D0BB90131E1E71269551E08FB0122F9
:103D800004EB82021832002DF4DB52F8040DFFF729
:103D900005FF013D1060F6E7E0050020E805002082
:103DA000DC050020546D0120608E012008000020F9
:103DB000546D0120AC050020087D0120C307F0B53B
:103DC00040D4214B1C68A0423CD3204B1D68A84224
:103DD00038D850F8043CABBB03680246C3F30F135A
:103DE000012673B9904242F8046C2BD0116851F847
:103DF000043C51F82370176041F82320013B0A4628
:103E0000EFE752F82310CF0702EB830C18D48C4253
:103E100016D88D4214D351F8047C8FB90F6807F07F
:103E20000F0EBEF1070F08D9CCF8007042F8043C21
:103E30000B680A60C3F30F13E1E741F8046CD0E7A5
:103E4000013BCEE7F0BD00BFE0050020DC0500200F
:103E50000D4930B50D4C0B461A6853F8045CC2F39B
:103E60000F12901C65B18B4214BF0A46002243F822
:103E7000042C01EB800103EB8003A342ECD330BDA3
:103E800012011A60F7E700BFE8050020546D012019
:103E9000144B2DE9F041144C1E464FF000083268D7
:103EA000C2F30F1712070FD07D1C9E424FEA850503
:103EB00005D018462A46314606F085FE03465A19B3
:103EC00004352B44C2F80080023706EB8706A64271
:103ED000E5D3E41AA410013C044A24011C601360D9
:103EE000BDE8F081E8050020546D0120D8050020D0
:103EF0002DE9F0419AB0FFF7DDFB214D0746002484
:103F000055F824000134FFF759FF642CF8D11D4BFC
:103F10001868FFF753FF1C4B186808B1FFF74EFFF6
:103F20001A4DDFF874800026D8F800309E4218DB66
:103F3000FFF78EFFFFF7D0FEFFF7AAFFFFF7BAFBF0
:103F4000134B14491B681B68C3F30F13C21B023BBE
:103F500001A807F0ABF901A802F015F81AB0BDE806
:103F6000F0812B7813B90136F035DDE72C69013C7F
:103F7000002CF8DB05EB84039869FFF71FFFF6E7D9
:103F8000608E012008000020546D0120087D012072
:103F9000D8050020A3C70000AC0500202DE9F84398
:103FA0001B4C23681B684D1CC3F30F139D42064630
:103FB00088461746A1460CDBFFF79AFF23681B686B
:103FC000C3F30F139D4204DB0A20BDE8F843FDF75D
:103FD000E7BB08F10202D9F800009B1A1B0140F868
:103FE0002230002340F8043C06F00F06034646EA60
:103FF0000816940043F8046B0119083CC9F8001036
:104000001C44A34201D3BDE8F88343F8047BF8E7DE
:10401000D8050020F8B510F0010704460E462CD153
:10402000174B1B68834228D8164B1B68834224D940
:10403000154D28600068012200F00F00FFF7AEFF69
:104040002C682F600546C0B12146043051F8042B7E
:10405000C2F30F12B242A8BF3246920006F0A8FD8A
:10406000FFF728FE44F8045CFFF736FE2268074B92
:1040700044F8047C134023602C462046F8BD00BF62
:10408000E0050020DC050020546D0120F0FF0F004A
:10409000011D0022042091FBF0F1FFF77FBF38B52E
:1040A000054608460C46FFF7F3FF50B1C21C2B46ED
:1040B000591B8C4206DC002CACBF0419041C0023E5
:1040C000237138BD13F8011B02F8011FF0E7F0B5AA
:1040D00002289BB00C4604DC1C20FDF761FB1BB0E2
:1040E000F0BD0868C20706D4042804D9036803F0A9
:1040F0000F03042B01D00E20EFE74B6813F00107EC
:10410000F9D1042BF7D91B6803F00F03042BF2D16C
:104110008B68DB0701D40D20DFE7FFF7A3FD064620
:104120006068FFF79FFDA5681AAC014604F8647D3E
:104130006D10304603F077FC29466423224603F0D5
:10414000D4FC204607F0F8F801462046FFF7A7FF09
:10415000C5E7000010B50446ADF5806D10B9FFF756
:1041600097FF0BE003F085FB0138062827D8DFE82E
:1041700000F0080810172804230000200DF5806DBA
:1041800010BD204603F0EFFB011B2046FFF787FF21
:10419000F4E7204603F09BFB400040F00100EDE710
:1041A00069464FF48062204603F0ABFB684607F097
:1041B000C3F801466846E9E704210348E6E7002022
:1041C000CDE70420DAE700BF30C80000022838B588
:1041D0000C4604DC1C20BDE83840FDF7E1BA086855
:1041E000C10706D4042804D9036803F00F03042B85
:1041F00001D00E20EFE76368DA07FAD4042BF8D970
:104200001B6803F00F03042BF3D1A368DB0701D471
:104210000D20E0E7FFF726FD05466068FFF722FD69
:10422000A46801466410284603F0FDFB214603F014
:1042300039FCBDE83840FFF78DBF012838B50C4682
:1042400004DC1C20BDE83840FDF7AABA0868C107A5
:1042500006D4042804D9036803F00F03042B01D00B
:104260000E20EFE76368DA07FAD4042BF8D91B684D
:1042700003F00F03042BF3D1FFF7F4FC054660684D
:10428000FFF7F0FC0146284603F0CDFB03F049FCA4
:10429000400040F0010038BD012870B505460C46CD
:1042A00004DC1C20BDE87040FDF77ABA0868C1073D
:1042B00006D4042804D9036803F00F03042B01D0AB
:1042C0000E20EFE76368DA07FAD4042BF8D91B68ED
:1042D00003F00F03042BF3D1FFF7C4FC064660681C
:1042E000FFF7C0FC022D014615D0A468E30712D5E4
:1042F0006410304603F097FB054603F0BAFA012834
:1043000012D1002C02DD0135012C07D12846BDE871
:104310007040FFF71FBF4FF0FF34EAE7284603F075
:1043200031FB013C0546EFE70228EFD1002CEDDD23
:104330000135012CEAD000221146284603F04CFB3F
:1043400003F020FB013C0546F3E70000086810B5C8
:1043500010F001041AD0441007EE904A9FED187A2D
:10436000F8EEE77A67EE877A17EE900A06F082F8A1
:1043700004F0A6FC0022134B06F0D4F804F056FC1F
:1043800006F080FB400040F0010010BD042812D967
:10439000036803F00F03042B07D1FFF763FC0A2225
:1043A000214607F08DF80446D6E7032B03D10A22F5
:1043B00021460430F5E70D20FDF7F2F9CCE700BF08
:1043C000D30237390000D040086808B5C30706D4C7
:1043D000042804D9036803F00F03042B04D00E2033
:1043E000BDE80840FDF7DCB9FFF73CFC0378232B60
:1043F00008BF01301022002107F062F800F10053DD
:10440000B3F1804F01D31420EAE7400040F00100EF
:1044100008BD0000024A0348062101F001BB00BFAD
:1044200000C80000FAC70000002070471E20FDF7FA
:10443000B7B91E20FDF7B4B91E20FDF7B1B91E2093
:10444000FDF7AEB91E20FDF7ABB91E20FDF7A8B9E8
:104450001E20FDF7A5B91E20FDF7A2B91E20FDF70D
:104460009FB91E20FDF79CB91E20FDF799B91E20AB
:10447000FDF796B91E20FDF793B91E20FDF790B900
:104480001E20FDF78DB91E20FDF78AB91E20FDF70D
:1044900087B91E20FDF784B91E20FDF781B91E20C3
:1044A000FDF77EB91E20FDF77BB91E20FDF778B918
:1044B0001E20FDF775B90000024A0348182101F0DB
:1044C000AFBA00BF6CC800002CC90000034B01222A
:1044D0001A60034B1868904010437047786D0120B4
:1044E000586D01202DE9F043EFF31084012304F00F
:1044F000010483F31088164A164912680E68013ABF
:104500009340154A1568154A12684FF002094FF09A
:104510000E0C4FF00D0E4FF00608A3B118422A60A2
:104520000AD0774639000139FDDC32604746390050
:104530000139FDDC5B08F0E74F4639000139FDDC4D
:1045400032606746F3E784F31088BDE8F08300BF6C
:1045500020000020606D0120646D01206C6D012041
:1045600070B5084E084D002456F824000021FFF7CE
:10457000BDF855F8240000210134FFF7B7F8052CE9
:10458000F2D170BD68CA0000B4CD00002DE9F3413E
:104590003B4D4FF441732C68ADF804300A238DF87D
:1045A0000630BCBBFFF7DCFFDFF8E480264658F896
:1045B000267001213846FFF799F801360021384668
:1045C00004F05AFA052EF2D100260DF1040816F86F
:1045D000087001213846FFF789F801360121384675
:1045E00004F04AFA032EF2D100210420FFF77EF8EE
:1045F00000213046FFF77AF800210A20FFF776F80D
:1046000001232B60FFF756F81E4B1860204602B0BE
:10461000BDE8F0811B4B1C68FFF74CF8844298BF43
:10462000001BB0F57A6F29DB022004F0F3F80420B8
:1046300004F002F90446032004F0FEF807460A20BD
:1046400004F0FAF80646012004F0E4F8012004F032
:10465000F3F8E0193044C0F532600323023090FBD8
:10466000F3F0094B0028BCBF00221A60074AA8BF1C
:10467000186000232B6013600124C7E70024C5E7FE
:10468000706D01207C6D0120586D0120786D012036
:10469000B4CD000008B5054B00221A60044B1B681E
:1046A0000BB103F085F8002008BD00BF746D012038
:1046B000EC7A012010B5041E1CDA00241049114BBD
:1046C000114A0B6004331360104B53F824301F2B36
:1046D00081BF0F4808600F49116003F01F024FF0BF
:1046E000010303FA02F38CBF0C310B490B4A0B6038
:1046F000136010BDFEF7F8FFA042DEDDDEE700BF6D
:10470000646D012008050050606D012080D8000014
:10471000080800500C080050180500506C6D01206E
:1047200008B50B68DA074CBF5B104FF0FF33012868
:104730000DDD4A68042A14BF1822202205491846B4
:104740000A60FEF7F7FFFFF7B5FF002008BD18224B
:10475000F4E700BF2000002010B510F0010402D0E3
:104760004410204610BD042812D9026802F00F023E
:10477000042A07D1FFF776FA0A222146BDE8104045
:1047800006F09EBE032A03D10A2221460430F5E733
:104790000D20FDF705F8E4E7086810F0010370B597
:1047A0001CD0FFF7D9FF0346203B5E2B27D8154CC2
:1047B00003EB83030022012110462344052A1AD06B
:1047C0009E5C052410252E4218BF4018013C4FEA7C
:1047D00041014FEA6505F6D10132EFE70428E3D93C
:1047E000026802F00F010429DED1C2F30F13002B7F
:1047F000DAD00379D8E7400040F0010070BD012015
:10480000FCE700BF7CCA000038B508680D46FFF71A
:10481000A3FF04466868FFF79FFF621E042A014653
:1048200012D8431E042B0FD8084803EB830313440C
:104830000568012202FA03F32B430360044B1B6853
:1048400013B1204602F0B5FF002038BD746D012081
:10485000EC7A012038B508680D46FFF77DFF044665
:104860006868FFF779FF621E042A014614D8431EC8
:10487000042B11D8094803EB83031344012202FAE5
:1048800003F3026822EA0302054B02601B681BB1B6
:104890000022204602F08DFF002038BD746D0120FB
:1048A000EC7A01202DE9F04F054685B008680C46EA
:1048B000FFF752FF022D01903CDD6068FFF74CFFCF
:1048C0000746A068FFF748FF0446231DDFF8C8A08D
:1048D0000293661E4FF00108029B9E4206F10109F9
:1048E00035D006EB8602531E07F1050B3D460393B8
:1048F000AB4522D0042E19D86A1E042A16D8039B71
:10490000019ADAF800005919224B4FF0010C18EA0D
:10491000020E0CFA01F11B6811D00143CAF8001015
:1049200023B162464946284602F043FF4FEA480851
:104930000135DDE701242746C7E74E46CCE720EAEC
:104940000101CAF80010002BF0D07246EAE73D1DC5
:10495000042D1BD8012C19D1DFF83C80DFF83490EE
:104960000026D8F8003004FA05F223EA0203C8F85A
:104970000030D9F80030013623B100223146781DCD
:1049800002F017FF052E05F10505EAD1002005B05C
:10499000BDE8F08FEC7A0120746D01202DE9F84319
:1049A000394B1B680C461BB94FF0FF30FFF782FEF6
:1049B000206810F001083AD1042838D9036803F0C0
:1049C0000F03092B33D10746304D57F8044F304EB3
:1049D000641040F25969A04552DA57F8040FFFF706
:1049E000BBFEC0F30742C0F307235B43524393FB74
:1049F000F9FC92FBF9F32A68202AC1B208BFC0F380
:104A000005604FEA032308BF56F8202043EA0C4311
:104A100001FB01F191FBF9F143EA010308BF42EA0E
:104A200003231846FFF75EFD08F10108D3E7FFF7FF
:104A300093FEC0F30742C0F3072340F259655B437E
:104A4000524393FBF5F492FBF5F3104A1268202AC7
:104A5000C1B204BF0E4AC0F305604FEA032308BF8A
:104A600052F8202043EA044301FB01F191FBF5F1E8
:104A700043EA010308BF42EA03231846FFF732FD69
:104A80000020BDE8F88300BF6C6D012020000020ED
:104A900058CC0000086808B5C30703D5FFF75CFED3
:104AA000054B1860054B1B681BB1034B186802F0DF
:104AB00081FE002008BD00BF746D0120EC7A01204A
:104AC0002DE9F843434E326852B9434B1B683BB95A
:104AD000424B1B68002B74D0BDE8F843FFF756BD6E
:104AE0003F4D2C6884BB3D4B1B68002B65D13A4A77
:104AF000336810681146002865D13A4F3A4EDFF806
:104B0000F4800B60002157F82400FEF7EFFD56F803
:104B1000249001214846FEF7E9FDB9F1220F10D893
:104B200058F82920314B1F2AD8BF4FF0A04302F07C
:104B30001F0203EB8203D3F8002742F44072C3F84C
:104B400000270134052CDDD12B68264EDFF8889034
:104B5000254F002BCCBF03F1FF330423002156F86F
:104B60002300FEF7C3FD2A68214B53F8228000245E
:104B700004EB840101EB0803D9F8001057F8240076
:104B8000194101F00101013403F076FF052CEFD14A
:104B90002B68012156F82300FEF7A8FD2B680021A1
:104BA00056F8230003F068FF2B68013393FBF4F4FD
:104BB00004EB84041C1B2C6003E0FFF7E7FC0028D7
:104BC00095D1BDE8F883002B97D11360BDE8F84379
:104BD000FFF7C6BC746D0120686D0120786D01205F
:104BE0005C6D012068CA0000B4CD000000030050D5
:104BF00058CD000080D800004FF0FF30FFF75ABDBD
:104C0000024A0348092100F00BBF00BF6CCD000031
:104C1000C8CD00004FF0805310B51A69094B02242B
:104C2000C3F8044522F00302884203D30022C3F8EC
:104C3000042510BDD3F80044002CFBD0C3F80805B0
:104C40001044F1E700E00140002815BF4FF4D221E5
:104C50004FF4B4214FF4B4204FF49620FFF7DABF9D
:104C600000280CBF4FF496234FF4B4231868030EAA
:104C7000532B0CBF20F07F4000207047064B0122D1
:104C8000C3F80425D3F80024002AFBD000220160D9
:104C9000C3F80425704700BF00E00140002821F060
:104CA0007F4141F0A6410CBF4FF496204FF4B42051
:104CB000FFF7E4BF0A4B30B50124C3F804450029CF
:104CC00003DC0022C3F8042530BD52F8044BD3F8AE
:104CD0000054002DFBD040F8044B0139EFE700BF32
:104CE00000E0014038B54C68023405460A462146CA
:104CF000FFF7E0FF05EB840038BD0000124B1B6896
:104D0000002B0BBF4FF4B4224FF4D2224FF4962362
:104D10004FF4B42328B91A1DDB79522B08BF104673
:104D2000704782420DD9C378522B0AD143680233AF
:104D300000EB8300824204D9C378522B18BF0020B5
:104D400070470020704700BF806E01202DE9F041C0
:104D50000020B4B0FFF7D2FF0024DFF8A48005469E
:104D6000274626464DBB224D2868FFF779FF3B4674
:104D70003246CDE900401F4902A806F097FA02A882
:104D800001F001F91C4B1A682B68002B0CBF4FF483
:104D900096234FF4B423D21A4FF470416423534343
:104DA000009193FBF1F302A8144906F07FFA02A8E0
:104DB00001F0E9F834B0BDE8F08169682A68019132
:104DC0008B1C1F44D1B2C2F307239C42C2F307429B
:104DD000009102A84146B8BF1C4606F067FA02A837
:104DE00001F0D1F82846FFF789FF01360546B9E7FB
:104DF000806E0120D2CE0000846E01207CCE0000A7
:104E0000BECE000070B50020FFF72AFF0546012046
:104E1000FFF726FF0C4B1E68B6FA86F485424FEA70
:104E20005414B8BF054620461C60FFF70DFF074A23
:104E3000074B002E18BF1346064A691C2046BDE8E2
:104E400070401360FFF72ABF806E012004B0040099
:104E500004A00500846E012070B50020FFF700FF5C
:104E600002460120FFF7FCFE1F4E204C054672B99A
:104E700068B94FF4D2214FF49620FFF7CBFE012101
:104E80002846FFF70BFF1A4B3560236029E0AA4242
:104E900008DD00233360164B23604FF4B4212368F0
:104EA000002017E001233360124B23604FF4D2211E
:104EB000F5E7120E522A08D000B123600E4801F027
:104EC00062F8BDE87040FFF79DBF5A68023203EBFD
:104ED000820301208B4205D21A68551CE9D10028B3
:104EE000D3D170BD2160FCE7806E0120846E01206B
:104EF00004B0040004A0050097CE000010B5002007
:104F0000FFF7FCFE014608B9084610BD8478FFF79C
:104F1000F5FEDA2C08BF0146F5E7000038B50021A0
:104F20004FF4FF62124805F067FEFFF7E7FF1049F4
:104F3000002400B938BD0368C3F307420A2A0BD125
:104F4000C3F30722FF2A04D001EBC20541F8320067
:104F50002B71FFF7D3FEECE7132AFAD1C3F3072333
:104F6000FF2B1EBF01EBC30241F833401471F0E781
:104F70006886012000B59BB0FFF76EFFFFF7CEFFFC
:104F800000230B491A4651F8330000B101320133B6
:104F9000FF2BF8D1074901A806F088F901A800F015
:104FA000F2FF054800F0EFFF1BB05DF804FB00BF07
:104FB0006886012007CF00001BCF00002DE9F04FCD
:104FC0004FF480729FB0604C6048002105F014FEE1
:104FD0004FF4807200215E4805F00EFED4F8009078
:104FE000B9FA89F84FEA58184046FFF72DFEA24655
:104FF000584B594C0020B9F1000F08BF1C46FFF771
:105000007DFF064648BB4846FFF72AFE534D411C2C
:105010004046FFF743FECAF800802C60FFF77EFF92
:10502000FEF7AEFDDAF800302A68002B0CBF4FF413
:1050300096234FF4B423D21A4FF4704164235343A0
:10504000009193FBF1F305A8454906F02FF905A857
:1050500000F099FF1FB0BDE8F08F3568C5F3074336
:10506000A3F10A02092AC5F3072546D8374B595D33
:1050700091BB10223B48DFF8ECB005F0BDFD374690
:105080003A68C2F307218D4209D1C2F307410B29C7
:1050900026D013292BD00A2901D1CBF8007038462D
:1050A000FFF72CFE07460028EAD12E4F396881B160
:1050B0002046FFF717FE0123044657F8231029B1B5
:1050C00020460393FFF70EFE039B04460133042B97
:1050D000F3D11E4A012353553046FFF70FFE90E7E8
:1050E000D2B2022ADBDC0BEB82025760D7E7102238
:1050F0000021584605F080FDD1E7A3F11502082AEA
:10510000EAD8134A525D002AE6D1152B0CBF31466E
:10511000002130460368C3F30742152A0ED01D2A2A
:1051200008BF0021FFF7EAFD0028F3D119B120469E
:10513000FFF7D8FD04460123054ACCE7C3F3072354
:105140009D4208BF0146EDE7806E0120806D012081
:10515000886E012004A0050004B00400846E0120C4
:1051600061CE0000F08F0120FFF728BF2DE9F84F36
:10517000DFF8A8B0274F03339246042293FBF2F6E0
:10518000DBF80030B41C002B3B684FEA84040CBFF2
:105190004FF4B4224FF4D22223449A4281460D4662
:1051A000B84614D2FFF70AFFDBF80030002B3B684B
:1051B0000CBF4FF4B4224FF4D22223449A4206D2B9
:1051C000154800F0E0FE00273846BDE8F88F2D02B4
:1051D0005FFA8AF141F0A441ADB2D8F800700D43F6
:1051E0004FEA094101F47F0129433846FFF746FDA4
:1051F00007F108053146381DC8F80050FFF73EFD9D
:105200001EB10A9A2846FFF755FD083C2544C8F808
:105210000050D9E7846E01203BCE0000806E012053
:105220000A4B0022C3F8002101225A60D3F8002162
:10523000002AFBD00022C3F80C2101229A60044B03
:105240000222C3F880211A60704700BF001000409E
:1052500000E100E0074B0222C3F88020064B002249
:10526000C3F8102101221A61D3F81021002AFBD0C3
:10527000704700BF00E100E00010004008B504499D
:105280000A780AB1FFF7E6FF0020087008BD00BFEA
:10529000896F0120024B1868400040F00100704700
:1052A0000C700120024B1868400040F0010070476C
:1052B000240000201FB5064B06491A6801A805F016
:1052C000F5FF082101A8FEF7EAFE05B05DF804FB32
:1052D00010700120ACCF00001FB54FF0805306497D
:1052E0001A6E01A805F0E2FF082101A8FEF7D7FE1B
:1052F00005B05DF804FB00BFACCF000010B5054C55
:10530000204606F019F801462046BDE81040FEF799
:10531000C6BE00BF15700120104B1B685A1C10B58B
:1053200014D0CBB1012B13D0022B13D0042B13D0EC
:105330000B4C0C4A052B08BF1446204605F0FCFF19
:1053400001462046BDE81040FEF7A9BE064CF4E732
:10535000044CF2E7054CF0E7054CEEE7280000208E
:10536000B6CF0000BCCF0000B1CF00007FC6000068
:1053700078C6000070B504460D461646FEF7A2F941
:105380004FF0805301221B6E6270E270020AA2711C
:10539000020CE2711A0A002160716372000EA2729F
:1053A0001A0C1B0E2670A17025712072E2722373F5
:1053B00070BD000010B521480278002A3DD14FF0A1
:1053C0008043C3F8002101221A60D3F80021002A8B
:1053D000FBD01B4B1B4C00220721C3F80C25C3F844
:1053E00008151949C3F81025C3F81C15C3F824255E
:1053F0000121C3F82C250822C3F83015C3F8142561
:10540000C3F818450224C3F834454FF6FF74C3F8B7
:105410003C450E4CC3F838451824C3F85445C3F82E
:105420000423D3F8002242F01002C3F80022084AF5
:10543000C3F80425FFF7F4FE017010BD896F012049
:105440000010004020000402746962752110010000
:105450008A6F0120F8B5104B1B7804460BB9FFF793
:10546000A9FF0E4E3378ABB10D4A1278D21A02F072
:1054700003010C4A02EB411202F120071068516847
:10548000254603C50832BA422C46F7D1013B33709A
:105490000120F8BD1846FCE7896F01201470012037
:1054A000886F01208A6F012030B5002889B02ADD7D
:1054B0000D6815F0010426D1042D26D92B6803F0C0
:1054C0000F03092B21D16B683F2B1EDD6846FFF7C8
:1054D000C1FFB0B19DF800200435A242A8BF1DF85D
:1054E000043004F10104A6BF5B0043F00103012373
:1054F000202C45F8043FF0D1054BDDF809201A6057
:10550000042009B030BD0020FBE72046F9E700BFCA
:105510001070012030B5384B1B788BB00BB9FFF7FA
:1055200049FF02A8FFF796FF10B900200BB030BD6D
:105530009DF808300B2BF8D99DF80930012BF4D1D8
:105540009DF80B30012BF0D12C4D2D4C2D4ADDF860
:10555000111000232B6023709DF80C3013602A4A31
:10556000116023B9DDF815302B6000230FE0012B0B
:1055700011D1DDF815309DF819202B600DF11A01BD
:105580000E239342A8BF134600229A4230D1002234
:10559000E2540420CAE7022B05D19DF815201223FE
:1055A0000DF11601EDE7042B0DD10AAA6B4652F856
:1055B000130D516803C3DDE9000103F0A9FA05F0FA
:1055C00061FA2860D1E7052BCFD10AAA6B4652F8C1
:1055D000130D516803C3DDE9000103F099FA05F0EA
:1055E00051FA9DF81D2028600A230DF11E01C8E71D
:1055F000885CA0540132C8E7896F01200C7001203B
:1056000015700120280000201070012010B5154BE6
:105610001B7804460BB9FFF7CDFEFFF71BFE124BBC
:105620000022C3F80445C3F8002101221A60D3F810
:105630000021002AFBD00022C3F80C2101229A602D
:10564000094AD2F80C31002BFBD0084B1978084BD3
:1056500003EB4113C2F80435FFF7FCFDBDE8104031
:10566000FFF7DEBD896F012000100040886F012028
:105670008A6F012000B5002889B01DDD0B6813F08A
:10568000010219D1042B17D9196801F00F0109295A
:1056900012D159683F290FDD043353F8040F10F07D
:1056A000010118BFC0F347010DF802100132202A92
:1056B000F3D16846FFF7AAFF002009B05DF804FBAC
:1056C000002810B511DD0C68E3070ED56410532CCB
:1056D0000BD8074B1B780BB9FFF76CFEFFF7BAFD31
:1056E000044BC3F80845FFF79BFD002010BD00BF29
:1056F000896F012000100040002810B50DDD0C68F6
:10570000E3070AD56410FF2C07D8054B1B780BB9AB
:10571000FFF750FE034BC3F82445002010BD00BF27
:10572000896F012000100040002813B515DD0C68BA
:10573000E10712D564100A4A0A4B072CCDE9002371
:105740000BD8094B1B780BB9FFF734FE02AB1C4496
:10575000064B14F9082CC3F80C25002002B010BD2C
:10576000E2ECF0F4F8FC0004896F01200010004026
:1057700070B5002888B020DD086810F001041CD145
:1057800004281AD9036803F00F03042B15D1FEF780
:1057900069FA064605F0D0FD122828BF12200546FA
:1057A00000F10D0202216846FFF7E4FD8DF80D506F
:1057B000A54205DC6846FFF729FF002008B070BD50
:1057C0000DEB0403325D9A730134F1E72DE9F041EA
:1057D000012888B00D4630DD086810F001042CD196
:1057E00004282AD9036803F00F03042B25D14B6842
:1057F000DB0722D5FEF736FA804605F09DFD6D6881
:105800000E2828BF0E206E10074600F1110201215C
:105810006846FFF7AFFD6B128DF80D606D14360E04
:105820008DF80E308DF80F508DF810608DF81170D6
:10583000A74206DC6846FFF7E9FE002008B0BDE895
:10584000F0810DEB040318F804209A740134EFE79B
:1058500030B5002889B016DD0C68E30713D5651054
:10586000684610220021FFF785FD63128DF80D5068
:1058700064142D0E68468DF80E308DF80F408DF8AB
:105880001050FFF7C3FE002009B030BD174BD3F80E
:10589000002122B10022C3F8002101229A60D3F82E
:1058A0000C2102B30021C3F80C11D3F80024012A03
:1058B0000F4A19D1D3F848355B4213600D4A13786B
:1058C000032B9CBF013313700B4A1378013303F091
:1058D00003031370094A02EB4313044AC2F8043568
:1058E000024B01229A6070471160F9E700100040F6
:1058F0002400002014700120886F01208A6F01208D
:10590000024A0348102100F08BB800BF2CCF0000E2
:1059100023CF0000044A05491368C8540133C3F378
:1059200009031360704700BF4474012044700120D4
:1059300070B51149114A0B68834202DC00230B60E9
:1059400017E0855CA5F1FA06012E00F1010405D8E7
:105950009C420FDAA55C013D1F2D01D92046EBE7E3
:105960000446151A165D2E550134A342FADC181AA6
:10597000086070BD1570FAE750780120507401205E
:1059800008B5FDF797FE074B1A68824284BF0022D4
:105990001A601B68C01A44F62063984294BF002026
:1059A000012008BD4070012070B5094C094D0A4E18
:1059B00023682A68934200D170BDF05CFEF7DAF8E4
:1059C0000028F9D023680133C3F309032360EFE70C
:1059D00048740120447401204470012070B5074EC2
:1059E000074D044633682A689B1ADB43C3F3090357
:1059F000A34200DB70BDFFF7D7FFF3E7447401203B
:105A00004874012010B5FFF779FA044608B920461A
:105A100010BD83781D2B08BF0446FFF76FF9F5E72B
:105A2000F0B5074D2B680B2B08DC064F0C245C43AC
:105A30003E19C6E90112013338512B60F0BD00BF99
:105A40004C740120009001202DE9F04FB3B00446C2
:105A500005F072FC012803D8002033B0BDE8F08FB8
:105A600023785B2BF8D101382518235C5D2BF3D10B
:105A700001343A21204605F048FC06460028EBD0C8
:105A8000071B002FE8DD21463A46684605F06EFC0C
:105A900032AB711C00241F446D1AA54207F8C84C94
:105AA000DADD2A4619A805F061FC32AB1D44134B20
:105AB000134ED3F8009005F8644C4FF00C0AA14542
:105AC000CADD0AFB04F36946985903EB060805F0A2
:105AD00029FC054618B9D8E90187454501DB0134A1
:105AE000EDE719A957F8350007EBC50B05F01AFCCF
:105AF00010B9DBF80400B0E70135EEE74C74012083
:105B00000090012008B5FBF785FCFFF779F8FBF75B
:105B1000A7FCFDF7A9FFFEF77DFCFEF7CDFCFFF724
:105B2000EFFE01F0D7F801F01BFE01F045FEBDE8E5
:105B3000084002F07BB8000008B54FF4166200215F
:105B4000034805F059F8034B00221A6008BD00BF56
:105B5000087D0120AC050020174B53F83000836806
:105B600003F07F031C2B70B50D46144601D00020B6
:105B700070BDC36803F07F02042AF8D1026902F005
:105B80007F02192AF3D11B0A00EB83001030FEF7C5
:105B900069F80378064633B105F0CEFBA042E6D1A2
:105BA0000023A34201DB0120E2E7F15CEA5C9142C1
:105BB000DDD10133F5E700BF68860120064B074AB7
:105BC0001B6812689B1ADB43C3F309038342D4BFEB
:105BD00000200120704700BF447401204874012058
:105BE000F8B507460E4614461D4673B90320FFF765
:105BF000E5FF10B3FA20FFF78DFEF8B2FFF78AFE3B
:105C0000F0B2BDE8F840FFF785BE501DFFF7D6FFA4
:105C100098B1FB20FFF77EFEF8B2FFF77BFEF0B2F3
:105C2000FFF778FEE0B2FFF775FEC4F30720FFF739
:105C300071FE2E46731B9C4200DCF8BD16F8010B6A
:105C4000FFF768FEF6E70000F8B50C4E0C4D002497
:105C5000F0273368A34203DCBDE8F840FFF76CBFD0
:105C600007FB04F359195B5D2BB100231A464978F1
:105C70001120FFF7B5FF0134EBE700BFAC050020B2
:105C8000087D0120F8B50E4C0E4E07460025BC429B
:105C900005F1010511D0237853B100231A4661782C
:105CA0001120FFF79DFFF0220021204604F0A4FF01
:105CB0000A2D04F1F004EAD1F8BD3560F8E700BF21
:105CC000087D0120AC0500202DE9F04F12F00106FF
:105CD000ADF54F7D82468B4617D001238DF81430E9
:105CE00042FA03F354128DF8153052141B0E8DF83E
:105CF00017208DF818308DF8164005AB0522FFF7F8
:105D00006FFF0DF54F7DBDE8F08F042A2CD9116887
:105D100001F00F03042B38D105AD022310462B7080
:105D2000FDF7A0FF044605F007FBB0F5487F0346EA
:105D300004F1FF31A8BF4FF448739E4206F10102FF
:105D40000DD1B0F5487F06D96D4B19889B78ADF819
:105D500032138DF834332B4659465046CFE716465A
:105D600011F8012FAA55E8E740F0C680A2F1040C13
:105D7000DCF100024FF0030342EB0C028DF814300B
:105D80008DF8152005AB0222E6E7092B40F0918043
:105D9000154604238DF8143055F8043F4FEA630884
:105DA000B8F1200F8DF815804FEA6323A8BF4FF09C
:105DB00020088DF816308DF8178006AC03220521D7
:105DC000B04502DC05ABE21AC6E755F8040F10F047
:105DD000010706D1042847D9036803F00F03022BFB
:105DE0000DD14FF0010323704310637047121B0E57
:105DF0004014A770E070237105340136E0E7042BEE
:105E000030D123464FF0020C03F802CBCDE901213B
:105E100000930393FDF726FF814605F08DFA0C28C9
:105E2000DDE901210AD8009B6070874201D1DC19AD
:105E3000E3E719F80740DC550137F6E723460C2065
:105E400003F8010F09F1FF3009F1080910F8017F8B
:105E500003F8017F4845F9D12E23E372237363735E
:105E60000E34CAE7012B08D12346071F03F8022B83
:105E70007842784160701C46BFE7092B09D10423A2
:105E800023704368581060705B12A370E77004348D
:105E9000B3E7032B0AD121700368C3F30F10C3F3D8
:105EA0004173C3EB800363701B12EEE7277001346C
:105EB000A3E7032B7FF425AF05238DF81430C1F33E
:105EC0000F13C1F34171C1EB830164294FEA212310
:105ED0008DF81510A8BF64218DF816308DF81710B5
:105EE00003328E4205AB01DB0A1D35E7334412F85D
:105EF000010F18710136F4E7002A7FF402AF35E78D
:105F0000D2C200000F4970B5F022002402FB041336
:105F10005D78854203D001340A2CF7D170BDF022A0
:105F20001846002104F068FE074A1368013BA342AB
:105F300000D11460002329461A461120BDE87040A4
:105F4000FFF74EBE087D0120AC05002030B5B3B090
:105F500032AC0223054604F8C83D05F0EDF9C72828
:105F600028BFC720691E0023984207DC421C234635
:105F7000FE211420FFF734FE33B030BD013311F899
:105F8000012FE254F0E770B5B2B032AC02230546FF
:105F900004F8C83D05F0D0F9C72828BFC720064639
:105FA0000023681E9E420BDC06F13200FFF716FD4F
:105FB0002346721CFF211420FFF712FE32B070BD81
:105FC000013310F8012FE254ECE700002DE9F04F07
:105FD0000128B9B08146884603DC1B20FBF7E0FBB3
:105FE00057E00868C20729D4042827D9036803F0BA
:105FF0000F03042B22D1FDF735FE0546D8F8040027
:10600000C3071DD404281BD9036803F00F03042B16
:1060100016D1FDF727FE0646204B1B680393002789
:10602000039BBB420EDC00962B461D4AC82106A8E6
:1060300005F008F906A8FFF7A6FFCEE7194DDDE742
:10604000184EE9E70C237B43174A2946985803EB7F
:10605000020B05F067F9044618B9DBE9013A9C42E6
:1060600001DB0137DCE70AEBC40231465AF83400A1
:106070000593049205F056F9DDE90423834658B9E7
:10608000536808F10801A9F102009847074BC3F8CB
:1060900000B039B0BDE8F08F0134E0E74C74012066
:1060A0008DD00000F9C7000000900120546D012040
:1060B0002DE9F0411F4F204AD7F800800546002304
:1060C000F02098450EDC0024F02000FB04F153186A
:1060D000565C8EB101340A2CF7D11848BDE8F04166
:1060E000FFF751BF00FB03F154186478AC4201D1B3
:1060F000515CE9B90133E4E7F0223146184604F077
:106100007BFD0F49457051F8351085700222A0457E
:106110000270C0E90212C0E9046601DC01343C608F
:10612000002329461A461020BDE8F041FFF758BD6C
:10613000BDE8F081AC050020087D0120D5D4000029
:106140006886012070B5FFF77FFD094EFF246FF0D0
:10615000070505FB046393F8FC37043B012B03D8C8
:10616000E043C0B2FFF7A4FF013CF2D170BD00BF15
:10617000688601202DE9F04106460F46FDF78FFFA6
:106180000D4BDFF838801860002408EBC4031B793E
:10619000062B01D0032B09D1E5B23A4631462846F9
:1061A000FFF7DAFC10B12846FFF782FF0134FF2C1D
:1061B000EBD1BDE8F08100BF080000206886012017
:1061C000F8B5094F0546FF246FF0070606FB047378
:1061D00093F8FC37AB4203D1E043C0B2FFF768FF4E
:1061E000013CF3D1F8BD00BF688601202DE9F84FCE
:1061F000FDF760FA584B1A68824284BF00221A6089
:106200001A6842F20F71821A8A420BD953491860F8
:1062100000235A181279073A022A0FD90833B3F526
:10622000FF6FF6D1BDE8F88F0720FFF7C9FF8AF8A6
:1062300000802EE00820FFF7C3FF3FE0FDF742FAA1
:10624000002814BF044601240020FDF7E5FA81462A
:106250000020FDF7F5FA424D424E0746B9F1000F16
:1062600017D02B68002B70D133682C60002B6FD0B7
:10627000DFF8F8B0DFF8F0A09BF800304FF001082D
:10628000002BD1D10920FFF79BFF8AF800808BF803
:106290000080AFB133689BB92B6834601BB3DFF863
:1062A000C8B0DFF8C8A09BF800304FF00108002B01
:1062B000C0D10920FFF784FF8BF800808AF80080A6
:1062C0002B6883B1284A1178904661B99C4238BF47
:1062D0002C602B68E31A312B05D90720FFF770FFDC
:1062E000012388F80030326882B1204B1978984633
:1062F00061B9A24288BF34603368E41A312C05D9F1
:106300000820FFF75DFF012388F800302B685BB1A0
:10631000B9F1000F08D1144C227812B90720FFF709
:106320004FFF00232B6023703368002B3FF47AAFBC
:10633000002F7FF477AF0D4C227812B90820FFF7B9
:106340003FFF0023336023706CE7002FA2D1B9E731
:10635000002FA1D1B4E700BF3C7001206886012066
:106360002C70012034700120307001203870012021
:1063700013B50446FFF768FC002301930E4B1B681E
:1063800013B901A8FDF72AFA00210846FEF782F9A1
:10639000FEF796FBFDF768FAFDF742FBFDF75CFBA5
:1063A000FEF72AFCFDF7B0F924B1FDF70BFC03481A
:1063B000FFF7E9FD02B010BDEC7A0120C6D4000061
:1063C000002301461A461120FFF70ABC07B5131235
:1063D0008DF801208DF802301314120E8DF8001084
:1063E0008DF803308DF8042001466B4605221320FA
:1063F000FFF7F6FB03B05DF804FB0A4601461220E6
:10640000FFF762BC70B505460C46FDF767F958B159
:1064100004F13200FFF7E2FA2B46224600211B204E
:10642000BDE87040FFF7DCBB70BD10B414460346F6
:106430000A46142021465DF8044BFFF7D1BB00004B
:1064400030B5084C01444FF0FF33884201D3D843A4
:1064500030BD10F8015BDAB26A4054F8222082EABB
:106460001323F2E7A8D00000FE2837B5044614D85D
:106470000B4B53F8300080B1416808308900FFF7BA
:10648000DFFF02AD45F8040D0920FFF7A7FA2B4600
:10649000042221461720FFF7A3FB03B030BD00BF45
:1064A00068860120F8B50746FFF7ACFA4FF0FF35D4
:1064B00004460CB92846F8BD2668C6F30743152BD9
:1064C0000CD104F10801384604F02CFF08B9C6F3DA
:1064D00007252046FEF712FC0446EAE71D2B08BFFD
:1064E0004FF0FF35F5E700002DE9F04FC24CC34DEA
:1064F0009DB0FFF759FA2068C0F580612844FDF788
:1065000021FB23680344064623607BB1BC4F002E69
:106510000FDC2B78FA2B40F035812368022B16DC38
:10652000FFF72EFA10B10120FFF702FA1DB0BDE807
:10653000F08F2068C0F580612844FDF703FB2368D5
:10654000034406462360FDF7B5F83860DFE7687856
:10655000AC78831E182B00F20B81DFE813F01900D2
:106560002D00310035003800410009014B0080004A
:106570008A008E00A400E500F60009010901090166
:1065800009010901090109010901090109010401C0
:10659000FF2C0FD02046FFF7B5FC9A4A002342F8A3
:1065A000343002EBC40221461371132000931A46C3
:1065B000FEF7DCFD0320B7E72046FFF779FDF9E79A
:1065C0002046FFF79FFCF5E7FFF7BCFDF2E7FFF77A
:1065D0003BFB0020FFF7CCFE8B48FFF7D4FCE9E73C
:1065E000632CE7D8894B214653F824201520FFF768
:1065F0006BFBDFE7FFF706FA6FF007080446002C95
:10660000D8D02768C7F30743152B04D02046FEF7E0
:1066100075FB0446F3E704F10806304604F08CFEEF
:1066200005460530FFF7DAF9FB20FFF773F91D2067
:10663000FFF770F9C7F30720FFF76CF9E8B2FFF72F
:1066400069F9C5F30720FFF765F9A8EB0407F3190B
:106650009D42DBDD16F8010BFFF75CF9F7E700233D
:1066600000931A4619461D20FEF780FDFDF7AAFA91
:10667000A0E72046FFF7F8FE9CE7FDF731F8644AF3
:1066800000906421634B03A804F0DCFD022303A8FF
:106690008DF80C3004F050FE03AB024600211620AA
:1066A000FFF79EFA86E75C4BDFF858811F680025EC
:1066B000FA2397FBF3F758F8354008EBC50354B3BA
:1066C000D4F8049093F804B04FEA8906B01DFFF7A0
:1066D00085F9FB20FFF71EF9012006F1010AFFF7FB
:1066E00019F9E8B2FFF716F95FFA8AF0FFF712F925
:1066F000CAF30720FFF70EF95846FFF70BF90834E5
:106700002644A6420BD8FFF74FF909FB07F001F02A
:10671000CFFFFFF749F90135FF2DCCD14AE714F837
:10672000010BFFF7F7F8ECE70024FFF78DFA22469C
:10673000214600942346DA20FEF718FD4FF4FF624D
:106740002146304804F058FA90E7012C02D1FEF7B8
:10675000FDFA2FE7022C02D1FEF706FD2AE7012001
:10676000FFF706FE26E700231A4621461A2097E780
:10677000A0F1C803052B3FF61DAF00221146FAF722
:1067800079FE17E7FB2B7FF4CEAE2268042A7FF751
:10679000C7AEB5F8037040F2F6339F423FF7C3AE81
:1067A0003B1D9A427FF7BCAEEB5CFE2B7FF4BBAE89
:1067B0006878AC781B2807F1FF367DD030D80728E1
:1067C00061D008283AD001282FD1FF2C11D02046C3
:1067D000FFF798FB6D79114B00932146BB1E2A46AB
:1067E0000A20FEF7C3FC074B43F8340003EBC40454
:1067F0002571781D98E600BF507801205074012063
:106800004070012068860120A8D40000608E01201D
:10681000BFD40000BAD40000040000205674012048
:106820001D285BD04DD31E2870D0A0F1C803052BC6
:10683000DFD83F4A3146FAF71DFEDAE7632CD8D895
:106840006B79022B0CD0032B14D0012BD1D1D5F8AE
:106850000630384A5B0043F0010342F82430C8E7B1
:10686000002EC6DDB91E3448FDF719FC314B43F844
:106870002400BEE7AB79002B2E4B0CBF0022042274
:1068800043F82420B5E7632EB3DC3246284903A839
:1068900004F08EF91CAB1E4403A8002306F8643CE8
:1068A000FFF700FE0028A4DB224B214653F82020EE
:1068B0001520FFF709FA9CE731461D48FFF75AFCFF
:1068C00097E7FF2C95D06A79022A92D81A4B009349
:1068D0002146BB1E0B20FEF749FC8AE7632EA8BFAA
:1068E0006326002303A99E420BDC1CAA26EAE6735A
:1068F0001344002203F8642C15200091731C2146D8
:10690000E9E7EA185279CA540133ECE7012C7FF425
:1069100070AF002E7FF76DAF6B791BB1322BA8BF24
:1069200032231C4664235C43044B1C6061E700BFB8
:1069300055740120608E012056740120040000204F
:10694000084B01221A60084A1368002BFCD0074B41
:106950001868042390FBF3F00638400040F0010073
:10696000704700BF00C0004000C1004008C50040A3
:106970000120704710B5064C204601F06DFA05491C
:10698000204601F0CFFA044B01221A6010BD00BF6F
:10699000107B0120801A06005478012010B5064CA7
:1069A000204601F059FA0549204601F0BBFA044B94
:1069B00001221A6010BD00BFCC7B0120801A0600A6
:1069C000587801201FB500210E20FCF78FFE012111
:1069D0000F20FCF78BFE01210D20FCF787FE1D48E0
:1069E00001F092F91C4B1D491B681D4A8B4212781D
:1069F0000FD84FF000730193002303938DF8082004
:106A000004AB13E90E00134805B05DF804EB01F088
:106A100091B914498B4202D84FF08063EBE71249D9
:106A20008B4202D84FF00063E5E710498B4202D851
:106A30004FF08053DFE70E498B4202D84FF00053EE
:106A4000D9E70C498B4294BF4FF080434FF000438D
:106A5000D1E700BFF07A01203000002048E80100B3
:106A60002C00002090D0030020A1070040420F001E
:106A700080841E0000093D00002814DD0B68DA0741
:106A800011D50D4A5B10012813600C4A09D04B68E0
:106A9000D90706D55B10022B09D0032B09D0012B97
:106AA00003D002231360002070470023FAE703237A
:106AB000F8E70123F6E700BF300000202C0000209B
:106AC00008682DE9F843C30704D40D20BDE8F84356
:106AD000FAF766BE4010FCF72DFE051E2FDBFCF713
:106AE00003FEA8422BDB00212846FCF7FFFD4FF4F4
:106AF000FA620121284601F013FE00B3DFF86C8032
:106B000000244FF00109002707264FF47A72012173
:106B1000284601F005FE90B12828C4BF09FA06F303
:106B20001F4316F1FF36F0D204F808700134052C2B
:106B3000E9D1012206210920FDF730FA08B9002029
:106B40000FE003460B2243F8042F074900F1180415
:106B500011F8012F520042F0010243F8042F9C4229
:106B6000F6D1BDE8F88300BF5B7801205C78012096
:106B70000028F8B521DD0C6814F001061DD1042CA5
:106B80001BD9236803F00F02032A16D1C3F30F1594
:106B9000C3F34173C3EB8505FFF714FF084F0334BC
:106BA000B54207DD14F8011F384601F0D0F8013670
:106BB0002070F5E7024801F0C9F80020F8BD00BFD9
:106BC000F07A012010B50468E30704D40D20BDE875
:106BD0001040FAF7E5BD6410FF2C01D91720F6E745
:106BE000FFF7F0FEE1B2044801F0B1F8024801F00D
:106BF000ADF8002010BD00BFF07A012038B5074D78
:106C0000FFF7E0FE0021284601F0A1F804462846DF
:106C100001F09CF8600040F0010038BDF07A0120DE
:106C2000274A82B001210023ADF80630C2F8F015E2
:106C3000C2F8001519461A0102F1804202F5E0423D
:106C40000133082BC2F81415C2F81015F3D11C4BF0
:106C50004FF4E062C3F818250422C3F81425C3F8E2
:106C600010250DF10602C3F82C260122C3F83026A8
:106C70001A60D3F80021002AFBD00022C3F80021BB
:106C800001225A600E4B1A46D3F804110029FBD09A
:106C90000021C3F8041101219960D2F81431002BAE
:106CA000FBD00020C2F81401C2F80005BDF8063080
:106CB0001BB28342C8BFA3F50B70400002B07047FF
:106CC0000070004008B5FFF7ABFF400040F0010046
:106CD00008BD0000024A03480E21FEF7A1BE00BF16
:106CE000ECD400005CD500000C4B1B6870B5064668
:106CF0000D4614460BB9FFF73DFEF1B2084801F00E
:106D00008FF9E9B2064801F06FF8E1B2044801F0EA
:106D10006BF80348BDE8704001F0EDB954780120EC
:106D2000107B012008B50368D90705D54168CA075B
:106D300002D58268D00704D40D20BDE80840FAF7D8
:106D40002FBD5810802801D91520F6E74910FF29DA
:106D500001D91620F1E75210FF2A01D91720ECE7DC
:106D6000FFF7C2FF002008BD0C4B1B6870B506463C
:106D70000D4614460BB9FFF711FEF1B2084801F0B9
:106D80004FF9E9B2064801F02FF8E1B2044801F0EA
:106D90002BF80348BDE8704001F0ADB958780120E8
:106DA000CC7B012001282DE9F0415EDD0D68EA076A
:106DB0005BD52F4B4C681B686D100BB9FFF7DAFDE4
:106DC000E9B22C4801F02CF914F0010613D064103C
:106DD000FF2C02D91720FAF7E3FCE1B2254801F0B5
:106DE00003F8244801F087F918B12320FAF7D8FCFA
:106DF0000020BDE8F081042CF3D9236803F00F02D2
:106E0000092A1AD154F8047FDFF868807F10B7424E
:106E1000E7DD54F8045FEB070BD56D10FF2D02D9A9
:106E20001720FAF7BDFCE9B2404600F0DDFF01365D
:106E3000EDE71720FAF7B4FCF9E7032AD1D1261DB4
:106E4000C4F1FF24C3F30F1504F57F04C3F34173AA
:106E5000084FC3EB8505FC343319AB42C1DA16F891
:106E6000011B384600F0C0FFF6E70120C1E700BF74
:106E700054780120107B012038B5134B1B68044661
:106E80000D460BB9FFF776FDE4B221460F4801F03D
:106E9000C7F8E9B20D4800F0A7FF00210B4801F048
:106EA000C9F808B1404238BD01222146074801F027
:106EB000B4F8064800F08FFF0028F4D00348BDE87E
:106EC000384000F08BBF00BF54780120107B0120B8
:106ED00008B50368D90702D54168CA0704D40D2054
:106EE000BDE80840FAF75CBC5810802801D915208D
:106EF000F6E74910FF2901D91620F1E7FFF7BCFF9B
:106F0000400040F0010008BD38B5124B1B68044634
:106F10000D460BB9FFF742FDE4B221460E4801F0E1
:106F20007FF8E9B20C4800F05FFF0B4801F0E3F88E
:106F300008B1404238BD01222146074801F06DF8F2
:106F4000054800F048FF0028F4D00348BDE8384069
:106F500000F044BF58780120CC7B012038B50D21CA
:106F60001D20FFF7D1FF5A28174C0CD101222270A7
:106F70002A211D20FFF7F8FE022001F099FB134B98
:106F800001221A6038BD0F211920FFF7BDFF3328F9
:106F900005D1022323708F2220211920EAE70D2139
:106FA0001E20FFF7B1FFC7280AD1032500222A219E
:106FB0001E202570FFF7D8FE2A462A211E20D9E779
:106FC00000232370D8E700BF34000020647801203C
:106FD000002838B504DC1C20BDE83840FAF7E0BBD7
:106FE0000B6813F0010401D10D20F5E75B10012BB4
:106FF0002ADD022B03D0052BB4BF02240324194B36
:107000001B680BB9FFF7AAFF174B93F90050022D2D
:107010001CD0032D1ED0012D11D1032C08BF02243A
:1070200000222A211D20FFF79FFE22460E211D204F
:10703000FFF79AFE2A462A211D20FFF795FE02201F
:1070400001F036FB002038BD0024D8E722012321BF
:107050001920F2E7032C14BF224602220E211E2023
:10706000EBE700BF6478012034000020204B1B6850
:1070700010B504460BB9FFF771FF1E4B93F90030B2
:10708000022B0AD0032B25D0012B26D121461D200F
:10709000FFF73AFF4FF0FF3405E0012C13D129210F
:1070A0001920FFF731FF7F28C8BFA0F580706FF06F
:1070B0007E039842B8BF1846C82358437F2390FBED
:1070C000F3F0604310BD032C0BD12B211920DFE717
:1070D0002D21FBE721461E20DAE74FF0FF34002088
:1070E000EAE7052CF4D04FF0FF340020DFE700BFC3
:1070F000647801203400002008B50120FFF7B6FFB6
:10710000400040F0010008BD08B50320FFF7AEFFC6
:10711000400040F0010008BD08B50520FFF7A6FFBC
:10712000400040F0010008BD38B5134B1B6813B98F
:107130000120FFF79BFF114B93F90030013301D180
:10714000FFF70CFF0120FFF791FF04460320FFF734
:107150008DFF05460520FFF789FF6D4304FB0454AE
:1071600000FB004003F074F901F0EEFD03F08AFC2F
:10717000400040F0010038BD647801203400002058
:10718000234B1B6870B506460BB9FFF707FC214C73
:1071900094F9001000291BDA0F211920FFF7B4FE23
:1071A000332811D11C4B68221A701C4B1E2500225B
:1071B0001A7060210C2228462570FFF7D5FD0222A7
:1071C00061212846FFF7D0FD94F9001000291EDB4D
:1071D000C9B21348124D00F023FF0F4B1048197825
:1071E00000F002FE0E4800F086FF21780C480622CF
:1071F00000F013FF741E0536284600F0ECFD30B198
:10720000284600F0EBFD04F8010FB442F4D170BD44
:10721000587801203500002037000020360000207B
:10722000CC7B012073B5002368460093ADF8043091
:10723000FFF7A6FFFFF758F91C4B9DF8015093F993
:1072400000609DF802009DF800309DF803409DF815
:1072500004209DF8051006B345EA032344EA002004
:107260001BB200B241EA0222114991F90010102923
:1072700012B202BFDB105210C010002BB8BF5B422D
:107280000028B8BF4042002A1844B8BF52421044F8
:10729000400040F0010002B070BD43EA052340EA1F
:1072A00004201BB200B242EA0122DDE736000020D2
:1072B000350000200128F8B535DD0F68FB0732D511
:1072C0004D6815F001062ED1042D2CD92B6803F042
:1072D0000F03092B27D16C68144B64101B68202CFA
:1072E000A8BF20240BB9FFF745FBC7F3470122468F
:1072F0000F480F4F00F091FE0435A64211DA0C48FA
:1073000000F069FD18B9700040F00100F8BD384682
:1073100000F064FD400040F0010045F8040F013624
:10732000EBE76000F0E70120F0E700BF54780120B0
:10733000107B01200A4B0B4A30B5D3F834450A4B79
:10734000A34208BF1346013B0246FF24151AA94277
:1073500005DD13F8015F02F8015B1C70F6E730BD34
:10736000008002406C7801206C790120064B0122DC
:107370005A60DA60D3F85821002AFBD00022C3F803
:107380000025024B1A607047008002406878012097
:1073900038B52C4B1B680D4623B92520BDE8384075
:1073A000FAF7FEB9012801DC1C20F7E70C68E107B9
:1073B00009D4042C09D9236803F00F03DA1E012A2B
:1073C00005D92420EAE70223F8E70123F6E76A68F3
:1073D000D20701D41120E1E7042B0CD12046FCF7A1
:1073E00041FC03F0A9FF6A685210013A01D48242BD
:1073F00009DB1220D2E72068C0F30F12C0F34170FE
:10740000C0EB8200EFE71049D1F82031C3B1801AF8
:1074100080280E4AA8BF802004340023834204DA67
:1074200014F8015B9D540133F8E70023C1F84805C7
:10743000C1F8203101238B60400040F0010038BDCD
:107440001846F9E768780120008002406C7A012034
:1074500070B5174D174CD5F83435174E9C4214BFF4
:10746000234633464FF480721846FF2103F0C4FBD5
:107470004FF48073C5F83405C5F838350023C5F8D6
:10748000083101232B60D5F83405844208BF344607
:1074900004F1FF00A21E0178FF2900F1FF3301D1A2
:1074A0009A4202D1001B013070BD1846F3E700BFBD
:1074B000008002406C7901206C780120002838B5EA
:1074C00004DC1C20BDE83840FAF76AB90D68EB0708
:1074D00006D4042D04D92B6803F00F03032B01D02D
:1074E0002420EFE7124B1B680BB92520EAE7114B6C
:1074F000D3F808310BB9012038BDFFF7A9FF041EEE
:10750000F9D001DA1B20DDE7284650F8043BC3F32D
:107510000F12C3F34173C3EB82039C4228BF1C4686
:107520002146FFF707FF600040F00100E4E700BFDD
:1075300068780120008002400028F8B504DC1C2097
:10754000BDE8F840FAF72CB90968CB0701D40D2043
:10755000F6E71E4D1E4C2B68491023B1D4F80035B8
:107560000BB1FFF703FF1B4B1A68C4F814255B68C7
:10757000C4F80C354FF486734B43C4F82435164BCE
:107580004FF48072FF21184603F036FB4FF48073EE
:10759000C4F83405C4F83835104BC4F8443580239A
:1075A000C4F848352023C4F80032002601270823F8
:1075B000C4F800350520C4F808612760C4F84865A0
:1075C000A76001F075F82F603046F8BD687801209B
:1075D0000080024080D800006C7801206C7A012085
:1075E00070B5124E04460D46002D14DDD6F820313C
:1075F00093B1802D10DC0E4B621914F8011B03F8B7
:10760000011FA242F9D1094B0022C3F84855C3F823
:10761000202101229A6070BDFDF752FAFEF7E6FDC7
:10762000FEF762FF012001F043F8DDE70080024031
:107630006B7A012006490A6808B52AB1054BD3F8D0
:1076400000350BB1FFF792FE0020086008BD00BFB7
:10765000687801200080024038B51C4B1B6823B9B4
:107660002520BDE83840FAF79BB8194BD3F808310C
:1076700013B9184D284638BDFFF7EAFE041EF8D0AE
:1076800001DA1B20EDE7E11C002289100320FCF742
:1076900085FC054608B90A20E3E721460430FFF7D8
:1076A00049FEEB07E6D4042DE4D92A6802F00F0363
:1076B000032BDFD104F00303C3F104035B0703F0E2
:1076C000C04322F0C04213432B60D3E76878012007
:1076D0000080024038000020002837B504DC1C2060
:1076E000FAF75EF803B030BD1C4B1B680BB92520C0
:1076F000F6E7086810F001040CD04310FF2B01D905
:107700002820EDE702A8012100F8013DFFF768FFFE
:107710000020E7E7042813D9036803F00F02042AC6
:1077200010D1FCF79FFA054603F006FE80280146BB
:1077300003D92620FAF734F8EAE72846FFF750FF86
:107740002046CFE7032AFBD1C3F30F11C3F34173E4
:10775000C3EB81018029ECDC0430EFE7687801207D
:10776000024A03480621FEF75BB900BFF8D50000C6
:1077700028D6000000207047012070470020704785
:10778000002070470020704701207047002070479C
:10779000002070470020704700207047002070478D
:1077A000002070470020704700207047002070477D
:1077B0007047704770470000024A03480F21FEF7E8
:1077C0002FB900BF48D60000C0D6000002461046C0
:1077D00001320378013B1F2BF9D9704708B5FFF739
:1077E000F5FF0378002B39D0222B00F1010011D1D5
:1077F000037823B1222B00F1010204D11046BDE829
:107800000840FFF7E3BF5C2B02D1437803B1821C31
:107810001046EDE73A2BF2D02C2BF0D07B2B0BD17E
:10782000FFF7D4FF0378002BE9D07D2B01D1013085
:10783000E5E7FFF7D3FFF5E75B2B10D002461046D4
:1078400012F8013B002BDAD0202BD8DD2C2B05D0F1
:1078500003F0DF015D2901D0222BF0D108BDFFF735
:10786000B5FF0378002BCAD05D2BE0D0FFF7B6FF41
:10787000F7E708B5F0B1FFF7A9FF0378222B1AD07C
:107880007B2B1AD05B2B1AD0A3F13002092A05D921
:107890002D2B05D14278303A092A07D8032009E078
:1078A000742B0ED0662B0ED06E2B0ED0181C18BF6A
:1078B0000120404208BD0420FCE70220FAE7012035
:1078C000F8E70520F6E70620F4E70720F2E738B5E9
:1078D000FFF77CFF03782D2B11D101304FF0FF34DF
:1078E000431E00210A2501E005FB012113F8012FA9
:1078F000303AD0B20928F7D904FB01F038BD012491
:10790000EEE710B51446FFF761FF0378222B02D093
:1079100000230B7010BD621E01300378222BF7D0BC
:10792000002BF5D05C2B07D0441C002AF0DD01F8B9
:10793000013B013A2046F0E74378622B00F1020454
:1079400009D0662B09D06E2B09D0722B09D0742B6D
:1079500008BF0923E9E70823E7E70C23E5E70A2343
:10796000E3E70D23E1E710B50446FFF737FF0346D1
:10797000A342184605D90278013A1F2A03F1FF33C2
:10798000F6D910BD08B590B1037883B1FFF71EFF9B
:10799000037803F0DF035D2B09D0FFF71FFF0378A7
:1079A0002C2B08BF0130BDE80840FFF70FBF0020B7
:1079B00008BD38B50D1E0DDD03785B2B0AD10130F3
:1079C000FFF704FF0124A54205D0FFF7DBFF10B14C
:1079D0000134F8E7002038BD38B5154609B1002359
:1079E0000B70F8B10378E3B1FFF7F0FE03782C2BAE
:1079F000044603D10130FFF7E9FE044623787D2BCE
:107A00000FD019B12A462046FFF77BFF2046FFF72B
:107A1000E5FE03783A2B05D10130BDE83840FFF789
:107A2000D5BE002038BD2DE9F0410D469AB0044680
:107A30002F789FB32E21284603F067FC804690B133
:107A4000461B303F092F13D82846FFF740FF014659
:107A50002046FFF7AEFF044604B3B8F1000F1DD077
:107A600001363544E4E7284603F066FC0646E8E7BD
:107A700023787B2B11D1601C642201A9FFF7ACFF96
:107A8000044658B13246294601A803F05DFC00289F
:107A9000E2D02046FFF7A2FEEEE7002420461AB00F
:107AA000BDE8F08138B50D1E04461CDDFFF7E1FE90
:107AB000012807D1601C012D00D138BDFFF762FFFE
:107AC000013DF8E702280ED100221146601CFFF7A5
:107AD00083FF012DF1D0FFF755FF00221146FFF77C
:107AE0007BFF013DF5E70020E7E7F8B50C1E0746F0
:107AF00015461E4613DDFFF7BCFE02280FD13246A5
:107B00002946781CFFF768FF012C00D1F8BDFFF76C
:107B100039FF32462946FFF75FFF013CF4E70020BA
:107B2000F4E710B50446C8B1FFF750FE03787B2B8D
:107B30000AD10130002400221146FFF74DFF68B141
:107B4000FFF74CFE0134F6E75B2B06D10130002431
:107B5000FFF718FF10B10134FAE70024204610BDEA
:107B6000002870B514DD0D68EB0711D56D10013DCF
:107B7000FDF7C4F900264FF0FF3460B916B3304664
:107B800003F0DAFB01463046BDE87040FCF787BAE7
:107B90004FF0FF35ECE70368C3F30742152A0BD11A
:107BA000C3F307239C42B8BF1C469D4201D100F19C
:107BB0000806FDF7A3F8E0E71D2A04BF00264FF0F2
:107BC000FF34F6E7601C400040F0010070BD00008B
:107BD00010B508680C46FCF745F8FEF763FC002872
:107BE000A2BF034B626843F82020002010BD00BFF5
:107BF000608E012008B50868FCF734F8FEF752FCE7
:107C00000028AABF024B012053F8200008BD00BF86
:107C1000608E012008B50868FCF724F8FEF742FCE6
:107C20000028ACBF0420002008BD0000024A034821
:107C30000421FDF7F5BE00BF5CD7000056D7000059
:107C400008B5FBF71BFFFBF7E1FFFDF75BFF0448FF
:107C5000FEF799F9FDF78EF9BDE80840FEF772BA14
:107C6000ABD70000FBF752BB38B50025057329B927
:107C70000B4B0C4A0C48252102F02CFF01600B49EC
:107C800051F82220027151F8233083719DF8103091
:107C900051F8233043710223C371856038BD00BFA2
:107CA000C3D7000022D80000D1D7000080D8000040
:107CB000037B23B943738373036101230373704709
:107CC00084B00DF1100C0CE90E009DF8081002684C
:107CD00000230129C2F80035039B12D00BD30329DE
:107CE0000CD0C2F85435019BC2F824350123C2F8E8
:107CF000003504B0704743F00203F2E743F0040399
:107D0000EFE743F00603ECE710B5FFF7D1FF036898
:107D10008279C3F808254279C3F80C250279C3F8A3
:107D20001025034BBDE810400ECBFFF7C9BF00BFC5
:107D3000047B012010B485B001AC84E80E0094E807
:107D40000E0005B05DF8044BFFF7BABF704703683B
:107D5000C3F81C15D3F80821002AFBD0D3F8180566
:107D60000022C3F80821C0B27047000007B5094BD4
:107D700009490A484FF080421A6000229A600222A4
:107D80001A710F2300930E220D23FFF76DFF03B02E
:107D90005DF804FB047B012000300240F07A0120F2
:107DA0002DE9F84380460D46174601EB02090C46C3
:107DB0004C45A4EB05060BD0D8F8003014F8011B95
:107DC0001B68404698470028F2D13046BDE8F8834A
:107DD0003E46FAE77047203000F03CBA203000F011
:107DE0002BBA203000F03CBA38B5437F0D460BB9B2
:107DF000002038BD00F16804204600F039FA002860
:107E0000F6D12046294600F008FA0120F1E70000EB
:107E10002DE9F0411E4600254FF47A73C0E9015365
:107E20000C4B044640F8203B8846174600F0ECF91E
:107E300004F1680000F0E8F99DF8183063769DF8C9
:107E40001C302676C4E90487A37665772046BDE812
:107E5000F08100BF68D80000F0B5837E2E4C2F4D16
:107E60000121C17654F82320437E54F8233012F0C8
:107E7000200F14BF2F464FF0A04702F01F0213F04F
:107E8000200F03F01F0308BF4FF0A04502F5E0727A
:107E900003F5E07340F20C6647F8226045F8236072
:107EA00003694FF0CC72C3F8242503690622C3F896
:107EB0000025827E036954F82220C3F80825427EFB
:107EC000036954F82220C3F80C2590F91830144A9D
:107ED0005C0903F01F03994004F1600342F823108A
:107EE00090F91830002BBDBF03F00F0302F6FC32EF
:107EF000D2189B18B5BF40234022137683F8002385
:107F000090F918300122590903F01F0302FA03F314
:107F1000034A42F82130F0BD80D800000003005031
:107F200000E100E0C37EA3B103690022C3F800258D
:107F30000A4B99420ED90A4B994294BF4FF0806187
:107F40004FF0C8610369C3F8241503690622C3F81A
:107F5000002570474FF0CC71F4E700BFA086010008
:107F600090D003002DE9F041044688461F4615468F
:107F7000002A50D000F12006304600F059F923695C
:107F8000C3F88885236901221A622369C3F834651E
:107F90002369C3F8385523691A602269D2F84C3135
:107FA0001BB9D2F82431002BF8D00023C2F84C3191
:107FB0002269D2F85C311BB9D2F82431002BF8D0F9
:107FC0000023C2F85C3122696FB9D2F8243153B969
:107FD0000123D3612369D3F84821002AFBD0002272
:107FE000C3F8482109E0012353612369D3F8042130
:107FF000002AFBD00022C3F804212369D3F82421EE
:1080000012B10022C3F824212369D3F83C0520666D
:10801000C0B2BDE8F0811046FBE70123FFF7A2BF25
:1080200010B5044680F8B010683000F001F9012363
:10803000637710BDF8B500234377036990F8B0204B
:10804000C3F88825036901261E62036900F16805EB
:108050000446C3F8445528460F4600F0FBF8236950
:10806000C3F8480523699E602369D3F850211AB9E3
:10807000D3F82421002AF8D00022C3F85021284642
:1080800000F0E8F8236930B1D3F860211AB9D3F8C9
:108090002421002AF8D00022C3F8602123696FB997
:1080A000D3F8242152B90122DA612369D3F8482197
:1080B000002AFBD00022C3F8482109E001225A61BE
:1080C0002369D3F80421002AFBD00022C3F804213D
:1080D0002369D3F8240168B10022C3F8242123695D
:1080E000D3F8C404C3F8C404022803D004280CBF86
:1080F00003200420F8BD0121FFF79CBF70B5436940
:10810000D3F86421044692B10022012500F1200633
:10811000C3F864210577304600F08AF86369C3F834
:10812000346563694022C3F8382563691D63636958
:10813000D3F86821DAB10025C3F8685104F1680664
:10814000012363772577304600F072F8D4F8B43015
:1081500003B19847636965773046C3F8446500F01A
:1081600079F86369C3F84805636901225A63636952
:10817000D3F8042162B10022C3F80421237F3BB16C
:108180006369D3F83C05D4F8B830206603B198474A
:108190006369D3F8242152B10022C3F82421636912
:1081A000D3F8D024C3F8D024636901225A6170BD8A
:1081B0000148FFF7A3BF00BF107B01200148FFF774
:1081C0009DBF00BFCC7B012007B514231322CDE94E
:1081D00000324FF04022114604230848FFF718FEF2
:1081E000074A08481E231F21CDE900310323114609
:1081F000FFF70EFE03B05DF804FB00BF107B01200B
:1082000000300040CC7B012008B54022002102F064
:10821000F3FC0022C0E9102208BD026C10B5531C0B
:10822000446C03F03F039C421CBF8154036410BDA7
:108230000023C0E910337047D0E9102393421FBFD9
:10824000C25C013303F03F03436414BF10464FF098
:10825000FF307047D0E91030181A48BF40307047DF
:10826000D0E91023934214BFC05C4FF0FF30704739
:10827000036C406C013303F03F031B1A5842584112
:10828000704700000649074A074B9B1A03DD043B71
:10829000C858D050FBDC00F013F8F7F7D1FF00000E
:1082A00028DD00000000002044020020FEE7FEE779
:1082B000FEE7FEE7FEE7FEE7FEE7FEE7FEE7FEE796
:1082C000394B1A680D2A08D14FF080420021C2F8BC
:1082D0000C11C2F81011C2F838151B680D2B46D1CD
:1082E0004FF08052314BD2F80414C3F82015D2F865
:1082F0000814C3F82415D2F80C14C3F82815D2F8C2
:108300001014C3F82C15D2F81414C3F83015D2F891
:108310001814C3F83415D2F81C14C3F84015D2F859
:108320002014C3F84415D2F82414C3F84815D2F821
:108330002814C3F84C15D2F82C14C3F85015D2F8F1
:108340003014C3F85415D2F83414C3F86015D2F8B9
:108350003814C3F86415D2F83C14C3F86815D2F881
:108360004014C3F86C15D2F84424C3F870250E4BA2
:108370001B680D2B09D14FF08043D3F80024D2079E
:1083800044BF6FF00102C3F80024094AD2F88830D4
:1083900043F47003C2F88830BFF34F8FBFF36F8F81
:1083A000044B054A1A6070473001001000C00040BD
:1083B00000ED00E03C0000200090D0030120704759
:1083C00003681322DB69184770470369C3F81C155B
:1083D0000369D3F81C21002AFBD00022C3F81C211A
:1083E0000120704710B490F95C30144C59090122F7
:1083F000203103F01F0302FA03F344F8213003692C
:108400005DF8044B0421C3F8081303695A6003693B
:10841000DA6003690022C3F8002502694FF0FF33D8
:10842000C2F80C350269C2F814350269C2F8083581
:1084300002691430C2F81035FFF7FABE00E100E01F
:108440001430FFF707BF1430FFF70ABF1430FFF7EF
:10845000F3BE0000036990F85E2010B5C3F80C2548
:10846000036990F85D20C3F8142590F86120036932
:10847000012A01BF90F85F40C3F81045036990F8E6
:10848000604006BFC3F8084503690022B1F5966F46
:10849000C3F86C2569D9B1F5166F69D9B1F5965F46
:1084A00069D9B1F5165F68D9B1F5615F67D9B1F5E2
:1084B000964F66D9B1F5E14F65D9B1F5164F64D93C
:1084C000B1F5614F64D9B1F5963F64D9B1F5E13F9B
:1084D00063D9B1F5613F63D9364B994263D9B1F5A0
:1084E000E12F63D9B1F5612F94BF4FF070634FF066
:1084F00080530269C2F8243503690422C3F80025B9
:1085000001690023C1F808310169C1F81C31016912
:1085100001230B6001698B600169C1F8042390F9A4
:108520005C20510902F01F0293406031224A42F858
:10853000213090F95C30002BBDBF03F00F0302F631
:10854000FC32D2189B18B5BF60236022137683F8E3
:10855000002390F95C300122590903F01F0302FA4D
:1085600003F3154A42F8213010BD4FF49E23C0E7B3
:108570004FF41D23BDE7114BBBE7114BB9E7114B7E
:10858000B7E7114BB5E7114BB3E74FF41D03B0E765
:108590004FF46B03ADE70E4BABE74FF0EB73A8E77F
:1085A0004FF06C73A5E74FF08063A2E74FF0E863EC
:1085B0009FE700BF90D0030000E100E000B013008F
:1085C0000050270000F03A0000A04E0000C07500E7
:1085D00000903A012DE9F0411E4600254FF47A73D0
:1085E000C0E901530D4B044640F8143B174688463A
:1085F000FFF70AFE0A4AC4F8108084F85C7052F84B
:10860000263084F85D309DF8183052F8233084F815
:108610005E3084F861502046BDE8F08114D9000036
:1086200080D8000010B50369D3F8082104464AB188
:10863000D3F818151430C9B2FFF7EFFD23690022F3
:10864000C3F8082110BD00000148FFF7EBBF00BFD1
:10865000887C012007B522230093022221230349AD
:108660000348FFF7B7FF03B05DF804FB00200040AC
:10867000887C012008B102F08DBD70470A4B196853
:108680000A4B30B5D3F804050C060D0A44EA000283
:108690004FF47A712B46A2FB014501FB0355E00B19
:1086A00040EA454030BD00BFEC7C01200010014095
:1086B00038B5044648B1FFF7E1FF054600F01AF867
:1086C000FFF7DCFF401BA042F8D338BD074B002268
:1086D000C3F8042182B0D3F80431054A0193019B09
:1086E00013680133DBB2136002B070470010014021
:1086F000EC7C01207047704708B500F067F8FFF781
:10870000FAFF0120FFF7D4FFFFF79AFA034CFFF7B7
:10871000A9FA002CFBD0AFF30080F8E700000000BE
:1087200038B5174B174D53F82030174813F0200F6A
:108730004FF0010403F01F0304FA03F408BF4FF0E5
:10874000A04000292B681149B3FBF1F300F5A260AA
:1087500002FB03F321464FF00A02B3FBF2F314BF0E
:108760002246002200F014F842F2107358434FF4EE
:108770007A722B68B3FBF2F3B0FBF3F038BD00BFA5
:1087800080D800003C0000200003005040420F0051
:1087900030B504680C40944206D1013B002BF8D15F
:1087A00012E0013B002B0FD004680C409442F8D13A
:1087B000002405680D40954204D101349C42F8D153
:1087C000002002E0201C00E0181C30BD0D4BE02210
:1087D00083F811234FF40032C3F880211A604FF060
:1087E00080430122C3F818259A6003F588330021DD
:1087F000C3F808150221C3F80413C3F844131A6020
:10880000704700BF00E100E0014B1860704700BFF7
:10881000580000200228064A064B1BBF00211160A9
:108820000121012212BF1A6011601860704700BF59
:10883000F87C012054000020222837B50CD84B4B7F
:1088400053F82030052B00F0828007D8032B12D07C
:108850007BD8022B00F08180002074E01D2B78D0A3
:1088600003D81C2BF8D1052206E01E2B73D01F2B3A
:10887000F2D1082200E002223D4B196808296EDD82
:108880000A296FDD0D29B5BF0C240E240223032312
:108890003848C0F8F0350123C0F8003500200546FF
:1088A000030103F1804303F5E04301300828C3F8D6
:1088B0001455C3F81055F3D12F4B18682F4B1B6874
:1088C00000021B0303F4805300F4E0601843294BBB
:1088D000C3F81805C3F81425C3F810250DF10602D6
:1088E000C3F82C260122C3F830261A60D3F80021E1
:1088F000002AFBD00022C3F8002101225A601D4B40
:108900001A46D3F804010028FBD00020C3F8040164
:1089100001209860D2F81431002BFBD00023C2F85C
:108920001431BDF906209A42124AB8BFADF806309C
:10893000A142C2F80035BDF9060004D035BF611A66
:10894000091BC840884003B030BD032294E70422CD
:1089500092E7062290E707228EE701228CE708249F
:10896000002395E70A24012392E700BF80D8000086
:10897000500000200070004054000020F87C0120CE
:10898000222830B53CD8224B53F82000214B00223E
:108990001D4653F82240B4F1FF3F32D11E4C45F83A
:1089A00022006FEA41411D4D1D4B246853F82230CF
:1089B0006FEA514125F81210012101FA04F4C3F8BD
:1089C0006005013CC3F8640505EB4202C3F8680585
:1089D000C3F86C050020C3F80015C3F80C05C3F8F4
:1089E0000405C3F80845C3F81405C3F81005C3F817
:1089F0002025C3F82415C3F82815C3F82C05996061
:108A000030BD8442CAD00132042AC2D1F8E700BF87
:108A100080D800004000002058000020F07C012099
:108A20003CD90000222815D8114B124A53F82030A7
:108A300013F0200F08BF4FF0A04203F01F030329DB
:108A400008D8DFE801F00210080C03F5E0730021FC
:108A500042F82310704703F5E0730C21F8E703F5A3
:108A6000E0730421F4E703F5E0730321F0E700BFAE
:108A700080D8000000030050222813D80A4B53F876
:108A800020000A4B10F0200F4FF0010200F01F00F1
:108A900008BF4FF0A043824011B9C3F80C257047BE
:108AA000C3F80825704700BF80D8000000030050BD
:108AB000222810D8094B0A4A53F8203013F0200F0F
:108AC00008BF4FF0A04203F01F03D2F81005D840B2
:108AD00000F0010070470020704700BF80D8000000
:108AE000000300502DE9F04106460D4601EB020857
:108AF0000C464445A4EB050707D0336814F8011B66
:108B00001B68304698470028F3D13846BDE8F0810D
:108B10002DE9F041C1F30A57A7F2FF35132D82B0BA
:108B200002460B460C464FEAD178064633DC002D50
:108B30004EDB3C49294103EA0100104326D0490895
:108B40000B4052EA03060CD04FF48023132D24EA85
:108B5000010143FA05F444EA01040CBF4FF000465A
:108B60000026314901EBC8082346D8E900453246C2
:108B70002046294601F020FBCDE9000122462B4684
:108B8000DDE9000101F016FB02460B4610461946CE
:108B900002B0BDE8F081332D07DDB5F5806FF5D16A
:108BA00001F00AFB02460B46F0E7A7F213474FF02D
:108BB000FF31F9400842E9D049080842D1D04FF0CE
:108BC000804320EA010143FA07F741EA0706C8E7B4
:108BD00021F000410143D9D0C3F3130101434E42B8
:108BE0000E43114D5C0C360B640406F4002305EBB8
:108BF000C80243EA0401D2E900450B460246294671
:108C0000204601F0D9FACDE9000122462B46DDE9E4
:108C1000000101F0CFFA21F00041024641EAC87399
:108C2000B4E700BFFFFF0F0050D90000F8B5C1F353
:108C30000A57A7F2FF35132D02460B460C4610DCEF
:108C4000002D29DB8C461D4929410B422AD04FF4C7
:108C500000242C41644424EA0104002621463046C5
:108C6000F8BD332D05DDB5F5806F1ED010461946D1
:108C7000F8BDA7F213474FF0FF3121FA07F738424A
:108C8000F4D00123C5F1330503FA05F5461928BFD1
:108C9000E41826EA0706E1E7013501F0004407D0B1
:108CA0000026DBE70028D2D1E0E701F085FAF8BD25
:108CB00044F07F5444F440140026CFE7FFFF0F0038
:108CC00030B51F4A21F00043934287B01CDD1D4A96
:108CD000934205DD02460B4601F06CFA07B030BD49
:108CE00002AA00F091F800F003000128DDE9042356
:108CF00012D002281CD0A0B1DDE9020100F068FB0F
:108D000001F1004107B030BD002300930022002391
:108D100001F086F807B030BDDDE9020100F058FB34
:108D2000DCE70124DDE90201009401F079F8D5E7E0
:108D30000124DDE90201009401F072F8E0E700BFD0
:108D4000FB21E93FFFFFEF7F2DE9F04F8BB0044699
:108D50000D4600F07BFA294B93F900A0BAF1FF3FD2
:108D600006460F4612D022462B462046294601F0E1
:108D700073FE834650B94FF000084FF000092046BB
:108D8000294642464B4601F03FFE20B9304639465F
:108D90000BB0BDE8F08F0122194BCDF820B0009246
:108DA000CDE90445CDE902450193BAF1000F17D092
:108DB00042464B464046494601F0DEFCBAF1020FFE
:108DC000CDE906010ED101F0A3FE21230360089B2B
:108DD00073B9DDE90667304639460BB0BDE8F08F60
:108DE000CDE90689684601F057F90028EFD1EAE796
:108DF00001F08EFE089B0360EBE700BF5C000020E3
:108E000060D90000000000002DE9F047CA4B21F0B6
:108E100000479F4290B08046894640F38F80C74B01
:108E20009F420C46924626DC0029B9A3D3E90023D1
:108E300040F38F8001F0BEF9C14B9F4204460D46BE
:108E400000F04781B4A3D3E9002301F0B3F902464F
:108E50000B46CAE900232046294601F0ABF9AEA330
:108E6000D3E9002301F0A6F90125CAE90201284649
:108E700010B0BDE8F087B34B9F4240F38980B24BFE
:108E80009F4200F31C813D15A5F21645A7EB055343
:108E900019461F46064601F0F5FD01F0D9FA804655
:108EA000894642464B4630463946CDE90A8901F0AB
:108EB00081F90022A54B01F035FB8946804601F07F
:108EC000E1FD01F0C5FA06460F4632463B464046F4
:108ED0004946CDE90C6701F06DF900229B4B01F08A
:108EE00021FB00220023CDE90E0101F083FD0028C3
:108EF00000F06081002330463946002201F07AFDFF
:108F0000002814BF01230223914A019202212A461C
:108F100000910AA8514600F083FB002C054614DAA4
:108F2000DAF80420DAF80C3002F1004203F10043D1
:108F30004542CAF80420CAF80C3006E0002000219F
:108F4000C2E90089C2E902010025284610B0BDE847
:108F5000F08701F031F97A4B9F4204460D4600F04C
:108F60000B816DA3D3E9002301F026F902460B46DD
:108F7000CAE900232946204601F01CF966A3D3E97B
:108F8000002301F019F94FF0FF35CAE90201DCE7CF
:108F900000F0FCFF62A3D3E900238046894601F07C
:108FA000C1FA00226B4B01F007F901F06BFD054699
:108FB00001F04EFA56A3D3E90023CDE9060101F0F2
:108FC000B1FA02460B464046494601F0F3F852A377
:108FD000D3E9002380468946DDE90601CDE902890F
:108FE00001F0A0FA1F2D02460B46CDE9042340F301
:108FF000B380DDE90423DDE9020101F0DBF88046FE
:1090000089463F15C9F30A53FB1A102B40F3B18070
:1090100045A3D3E90023DDE9060101F083FA804688
:10902000894602460B46DDE9020101F0C3F802461B
:109030000B46DDE90201CDE9082301F0BBF8424609
:109040004B4601F0B7F83AA3D3E90023804689469E
:10905000DDE9060101F066FA42464B4601F0AAF846
:109060000B46CDE904010246DDE9080101F0A2F852
:10907000C1F30A53FF1A312F8046894600F39C80C2
:109080009DED087BCAE900898DED027B42464B4687
:10909000DDE9020101F08EF8DDE9042301F08AF830
:1090A000002CCAE90201BFF650AF09F1004401F1FA
:1090B00000436D42CAE90084CAE9020345E702465B
:1090C0000B4601F077F80025CAE90201CAE9000160
:1090D0003BE715A3D3E9002301F06CF814A3D3E90F
:1090E00000230D46044601F065F802460B46CAE926
:1090F00000232946204601F05DF80DA3D3E90023A3
:1091000001F058F80125CAE902011EE7AFF300801B
:1091100000004054FB21F93F3163621A61B4D03D35
:1091200083C8C96D305FE43F0000601A61B4D03D70
:109130007370032E8A19A33BFB21E93F7BD90240C0
:10914000FB21F93FFB213941FFFFEF7F0000704118
:10915000E8D900000000E03F4046494601F02AF807
:10916000394B6A1E804653F82230BB4289463FF491
:1091700048AFCAE9008989E72BA3D3E9002301F0AE
:109180001BF82BA3D3E900230D46044601F014F885
:1091900002460B46CAE900232946204601F00AF898
:1091A00023A3D3E9002301F007F84FF0FF35CAE904
:1091B0000201CAE60323A7E61FA3D3E90023DDE9E2
:1091C000060101F0AFF906460F4602460B46DDE9FF
:1091D000080100F0EFFF8046894602460B46DDE9B4
:1091E0000801CDE9028900F0E5FF32463B4600F078
:1091F000E1FF13A3D3E9002306460F46DDE906018C
:1092000001F090F932463B4600F0D4FF02460B468F
:1092100040464946CDE9042300F0CCFF804689460C
:10922000A7E700BFAFF300800000601A61B4D03D33
:109230007370032E8A19A33B0000002E8A19A33BEA
:10924000C14920259A837B3968D900005E4A8A4348
:109250002DE9F04104460D4600F0958000290B46AB
:109260000646844656DD0F1500F0A580C3F31303B0
:10927000A7F2FF3743F480134FEADC72F80702EBE2
:1092800043034FEA4C0504D5ED0F05EB43034FEACA
:109290008C0500267F10B44616224FF400110CEB0B
:1092A000010098424FEAD5744FEA450503DC1B1ACA
:1092B00000EB010C0E44013A04EB43034FEA510169
:1092C000EDD11046964620244FF0004209E051D0DF
:1092D0005B00013C03EBD5734FEA52024FEA4505B0
:1092E00037D0634502EB0E01F1DD002901EB020EE0
:1092F0000ADBE046A3EB0C03A94288BF03F1FF336E
:109300006D1A1044C446E3E7BEF1000FF1DB0CF127
:109310000108EFE721F00042024329D0002942D1A1
:109320000146CA0A153B4905002AFAD012F48010FA
:1093300001D044E060465200D40200F1010CF9D59E
:10934000CCF1200401FA0CFCE1401F1A41EA0203AF
:109350008CE72B4321D14408731003F17F53F207AC
:1093600003F5001348BF44F0004403EB07512046C7
:10937000BDE8F081A942ABD8002901EB020EC3DBA6
:1093800098460023BCE702460B4601F0CBF8224684
:109390002B4600F011FFBDE8F081411C16BF421CB6
:1093A00001365408D8E7024600F004FF02460B4697
:1093B00001F0E2F9DCE71A4631463B46B6E78C4657
:1093C00020244FF0FF30BFE70000F07F00000000D6
:1093D0002DE9F04F21F00048B8F1795F85B00646DD
:1093E0000F4692469B466BDA01F04CFB002800F0DA
:1093F000E18032463B463046394601F093F874A38B
:10940000D3E9002304460D4601F08CF872A3D3E99A
:10941000002300F0D1FE22462B4601F083F870A312
:10942000D3E9002300F0C6FE22462B4601F07AF86D
:109430006DA3D3E9002300F0BFFE22462B4601F0C6
:1094400071F86BA3D3E9002300F0B4FE22462B464B
:1094500001F068F868A3D3E9002300F0ADFE2246CE
:109460002B4601F05FF8CDE900010022664B204653
:10947000294601F057F8DDE9002380468946204659
:10948000294601F04FF8524604460D465B463046E9
:10949000394601F047F802460B462046294600F0BF
:1094A00089FE02460B464046494600F083FE0246CE
:1094B0000B460020554900F07DFE05B0BDE8F08F59
:1094C00002460B4601F02EF841A3D3E900230446DF
:1094D0000D4601F027F840A3D3E9002300F06CFE0D
:1094E00022462B4601F01EF83DA3D3E9002300F0ED
:1094F00061FE22462B4601F015F83BA3D3E9002379
:1095000000F05AFE22462B4601F00CF838A3D3E9AE
:10951000002300F04FFE22462B4601F003F836A34D
:10952000D3E9002300F048FE2B46224600F0FAFF64
:10953000374B9845CDE9000197DD364B98453EDC29
:10954000A8F500130022002030499046994600F00B
:1095500031FECDE9020100222B4B2046294600F0C6
:10956000E1FF42464B4600F025FEDDE90023804640
:1095700089462046294600F0D5FF524604460D464E
:109580005B463046394600F0CDFF02460B4620468A
:10959000294600F00FFE02460B464046494600F0C1
:1095A00009FE02460B46DDE9020100F003FE05B0AC
:1095B000BDE8F08F1549002005B0BDE8F08F9FEDA4
:1095C000107B4FF000088DED027BDFF84C90C2E776
:1095D000D43888BEE9FAA8BDC4B1B4BD9EEE213E20
:1095E000AD529C804F7E923E9015CB19A001FA3E61
:1095F0007751C1166CC1563F4C5555555555A53F31
:10960000000000000000E73F0000E03F0000F03FE6
:109610003233D33F0000E93F0000D23F000000009A
:109620002DE9F04FADF5197DBE4CA29EBE4D54F80C
:1096300026600793D41E85FB0475E417C4EBA504CC
:1096400024EAE4741D46631CA3EB8303013D02EB93
:10965000C3030593731904960994019503900B9124
:10966000A4EB05071AD43B44002400255E1C0DF131
:109670008008DDF88C9208E059F8270000F0E8FE39
:109680000137B742E8E8020108D0002FF4DA0137C9
:1096900020462946B742E8E80201F6D1049B002B98
:1096A000079B4FEAC30302932ADB039A20A902EB2C
:1096B000030801EB0309049B72AA02EBC30B0DF52F
:1096C000E07A019B002B4FF000064FF0000711DB02
:1096D000039C4D4675E90223F4E8020100F022FFE5
:1096E00002460B463046394600F066FD44450646C4
:1096F0000F46EFD1EAE80267DA4509F10809E0D13F
:10970000DDE90204049920448B0082460BA8A3F1F2
:109710000802C31808930CAB13440A938B4698AB0A
:1097200003EBCB03BBF1000F53E9284529DD70ABF8
:1097300003EBCB080DF1300900227C4B2046294673
:1097400000F0F0FE01F09EF900F082FE0022784B5E
:1097500006460F4600F0E6FE02460B462046294626
:1097600000F028FD01F08EF978E9022349F8040B96
:109770003946304600F020FD70AB984504460D4652
:10978000DAD1DDF81490204629464A4600F088FCDC
:1097900000224FF07F5304460D4600F0C3FE00F058
:1097A000FBFB0022634B00F0BDFE02460B46204649
:1097B000294600F0FFFC0D46044601F063F980469F
:1097C00000F046FE0B4602462946204600F0F2FC19
:1097D0004B46002B06460F4640F3E1800BF1FF326B
:1097E0000CA9C9F1180351F8225045FA03F101FA06
:1097F00003F30CA8EB1A40F82230C9F1170588448E
:1098000043FA05F5002D2CDDBBF1000F08F101082E
:1098100040F381820C9C002C40F0A780BBF1010F2B
:109820000AD00CA9012251F8044F531C002C40F01F
:109830009E809B451A46F6D1059B002B0EDD012B21
:1098400000F0D980022B09D10BF1FF320CAB0CA92F
:1098500053F82230C3F3150341F82230022D00F0F3
:10986000AF80002200233046394601F0C3F80028BB
:1098700000F05382049B0BF1FF394B4510DC0BF1D8
:1098800080430CAA013B089802EB8303002253F8A3
:109890000419834242EA0102F9D1002A40F0B6805D
:1098A000049B0CAA013B52F82330002B40F0A1800E
:1098B0000A9A012352F8041901330029FAD05B44B3
:1098C0000BF10109994506934CDC099A079909EBBC
:1098D000020801EB0B0508F1804802EB030BA39B88
:1098E00008F1FF3803EB880870AB03EBC909A39BB1
:1098F00020A903EB8B0301EBC505029358F8040F75
:1099000000F0A6FD0B4601990246002905F1080B5F
:10991000C5E900234FF000064FF000071CDB039C55
:109920000CE000BF30DB0000ABAAAA2A0000703EAA
:10993000000070410000204075E90223F4E80201B4
:1099400000F0F0FD02460B463046394600F034FC8C
:10995000544506460F46EFD1029B9845E9E8026759
:109960005D46CBD1DDF818B0D9E6012300220CA961
:10997000C4F180749B4541F822400EDD51F823204C
:1099800001EB8B0001EB83036FF07F4100E01A686D
:109990008A1A43F8042B8342F9D101244CE706D1FB
:1099A0000BF1FF330CAA52F82350ED152AE70022E1
:1099B0007B4B01F03DF8002840F0A381054650E7BD
:1099C00032463B460020774900F0F4FB06460F463E
:1099D000002C3FF446AF059A7249002000F060FB6E
:1099E00002460B463046394600F0E4FB06460F4679
:1099F00037E7012363E70BF1FF320CAB0CA953F8F7
:109A00002230C3F3160341F8223027E70CAB059A46
:109A100053F82930183ACDE9068505926BB909F15A
:109A20008043013B0CA901EB830353F8041909F1AE
:109A3000FF39183A0029F8D00592059A59490020B3
:109A400000F02EFBB9F1000F04460D46C0F2C081B4
:109A50004FEAC90370AA02EB030808930CAB03EBAF
:109A60008906DFF844B14FF0000A08F10807043610
:109A700056F8040D00F0ECFC22462B4600F052FD97
:109A80005B4667E9020152462046294600F04AFD3E
:109A90000CAB9E4204460D46EAD148AB03930193BA
:109AA000CDF8149009F10103DDF810900293C3463C
:109AB0004FF0000AB9F1000FC0F22A81DFF8EC8004
:109AC0005D4635A3D3E9002300260027002403E0E8
:109AD000544510DCF8E80223F5E8020100F022FD0D
:109AE00002460B463046394600F066FB0134A1457C
:109AF00006460F46ECDA019BE3E802670193029BFE
:109B00000AF1010A9A45ABF1080BD3D1A29BDDF80B
:109B10001490032B39D8DFE813F0D90006000600B3
:109B20004D0048AB0393B9F1000F4FF000004FF028
:109B3000000109DB039D05EBC904083474E9022325
:109B400000F03AFBA542F9D1079B002B40F01E81A3
:109B50000B9BC3E900010B4603990246D1E90001C2
:109B600000F028FBB9F1000F0CDD4AAD01240134EF
:109B7000F5E8022300F020FBA145F8DA079B002B53
:109B800040F014810B9BC3E90201069B03F0070020
:109B90000DF5197DBDE8F08F00000040FB21F93F75
:109BA0000000E03F0000F03F0000703EF8DA0000E7
:109BB00048AB0393B9F1000F40F32781039ACDF826
:109BC00010904FEAC9030193D318D3E900AB09F110
:109BD0000053013B02EBC9080293914678E9026702
:109BE00052465B463046394600F0E6FA04460D46DA
:109BF00002460B463046394600F0DCFA52465B46D8
:109C000000F0DAFAC145A246AB46C8E90201C8E94C
:109C10000045E3D1DDF81090B9F1010F40F3F58074
:109C2000019B039A02991344C900D3E9006701F12B
:109C3000080A019192440DF5947B7AE90289324633
:109C40003B464046494600F0B7FA04460D460246F8
:109C50000B464046494600F0ADFA32463B4600F01E
:109C6000ABFAD34526462F46CAE90201CAE90045A8
:109C7000E3D1019C039B1034002000211C4403F11C
:109C8000100574E9022300F097FAA542F9D1039C6C
:109C9000079ED4E90023D4E90245002E00F08A8013
:109CA00003F1004701F100430B99C1E90403069B4E
:109CB0002646944605F1004403F00700C1E900C7B9
:109CC000C1E902640DF5197DBDE8F08F089C039D84
:109CD0000834002000212C4474E9022300F06CFABF
:109CE000A542F9D1079B13B101F1004319460B9B23
:109CF000C3E90001069B03F007000DF5197DBDE8DF
:109D0000F08FBBF1000F08F1010874DD022581E539
:109D100000260027EFE600248EE5CDE90685059DA7
:109D2000304639466A4200F0BBF90022384B0646FD
:109D30000F4600F07DFE00B30022364B3046394618
:109D400000F0F0FB00F09EFE044600F081FB0022D4
:109D50002F4B00F0E7FB0B4602463946304600F039
:109D600029FA00F08FFE0BF101090CAB183543F80E
:109D70002B00059543F829405FE63046394600F050
:109D800081FE0CABD94643F82B0056E60B9C01F143
:109D90000043C4E900030B4603990246D1E90001E0
:109DA00000F008FAB9F1000F3FF7DFAE01F1004310
:109DB0001946E7E60B9EC6E90023069BC6E90401A7
:109DC00003F00700C6E902450DF5197DBDE8F08FE7
:109DD000A29B032B3FF6D9AE01A252F823F000BF9D
:109DE000F19D0000239B0000239B0000B19B00001D
:109DF0000020002176E732463B460020064900F06D
:109E0000D9F9022506460F462BE5002000213EE742
:109E1000000070410000703E0000F03F00000000B4
:109E20002DE9F04F21F00046B6F1795F85B0044688
:109E30000D469046994604DA00F024FE002800F012
:109E4000858022462B462046294600F06BFB0646BD
:109E50000F4602460B462046294600F063FB41A30D
:109E6000D3E9002382468B463046394600F05AFB40
:109E70003EA3D3E9002300F09DF932463B4600F0B3
:109E800051FB3CA3D3E9002300F096F932463B4650
:109E900000F048FB39A3D3E9002300F08BF93246E8
:109EA0003B4600F03FFB37A3D3E9002300F084F9E1
:109EB0000E9BCDE900019BB30022294B4046494649
:109EC00000F030FBDDE90023CDE9020150465946A0
:109ED00000F028FB02460B46DDE9020100F06AF9BA
:109EE00032463B4600F01EFB42464B4600F062F90C
:109EF00019A3D3E9002306460F465046594600F001
:109F000011FB02460B463046394600F055F9024631
:109F10000B462046294600F04DF905B0BDE8F08F0C
:109F200002460B463046394600F0FCFA0AA3D3E954
:109F3000002300F03FF952465B4600F0F3FA224658
:109F40002B4600F039F905B0BDE8F08F20462946D0
:109F500005B0BDE8F08F00BF495555555555C53F73
:109F60000000E03F7CD5CF5A3AD9E53DEB9C2B8AE7
:109F7000E6E55A3E7DFEB157E31DC73ED561C119E6
:109F8000A0012A3FA6F810111111813F21F00043D2
:109F900019467047000000002DE9F041C1F30A574F
:109FA000A7F2FF35132D02460B460C46884606469F
:109FB0001DDC002D3CDB364F2F4101EA070C5CEA2B
:109FC000000C19D030A3D3E9002300F0F5F80022EB
:109FD000002300F037FDC8B3002C04DA4FF48013DF
:109FE00043FA05F5A84428EA070400262EE0332D9D
:109FF00006DDB5F5806F2DD010461946BDE8F0811D
:10A00000A7F213474FF0FF3C2CFA07F70742F3D0B3
:10A010001DA3D3E9002300F0CFF80022002300F0B5
:10A0200011FD98B1002C21DB26EA070644460DE01D
:10A0300015A3D3E9002300F0BFF80022002300F0AD
:10A0400001FD18B1002C08DB0026344621463046BD
:10A05000BDE8F08100F0B0F8D0E724F000430D4AED
:10A060001E43002E18BF14460026EFE7142D08D01B
:10A070000123C5F1340503FA05F5AE1928BF98444C
:10A08000D2E704F10108CFE79C7500883CE4377EF5
:10A09000FFFF0F000000F0BF00207047000000002D
:10A0A000F8B5C1F30A5304460D460E4617460BBBDE
:10A0B00021F00046034633431BD0354B002200F00D
:10A0C00031FA344B9F4204460D4635DBC1F30A5347
:10A0D0000E46363B3B4440F2FE72934232DC002B8C
:10A0E00011DD26F0FF4626F4E00646EA0355204639
:10A0F0002946F8BD40F2FF729342EBD102460B466F
:10A1000000F05AF8F8BD13F1350F28DA4CF250334D
:10A110009F4222462B460ADD19A1D1E9000100F039
:10A120003DF817A3D3E9002300F0FCF9F8BD16A110
:10A13000D1E9000100F032F813A3D3E9002300F0C5
:10A14000F1F9F8BD22462B460DA1D1E9000100F03E
:10A1500025F80BA3D3E9002300F0E4F9F8BD26F0BD
:10A16000FF4626F4E006363346EA035520462946E4
:10A170000022094B00F0D6F9F8BD00BFAFF3008014
:10A180009C7500883CE4377E59F3F8C21F6EA50128
:10A1900000005043B03CFFFF0000903C03F0004340
:10A1A00021F0004242EA0301704700BF81F0004104
:10A1B00002E000BF83F0004330B54FEA41044FEAAC
:10A1C000430594EA050F08BF90EA020F1FBF54EA47
:10A1D000000C55EA020C7FEA645C7FEA655C00F0E3
:10A1E000E2804FEA5454D4EB5555B8BF6D420CDDB4
:10A1F0002C4480EA020281EA030382EA000083EA37
:10A20000010180EA020281EA0303362D88BF30BDD6
:10A2100011F0004F4FEA01314FF4801C4CEA11312C
:10A2200002D0404261EB410113F0004F4FEA03338B
:10A230004CEA133302D0524263EB430394EA050F16
:10A2400000F0A780A4F10104D5F1200E0DDB02FA85
:10A250000EFC22FA05F2801841F1000103FA0EF219
:10A26000801843FA05F359410EE0A5F120050EF1DF
:10A27000200E012A03FA0EFC28BF4CF0020C43FA10
:10A2800005F3C01851EBE37101F0004507D54FF01D
:10A29000000EDCF1000C7EEB00006EEB0101B1F56D
:10A2A000801F1BD3B1F5001F0CD349085FEA3000B3
:10A2B0004FEA3C0C04F101044FEA445212F5800FBE
:10A2C00080F09A80BCF1004F08BF5FEA500C50F15B
:10A2D000000041EB045141EA050130BD5FEA4C0C3E
:10A2E000404141EB010111F4801FA4F10104E9D1C7
:10A2F00091F0000F04BF01460020B1FA81F308BFBE
:10A300002033A3F10B03B3F120020CDA0C3208DD89
:10A3100002F1140CC2F10C0201FA0CF021FA02F164
:10A320000CE002F11402D8BFC2F1200C01FA02F1D4
:10A3300020FA0CFCDCBF41EA0C019040E41AA2BFF9
:10A3400001EB0451294330BD6FEA04041F3C1CDAC1
:10A350000C340EDC04F11404C4F1200220FA04F0E1
:10A3600001FA02F340EA030021FA04F345EA03018B
:10A3700030BDC4F10C04C4F1200220FA02F001FA4D
:10A3800004F340EA0300294630BD21FA04F02946CF
:10A3900030BD94F0000F83F4801306BF81F4801168
:10A3A0000134013D4EE77FEA645C18BF7FEA655CDB
:10A3B00029D094EA050F08BF90EA020F05D054EAAD
:10A3C000000C04BF1946104630BD91EA030F1EBFB2
:10A3D0000021002030BD5FEA545C05D140004941B6
:10A3E00028BF41F0004130BD14F580043CBF01F5A9
:10A3F000801130BD01F0004545F0FE4141F470018F
:10A400004FF0000030BD7FEA645C1ABF1946104669
:10A410007FEA655C1CBF0B46024650EA013406BF6A
:10A4200052EA033591EA030F41F4002130BD00BF29
:10A4300090F0000F04BF0021704730B54FF48064E6
:10A4400004F132044FF000054FF0000150E700BF67
:10A4500090F0000F04BF0021704730B54FF48064C6
:10A4600004F1320410F0004548BF40424FF00001B3
:10A470003EE700BF42004FEAE2014FEA31014FEAF6
:10A4800002701FBF12F07F4393F07F4F81F0605145
:10A49000704732F07F4208BF704793F07F4F04BF90
:10A4A00041F40021704730B54FF4607401F000456D
:10A4B00021F000411CE700BF50EA010208BF7047CD
:10A4C00030B54FF000050AE050EA010208BF7047BE
:10A4D00030B511F0004502D5404261EB41014FF427
:10A4E000806404F132045FEA915C3FF4D8AE4FF02F
:10A4F00003025FEADC0C18BF03325FEADC0C18BF12
:10A50000033202EBDC02C2F1200300FA03FC20FA62
:10A5100002F001FA03FE40EA0E0021FA02F11444AF
:10A52000BDE600BF70B54FF0FF0C4CF4E06C1CEAC8
:10A5300011541DBF1CEA135594EA0C0F95EA0C0F39
:10A5400000F0DEF82C4481EA030621EA4C5123EAAC
:10A550004C5350EA013518BF52EA033541F48011DB
:10A5600043F4801338D0A0FB02CE4FF00005E1FB8E
:10A5700002E506F00042E0FB03E54FF00006E1FBD8
:10A5800003569CF0000F18BF4EF0010EA4F1FF041B
:10A59000B6F5007F64F5407404D25FEA4E0E6D415B
:10A5A00046EB060642EAC62141EA55514FEAC5206C
:10A5B00040EA5E504FEACE2EB4F1FD0C88BFBCF5E8
:10A5C000E06F1ED8BEF1004F08BF5FEA500E50F199
:10A5D000000041EB045170BD06F0004646EA01015F
:10A5E00040EA020081EA0301B4EB5C04C2BFD4EB91
:10A5F0000C0541EA045170BD41F480114FF0000E8A
:10A60000013C00F3AB8014F1360FDEBF002001F0F7
:10A61000004170BDC4F10004203C35DA0C341BDC71
:10A6200004F11404C4F1200500FA05F320FA04F043
:10A6300001FA05F240EA020001F0004221F0004177
:10A6400010EBD37021FA04F642EB06015EEA430EEA
:10A6500008BF20EAD37070BDC4F10C04C4F120051A
:10A6600000FA04F320FA05F001FA04F240EA0200CD
:10A6700001F0004110EBD37041F100015EEA430E9E
:10A6800008BF20EAD37070BDC4F1200500FA05F2BE
:10A690004EEA020E20FA04F301FA05F243EA02033D
:10A6A00021FA04F001F0004121FA04F220EA02004C
:10A6B00000EBD3705EEA430E08BF20EAD37070BD92
:10A6C00094F0000F0FD101F00046400041EB010172
:10A6D00011F4801F08BF013CF7D041EA060195F054
:10A6E000000F18BF704703F00046520043EB03030E
:10A6F00013F4801F08BF013DF7D043EA06037047FB
:10A7000094EA0C0F0CEA135518BF95EA0C0F0CD005
:10A7100050EA410618BF52EA4306D1D181EA03014B
:10A7200001F000414FF0000070BD50EA410606BF45
:10A730001046194652EA430619D094EA0C0F02D18A
:10A7400050EA013613D195EA0C0F05D152EA0336CF
:10A750001CBF104619460AD181EA030101F00041ED
:10A7600041F0FE4141F470014FF0000070BD41F036
:10A77000FE4141F4780170BD70B54FF0FF0C4CF410
:10A78000E06C1CEA11541DBF1CEA135594EA0C0F2F
:10A7900095EA0C0F00F0A7F8A4EB050481EA030E7C
:10A7A00052EA03354FEA013100F088804FEA033363
:10A7B0004FF0805545EA131343EA12634FEA022231
:10A7C00045EA111545EA10654FEA00260EF00041F2
:10A7D0009D4208BF964244F1FD0404F5407402D244
:10A7E0005B084FEA3202B61A65EB03055B084FEAD5
:10A7F00032024FF480104FF4002CB6EB020E75EBD2
:10A80000030E22BFB61A754640EA0C005B084FEAF9
:10A810003202B6EB020E75EB030E22BFB61A754676
:10A8200040EA5C005B084FEA3202B6EB020E75EBC1
:10A83000030E22BFB61A754640EA9C005B084FEA39
:10A840003202B6EB020E75EB030E22BFB61A754646
:10A8500040EADC0055EA060E18D04FEA051545EA35
:10A8600016754FEA06164FEAC30343EA52734FEADE
:10A87000C2025FEA1C1CC0D111F4801F0BD141EA57
:10A8800000014FF000004FF0004CB6E711F4801FBC
:10A8900004BF01430020B4F1FD0C88BFBCF5E06F9C
:10A8A0003FF6AFAEB5EB030C04BFB6EB020C5FEAAC
:10A8B000500C50F1000041EB045170BD0EF0004E01
:10A8C0004EEA113114EB5C04C2BFD4EB0C0541EA33
:10A8D000045170BD41F480114FF0000E013C90E630
:10A8E00045EA060E8DE60CEA135594EA0C0F08BFF4
:10A8F00095EA0C0F3FF43BAF94EA0C0F0AD150EAF3
:10A9000001347FF434AF95EA0C0F7FF425AF104685
:10A9100019462CE795EA0C0F06D152EA03353FF4AD
:10A92000FDAE1046194622E750EA410618BF52EA2A
:10A9300043067FF4C5AE50EA41047FF40DAF52EAFE
:10A9400043057FF4EBAE12E74FF0FF3C06E000BF9B
:10A950004FF0010C02E000BF4FF0010C4DF804CDA8
:10A960004FEA410C7FEA6C5C4FEA430C18BF7FEA68
:10A970006C5C1BD001B050EA410C0CBF52EA430C96
:10A9800091EA030F02BF90EA020F0020704710F116
:10A99000000F91EA030F58BF994208BF90422CBFA5
:10A9A000D8176FEAE37040F0010070474FEA410C9E
:10A9B0007FEA6C5C02D150EA013C07D14FEA430CBC
:10A9C0007FEA6C5CD6D152EA033CD3D05DF8040B2D
:10A9D000704700BF8446104662468C46194663465F
:10A9E00000E000BF01B5FFF7B7FF002848BF10F136
:10A9F000000F01BD4DF808EDFFF7F4FF0CBF01207B
:10AA000000205DF808FB00BF4DF808EDFFF7EAFFF6
:10AA100034BF012000205DF808FB00BF4DF808EDB1
:10AA2000FFF7E0FF94BF012000205DF808FB00BFA6
:10AA30004DF808EDFFF7CEFF94BF012000205DF830
:10AA400008FB00BF4DF808EDFFF7C4FF34BF01203D
:10AA500000205DF808FB00BF4FEA410C7FEA6C5C08
:10AA600002D150EA013C0AD14FEA430C7FEA6C5C08
:10AA700002D152EA033C02D14FF0000070474FF080
:10AA8000010070474FEA410212F5001215D211D5AC
:10AA90006FF47873B3EB625212D94FEAC12343F0DB
:10AAA000004343EA505311F0004F23FA02F018BF5D
:10AAB000404270474FF00000704750EA013005D126
:10AAC00011F0004008BF6FF0004070474FF00000E9
:10AAD000704700BF1FB51C46094B1B680546D86868
:10AAE00052B1084B0091CDE9013207492B4622466D
:10AAF00000F028F800F0BAFD044B1A46F2E700BF58
:10AB00006000002040DB00004DDB0000F9C70000C2
:10AB1000014B1868704700BF6000002008B5074B64
:10AB2000044613B10021AFF30080054B1868836A17
:10AB300003B19847204601F075FB00BF00000000FC
:10AB40007CDB00000EB403B5014603AB054853F8A7
:10AB5000042B0068019300F081F802B05DF804EB6B
:10AB600003B070476000002070B50D4E0D4CA41B63
:10AB7000A4100025A54209D10B4E0C4C01F054FB4A
:10AB8000A41BA4100025A54205D170BD56F82530A0
:10AB900098470135EEE756F8253098470135F2E73A
:10ABA000300200203002002030020020400200204D
:10ABB00010B5431E0A44914200D110BD11F8014B5B
:10ABC00003F8014FF7E7884210B501EB020307D8FD
:10ABD000421E99420AD011F8014B02F8014FF8E7E2
:10ABE0008342F5D98118D21AD34200D110BD13F88F
:10ABF000014D01F8014DF7E702440346934200D1AD
:10AC0000704703F8011BF9E79368013B002B10B470
:10AC1000936008DA9469A34201DB0A2903D15DF845
:10AC2000044B00F063BC1368581C10601970084690
:10AC30005DF8044B7047F8B506460F461446D51824
:10AC4000AC4201D1002007E03A4614F8011B30461F
:10AC5000FFF7DAFF431CF3D1F8BD00002DE9F04FF8
:10AC60009DB00C4617460393064618B183690BB98D
:10AC700000F0F4FD7B4B9C4257D17468A389180700
:10AC80005DD52369002B5AD00023099320238DF82A
:10AC9000293030238DF82A304FF0010BB846454655
:10ACA00015F8013B0BB1252B54D1B8EB070A0BD09B
:10ACB00053463A4621463046FFF7BDFF013000F0CB
:10ACC000C280099B5344099398F80030002B00F090
:10ACD000BA8000234FF0FF32CDE905230493079398
:10ACE0008DF853301A93A846052218F8011B5E48C8
:10ACF00000F0C6FE049B78BBD90644BF20228DF825
:10AD000053201A0744BF2B228DF853202A782A2A71
:10AD10002AD0079AA84600200A25414611F8013B8F
:10AD2000303B092B69D960B324E0504B9C4201D1E0
:10AD3000B468A3E74E4B9C4208BFF4689EE72146E7
:10AD4000304600F025FC00289ED04FF0FF301DB0AB
:10AD5000BDE8F08FA846A2E7434A801A0BFA00F03C
:10AD6000184304904546BEE7039A111D12680391EB
:10AD7000002A01DB079204E0524243F002030792EB
:10AD8000049398F800302E2B0ED198F801302A2B1E
:10AD900038D1039B1A1D1B680392002BB8BF4FF0DC
:10ADA000FF3308F102080593324D98F80010032292
:10ADB000284600F065FE40B14023401B03FA00F036
:10ADC000049B034308F10108049398F800102A48F3
:10ADD0008DF82810062208F1010700F051FE002826
:10ADE00037D0264B1BBB039B073323F007030833E5
:10ADF0000393099B4B44099350E705FB0232012062
:10AE000088468AE7002308F10108059319460A25B8
:10AE1000404610F8012B303A092A03D9002BC3D041
:10AE20000591C1E705FB012101238046F0E703AB53
:10AE300000932246124B04A93046AFF30080B0F1D4
:10AE4000FF3F8146D5D1A3895B063FF57EAF0998C8
:10AE50007DE703AB00932246094B04A9304600F07E
:10AE600087F8ECE7D4DB000080DB0000F4DB0000B7
:10AE7000B4DB000086DB00008ADB0000000000007D
:10AE800037AC00002DE9F04791461F468A680B69F0
:10AE9000DDF820809342B8BF1346C9F8003091F81E
:10AEA000432006460C4612B10133C9F8003023682E
:10AEB000990642BFD9F800300233C9F8003025683E
:10AEC00015F0060507D104F1190AE368D9F8002046
:10AED0009B1AAB4228DC94F843302268003318BF39
:10AEE000012392062DD404F1430239463046C0476F
:10AEF000013020D02368E568D9F8002003F006036C
:10AF0000042B08BFAD1AA36822690CBF25EAE575BA
:10AF100000259342C4BF9B1AED184FF000091A3464
:10AF20004D451AD1002008E00123524639463046EB
:10AF3000C047013003D14FF0FF30BDE8F087013545
:10AF4000C3E7E1185A1C302081F84300224494F8EA
:10AF5000451082F843100233C5E7012322463946E3
:10AF60003046C0470130E6D009F10109D8E70000BA
:10AF70002DE9F04301F1430C0C46097E85B06E29A2
:10AF80001746064698460C9A00F0B38022D86329EB
:10AF900036D00AD8002900F0B980582900F0838003
:10AFA00004F1420584F8421032E0642901D0692995
:10AFB000F6D120681368050603F104012AD51B6841
:10AFC0001160002B03DA2D225B4284F843206F4886
:10AFD0000A2239E0732900F09D8008D86F2920D01B
:10AFE0007029DDD1236843F02003236003E0752935
:10AFF00017D07829D4D1782384F84530644855E0B7
:10B000001368191D1B68116004F1420584F8423071
:10B0100001238CE01B68116010F0400F18BF1BB2B9
:10B02000CFE713682568181D1060280601D51B6836
:10B0300002E06806FBD51B8854486F2914BF0A221A
:10B040000822002184F843106568A560002DC0F235
:10B050009580216821F004012160002B3DD1002D55
:10B0600040F08E806546082A0BD12368DB0708D59F
:10B07000236962689A42DEBF302305F8013C05F17E
:10B08000FF35ACEB05032361CDF800803B4603AAF6
:10B0900021463046FFF7F6FE01304DD14FF0FF302C
:10B0A00005B0BDE8F083394884F84510136821687D
:10B0B0001D1D1B6815600A060BD5CA0744BF41F069
:10B0C000200121601BB9226822F020022260102298
:10B0D000B7E74D0648BF9BB2EFE76546B3FBF2F119
:10B0E00002FB1133C35C05F8013D0B460029F5D185
:10B0F000B9E7136825686169181D106028061B6888
:10B1000001D5196002E06A06FBD51980002323618E
:10B110006546B9E71368191D11601D686268002152
:10B12000284600F0ADFC08B1401B606063682361F5
:10B13000002384F84330A7E723692A46394630467E
:10B14000C0470130AAD023689B0713D4E068039B53
:10B150009842B8BF1846A3E701234A46394630460D
:10B16000C04701309AD00135E368039A9B1AAB427D
:10B17000F2DCEBE7002504F11909F5E7002BACD16F
:10B18000037884F8423004F142056CE791DB00005B
:10B19000A2DB000038B50D4B1C68A36B05467BB9DC
:10B1A000182000F04DFC0A4A0A4BA063C0E90023B6
:10B1B000094B83600B23838101220023C0E9042310
:10B1C000A36B00221D615A6138BD00BF60000020E2
:10B1D0000E33CDAB34126DE6ECDE050038B5134B03
:10B1E0001C68A36B7BB9182000F02AFC104A114B95
:10B1F000A063C0E90023104B83600B2383810122ED
:10B200000023C0E90423A16B0C480A694B690C4C6C
:10B21000504304FB0300A2FB04230344541C43F1EA
:10B220000005C1E9044525F0004038BD600000205C
:10B230000E33CDAB34126DE6ECDE05002DF4515823
:10B240002D7F954C0CB430B5174B0C1E9DB01D686E
:10B2500008DA8B232B604FF0FF301DB0BDE8304083
:10B2600002B070474FF40273ADF8143014BF04F10C
:10B27000FF332346049307934FF6FF730290069023
:10B28000ADF81630209A21AB02A92846019300F0B0
:10B290006FFD431CBCBF8B232B60002CDDD0029BB9
:10B2A00000221A70D9E700BF600000200EB400B57C
:10B2B0009CB01DAB029006906FF0004109480791C9
:10B2C0000491094953F8042B05910068019302A9E0
:10B2D00000F04EFD029B00221A701CB05DF804EBDA
:10B2E00003B07047600000200802FFFF10B503465E
:10B2F0001A785C1C3AB9013B11F8012B03F8012FB5
:10B30000002AF9D110BD2346F2E7C9B2034610F86E
:10B31000012B1AB18A42F9D118467047002918BF8B
:10B320000023F9E710F8012B11F8013B012A28BF8F
:10B330009A42F7D0D01A7047034613F8012B002A1F
:10B34000FBD1181A0138704710B56AB10139841859
:10B3500010F8013B11F8012F934203D1A04201D014
:10B36000002BF5D1981A10BD1046FCE770B50139D5
:10B37000044602B970BD234611F8015F03F8015B72
:10B38000561E2DB91444A342F4D003F8015BFAE72A
:10B390001C463246EDE7F0B503787BB104462378CE
:10B3A0002046661C7BB14A1E631E12F8015F4DB138
:10B3B00013F8017FAF423446F7D0F0E70B78002B4B
:10B3C00018BF0020F0BD1846FCE72DE9F047804685
:10B3D000894692461E460F463D46089815F8014B91
:10B3E00000F0C6FA2044437813F0080332D12D2C24
:10B3F00032D17C78BD1C0122002E5DD0102E09D1E7
:10B40000302C07D12B7803F0DF03582B4FD16C7809
:10B4100010260235002A14BF4FF000416FF00041A2
:10B420000027B1FBF6FC384606FB1C1EA4F13003D6
:10B43000092B17D81C46A64223DD7B1C07D0844568
:10B440001CD301D1A64519DB00FB0640012715F8E6
:10B45000014BEBE72F46BFE72B2C04BFBD1C7C78CC
:10B460001A46C9E7A4F14103192B01D8373CE2E79A
:10B47000A4F16103192B04D8573CDCE74FF0FF37E8
:10B48000E5E77B1C08D12223C8F800300846BAF152
:10B49000000F07D1BDE8F08702B14042BAF1000FBA
:10B4A000F8D00FB105F1FF39CAF80090F2E7302467
:10B4B000002EAFD10826ADE7302CA3D00A26A9E78D
:10B4C000084B37B51C68084D236A002B08BF2B4674
:10B4D000009313460A4601462046FFF776FF03B065
:10B4E00030BD00BF60000020C4000020F8B50E464B
:10B4F0001446054618B183690BB900F0AFF9214B2A
:10B500009C422AD16C68A369A360A3891A072ED52F
:10B51000236963B323692068C01A6369F6B2834262
:10B52000374604DC2146284600F02EF928BBA368E4
:10B53000013BA36023685A1C22601E7063690130BE
:10B54000834204D0A389DB0719D50A2E17D12146DF
:10B55000284600F019F990B10FE00B4B9C4201D145
:10B56000AC68D0E7094B9C4208BFEC68CBE72146AA
:10B57000284600F00DF80028CCD04FF0FF373846B1
:10B58000F8BD00BFD4DB0000F4DB0000B4DB00003A
:10B59000324B70B51D6806460C4625B1AB6913B930
:10B5A000284600F05BF92E4B9C420FD16C68B4F931
:10B5B0000C309AB215072CD4D00611D4092232606F
:10B5C00043F04003A3814FF0FF303EE0254B9C4207
:10B5D00001D1AC68EBE7244B9C4208BFEC68E6E77E
:10B5E000510712D5616B41B104F14403994202D075
:10B5F000304600F095FA00236363A38923F0240307
:10B60000A3810023636023692360A38943F00803B7
:10B61000A38123694BB9A38903F42073B3F5007F99
:10B6200003D02146304600F0CBF9A28912F0010385
:10B630000CD00023A36063695B42A361236953B903
:10B64000B4F90C3013F08000BAD170BD920758BF26
:10B650006369A360F2E70020F7E700BF6000002005
:10B66000D4DB0000F4DB0000B4DB000008B50620EA
:10B6700000F0ACFC012000F0D5FD00008A892DE926
:10B68000F041054610070C4658D44B68002B05DCEA
:10B690000B6C002B02DC0020BDE8F081E66A002E76
:10B6A000F9D0002312F480522F68216A2B6032D027
:10B6B000606DA3895A0705D56368C01A636B0BB127
:10B6C000236CC01A00230246E66A216A2846B04766
:10B6D000431CA38906D129681D2948D8294ACA4094
:10B6E000D60744D500226260D9042269226004D5BD
:10B6F000421C01D12B6803B96065616B2F60002982
:10B70000C9D004F14403994202D0284600F008FA57
:10B7100000206063C0E701232846B047411CC8D120
:10B720002B68002BC5D01D2B01D0162B01D12F600B
:10B73000B1E7A38943F04003A381ADE70F69002F70
:10B74000A9D093070E6808BF4B690F6018BF00238C
:10B75000A6EB07088B60B8F1000F9CDD43463A4624
:10B76000216AA66A2846B047002806DCA38943F070
:10B770004003A3814FF0FF308EE70744A8EB000899
:10B78000E9E700BF0100402038B50B6905460C46CB
:10B79000DBB118B183690BB900F060F80C4B9C4227
:10B7A00009D16C68B4F90C307BB121462846BDE85C
:10B7B0003840FFF763BF074B9C4201D1AC68F1E70B
:10B7C000054B9C4208BFEC68ECE7002038BD00BF89
:10B7D000D4DB0000F4DB0000B4DB0000002310B574
:10B7E0000446C0E90033836081814366C281C0E9B9
:10B7F00004338361194608225C30FFF7FDF9054BDD
:10B800006362054BA362054BE362054B246223632D
:10B8100010BD00BF05C0000027C000005FC00000D1
:10B8200083C00000014900F085B800BF89B700005F
:10B8300070B54A1E682555430E4605F1740100F0A7
:10B84000BDF9044640B10021C0E900160C30A060EB
:10B8500005F16802FFF7D0F9204670BD836910B585
:10B86000044633BBC0E912330365124B124A1B680E
:10B870008262984204BF0123836100F01FF8606078
:10B88000204600F01BF8A060204600F017F80022C8
:10B89000E06004216068FFF7A1FF01220921A06890
:10B8A000FFF79CFF02221221E068FFF797FF0123B8
:10B8B000A36110BD7CDB000025B80000F8B51B4B70
:10B8C0001E68B369074613B93046FFF7C7FF48360D
:10B8D000D6E90134013B03D5336833B13668F7E765
:10B8E000B4F90C506DB16834F4E704213846FFF721
:10B8F0009FFF30600028F1D10C233B6004462046B6
:10B90000F8BD0B4B6566C4E90055A560C4E9033575
:10B91000C4E905550822294604F15C00FFF76CF9DB
:10B92000C4E90D55C4E91255E9E700BF7CDB00000E
:10B930000100FFFF2DE9F8438046894600F14804E5
:10B94000002614B93046BDE8F883D4E90175013FFB
:10B9500001D52468F5E7AB89012B07D9B5F90E307D
:10B96000013303D029464046C84706436835EEE711
:10B97000D0F8EC00704770B50E46B1F90E100029F2
:10B9800096B014461D4607DA00232B60B3891A06C9
:10B9900010D44FF480630EE06A4600F0A5FB002847
:10B9A000F2DB019A02F47042A2F500535A425A4166
:10B9B0002A60EEE740230020236016B070BD00002F
:10B9C0008B8973B59D0706460C4607D504F14703DE
:10B9D000236023610123636102B070BD01AB6A463D
:10B9E000FFF7C9FF00990546304600F0E7F848B96F
:10B9F000B4F90C309A05EFD423F0030343F00203AB
:10BA0000A381E3E70D4BB362A389206043F0800379
:10BA1000A381009B6361019B20615BB1B4F90E10AF
:10BA2000304600F073FB28B1A38923F0030343F0F1
:10BA30000103A381A3891D43A581CDE725B800009B
:10BA4000024B0146186800F0B9B800BF6000002042
:10BA500082B001B901A942B14BB113780B601278E1
:10BA6000101C18BF012002B070471046FBE76FF0B2
:10BA70000100F8E7000000000000000000000000E6
:10BA800001F0FF01102A2BDB10F0070F08D010F88F
:10BA9000013B013A8B422DD010F0070F42B3F6D193
:10BAA000F0B441EA012141EA014122F007047FF0AC
:10BAB00000070023F0E80256083C85EA010586EA03
:10BAC000010685FA47F5A3FA87F586FA47F6A5FA3F
:10BAD00087F68EB9EED1F0BC01F0FF0102F007024B
:10BAE00032B110F8013B013A83EA010313B1F8D1F6
:10BAF0000020704701387047002D06BF35460338D7
:10BB0000073815F0010F07D1013015F4807F02BF0F
:10BB1000013015F4C03F0130F0BC0138704700BF60
:10BB200038B50546002945D051F8043C0C1F002BC0
:10BB3000B8BFE41800F00CFB1F4A1368104633B975
:10BB4000636014602846BDE8384000F002BBA342A1
:10BB50000CD921686218934204BF1A685B6863605D
:10BB600004BF521822600460ECE713465A680AB119
:10BB7000A242FAD919685818A0420BD12068014492
:10BB8000581882421960DDD1106852685A60014429
:10BB90001960D7E702D90C232B60D3E7206821185E
:10BBA0008A4204BF11685268626004BF09182160AC
:10BBB0005C60C7E738BD00BFFC7C012070B5CD1CC0
:10BBC00025F0030508350C2D38BF0C25002D064641
:10BBD00001DBA94203D90C233360002070BD00F0C3
:10BBE000B7FA214A1468214691B9204C23681BB941
:10BBF000304600F0B3F920602946304600F0AEF937
:10BC0000431C24D10C233360304600F0A2FAE4E751
:10BC10000B685B1B18D40B2B0FD90B60CD50CC18C5
:10BC2000304600F096FA04F10B00231D20F00700C7
:10BC3000C31AD3D05A42E250D0E78C424B6816BFA9
:10BC4000636013600C46EBE70C464968CCE7C41C04
:10BC500024F00304A04205D0211A304600F07EF9FA
:10BC60000130CFD02560DBE7FC7C0120007D012086
:10BC7000F8B5074614460E4621B91146BDE8F8400E
:10BC8000FFF79CBF22B9FFF74BFF25462846F8BDBA
:10BC900000F060FAA0420FD221463846FFF78EFF2F
:10BCA00005460028F2D031462246FEF781FF314694
:10BCB0003846FFF735FFE9E73546E7E72DE9F04776
:10BCC0008E689E4282460C469046994637D88A89AD
:10BCD00012F4906F31D0256809696F1A65690223E3
:10BCE00005EB450595FBF3F509F101033B449D4246
:10BCF00038BF1D46530530D52946FFF75FFF06467E
:10BD000050B90C23CAF80030A38943F04003A38143
:10BD10004FF0FF30BDE8F0873A462169FEF748FF53
:10BD2000A38923F4906343F08003A38126616561B6
:10BD30003E44ED1B2660A5604E464E4500D94E465A
:10BD4000324641462068FEF73EFFA3689B1BA36076
:10BD500023681E4426600020DCE72A46FFF788FFA0
:10BD600006460028E2D121695046FFF7D9FEC8E710
:10BD70002DE9F04F9DB0804603938B891D060C463C
:10BD800016460FD50B696BB94021FFF717FF2060EE
:10BD9000206128B90C23C8F800304FF0FF30C7E00D
:10BDA000402363610023099320238DF82930302339
:10BDB0008DF82A304FF0010B37463D4615F8013B10
:10BDC0000BB1252B3ED1B7EB060A0BD053463246BA
:10BDD00021464046FFF772FF013000F0A480099B26
:10BDE000534409933B78002B00F09D8000234FF0D3
:10BDF000FF32CDE90523049307938DF853301A934E
:10BE00002F46052217F8011B4F48FFF739FE049B08
:10BE1000D0B9D90644BF20228DF853201A0744BF59
:10BE20002B228DF853202A782A2A15D0079A2F46DC
:10BE300000200A25394611F8013B303B092B4DD92A
:10BE4000B8B10FE02F46B8E73F4A801A0BFA00F06E
:10BE5000184304903D46D3E7039A111D12680391DD
:10BE6000002A01DB079204E0524243F002030792EA
:10BE700004933B782E2B0CD17B782A2B33D1039B58
:10BE80001A1D1B680392002BB8BF4FF0FF33023717
:10BE900005932E4D397803222846FFF7F1FD38B17E
:10BEA0004023401B03FA00F0049B03430137049333
:10BEB000397827488DF8281006227E1CFFF7E0FD10
:10BEC000002838D0234B13BB039B073323F0070311
:10BED00008330393099B4B4409936DE705FB02323A
:10BEE00001200F46A6E700230137059319460A25CE
:10BEF000384610F8012B303A092A03D9002BC8D054
:10BF00000591C6E705FB012101230746F0E703ABD6
:10BF100000932246104B04A94046AFF30080B0F1D5
:10BF2000FF3F8146D6D1A3895B063FF536AF09981E
:10BF30001DB0BDE8F08F03AB00932246064B04A969
:10BF40004046FFF715F8EAE780DB000086DB0000DB
:10BF50008ADB000000000000BDBC000038B5064CC4
:10BF6000002305460846236000F046F9431C02D131
:10BF7000236803B12B6038BD909001201F2938B58C
:10BF800004460D4604D9162303604FF0FF3038BD38
:10BF9000426C12B152F821304BB9204600F030F813
:10BFA0002A4601462046BDE8384000F017B8012B6C
:10BFB0000AD0591C03D1162303600120E7E70024AF
:10BFC00042F82540284698470020E0E7024B01460A
:10BFD0001868FFF7D3BF00BF6000002038B5074CDA
:10BFE0000023054608461146236000F0EDF8431C87
:10BFF00002D1236803B12B6038BD00BF90900120AF
:10C0000000F0D2B810B50C46B1F90E1000F0AAF845
:10C010000028ABBF636DA3891B1823F48053ACBF0A
:10C020006365A38110BD2DE9F0411F468B89DB05B7
:10C0300005460C46164605D502230022B1F90E101E
:10C0400000F074F8A389B4F90E1023F48053A3818F
:10C0500032463B462846BDE8F04100F023B810B513
:10C060000C46B1F90E1000F061F8431CA38915BF0E
:10C07000606523F4805343F48053A38118BFA381E8
:10C0800010BDB1F90E1000F01FB849B1FF2A85BFED
:10C090008A2303600A704FF0FF3098BF0120704779
:10C0A0000846704738B5074C054608461146002239
:10C0B00022601A4600F0AEF8431C02D1236803B197
:10C0C0002B6038BD9090012038B5064C0023054602
:10C0D0000846236000F058F8431C02D1236803B1DE
:10C0E0002B6038BD9090012038B5074C00230546E1
:10C0F00008461146236000F04FF8431C02D1236824
:10C1000003B12B6038BD00BF9090012038B5064CBC
:10C11000002305460846236000F04EF8431C02D178
:10C12000236803B12B6038BD9090012038B5074CCF
:10C13000054608461146002222601A4600F04CF8D7
:10C14000431C02D1236803B12B6038BD90900120BD
:10C150007047704751F8043C181F002BBCBF0B58A8
:10C16000C018704738B5074C0546084611460022EE
:10C1700022601A4600F038F8431C02D1236803B14C
:10C180002B6038BD90900120024B58221A604FF06E
:10C19000FF30704790900120024B58221A604FF0F8
:10C1A000FF30704790900120024B58221A604FF0E8
:10C1B000FF30704790900120024B58221A600020F7
:10C1C000704700BF90900120024B58221A604FF038
:10C1D000FF30704790900120024B58221A604FF0B8
:10C1E000FF30704790900120024B58221A604FF0A8
:10C1F000FF30704790900120044A05491368002BD6
:10C2000008BF0B461844106018467047047D012093
:10C2100098900120024B58221A604FF0FF3070476F
:10C2200090900120FEE700BFF8B500BFF8BC08BC45
:10C230009E467047F8B500BFF8BC08BC9E467047E4
:10C240006461746100000000D6C200001D0300009C
:10C25000DFC200000D040000E7C20000E10B000097
:10C26000EEC200000D0D0000F3C200001906000030
:10C27000F9C20000F107000004C3000077040000C9
:10C2800009C30000490F000015C300004F03000060
:10C290001FC30000B90A00002DC30000950700006D
:10C2A0003AC300007D09000046C300005D0700009E
:10C2B00072616E646F6D00616C6C006C6173740010
:10C2C000300066616C7365007472756500252E31EF
:10C2D00035732E2E2E006D616B654C697374006191
:10C2E00064644C6173740064656C657465006A6FA6
:10C2F000696E0073706C697400636F707946726F59
:10C300006D546F0066696E64006A6F696E53747273
:10C31000696E677300756E69636F6465417400755B
:10C320006E69636F6465537472696E67006E6577DA
:10C330004279746541727261790061734279746502
:10C34000417272617900667265654D656D6F7279D3
:10C3500000000000C1C3000029140000C6C3000093
:10C3600043140000E7C2000047140000CCC30000E3
:10C370002D140000D6C300004B140000DFC30000E2
:10C380004F140000E9C3000053140000F2C3000082
:10C3900057140000FDC300005B14000009C4000036
:10C3A0003114000012C400003B1400001CC4000043
:10C3B0003514000027C400003F14000066696C6556
:10C3C000006F70656E00636C6F736500656E644F1F
:10C3D0006646696C6500726561644C696E650072E1
:10C3E00065616442797465730072656164496E7455
:10C3F0006F00617070656E644C696E65006170708D
:10C40000656E6442797465730066696C6553697A18
:10C41000650073746172744C697374006E6578742E
:10C42000496E4C6973740073797374656D496E66F7
:10C430006F0000001C1800002C18000040180000BD
:10C44000B4180000E6180000161900004819000092
:10C450006A190000AA190000E4190000341A00004B
:10C46000721A0000D21A0000121B0000321B0000DA
:10C47000661B0000A61B0000C81B0000F21B00008A
:10C480001C1C0000E6310000C81C0000901D0000CC
:10C49000021E00004C1E0000B01E0000CC1E00005A
:10C4A000EA1E00002820000068200000DA200000BA
:10C4B000082100003821000066210000CA21000088
:10C4C0002E22000090220000F222000066230000CD
:10C4D000E023000040240000A0240000D624000037
:10C4E0001A25000060250000A6250000F8250000A0
:10C4F0004E2600008C2600001C270000502700005C
:10C5000096270000DC270000222800005C2800009D
:10C51000A2280000E8280000442A0000F21B0000C6
:10C52000661B00005C2900001C1800009029000018
:10C53000B6290000EA290000102A00001C1800009B
:10C540001C1800001C1800001C180000BA2A00006B
:10C55000F62A0000362B0000862B0000AC2B0000D2
:10C560001A2C0000642C0000942C00001C18000001
:10C570001C180000B22C0000E42C0000162D000056
:10C580004A2D00006E2D0000CC2D0000F02D000083
:10C59000122E0000342E0000662E0000982E00009F
:10C5A000BC2E0000E02E0000122F0000362F0000ED
:10C5B0001C1800001C1800001C1800001C180000AB
:10C5C0001C180000682F00008E2F0000B42F000000
:10C5D000DA2F000000300000343000006830000026
:10C5E0009C300000D0300000F63000001C3100000C
:10C5F000503100001C1800001C1800001C1800001E
:10C600001C1800001C1800001C1800001C1800005A
:10C610001C1800001C1800001C1800001C1800004A
:10C620001C180000763100007631000098320000BE
:10C63000C83200005B2564206974656D206C6973E5
:10C64000745D002825642062797465732900286F61
:10C65000626A65637420747970653A2025642900E4
:10C66000537461636B20756E646572666C6F7700DE
:10C67000626F6F6C65616E006E756D6265720073DE
:10C680007472696E67006C697374006279746520F6
:10C690006172726179000000070000000300000071
:10C6A00029C70000E533000031C7000091340000C5
:10C6B0003AC700009936000043C70000E933000084
:10C6C0004CC700009D36000054C70000253600000E
:10C6D0005DC700007135000068C700000D3800001C
:10C6E00073C70000353600007EC70000D137000058
:10C6F0008AC700001D35000096C7000027390000DA
:10C700000000000001000000020000000300000023
:10C71000040000000A0000001D0000006D69637243
:10C720006F3A62697420763200686173546F6E6587
:10C7300000706C6179546F6E650068617353657247
:10C74000766F00736574536572766F006461634938
:10C750006E69740064616357726974650073717502
:10C760006172655761766500736574557365724CC7
:10C77000454400616E616C6F675265616400616E73
:10C78000616C6F6757726974650064696769746189
:10C790006C52656164006469676974616C577269A1
:10C7A000746500474320746F6F6B20256420757398
:10C7B0006563733B206672656520256420776F7220
:10C7C0006473003C496E74656765723E003C4C6959
:10C7D00073743E003C4F626A6563743E003C42796C
:10C7E000746541727261793E000D0A564D205061A8
:10C7F0006E69633A2025730D0A006D69736300004A
:10C8000035C80000C94300003EC800004D43000089
:10C8100042C80000994200004AC800003B420000A4
:10C8200054C80000CD41000060C80000CF400000A7
:10C830006E756C6C00686578546F496E740073692E
:10C840006E006A736F6E476574006A736F6E436F34
:10C85000756E74006A736F6E56616C756541740015
:10C860006A736F6E4B6579417400000030C9000037
:10C870002944000038C900002D44000042C90000CE
:10C880003F4400004BC900004544000056C9000069
:10C890004B44000062C900005144000070C9000010
:10C8A0005744000078C900005D4400007EC90000C4
:10C8B0006344000093C9000069440000A8C9000057
:10C8C0006F440000B4C9000075440000C4C90000F2
:10C8D0007B440000D0C9000081440000DDC9000095
:10C8E00087440000ECC900008D440000FFC900002F
:10C8F0009344000015CA00009944000021CA0000BA
:10C900009F44000031CA0000A544000040CA000056
:10C91000AB4400004ECA0000B144000056CA0000FB
:10C92000334400005ECA0000394400006E657400A4
:10C930006861735769466900737461727457694618
:10C94000690073746F705769466900776966695347
:10C950007461747573006D794950416464726573D4
:10C9600073007374617274535349447363616E004E
:10C9700067657453534944006D794D4143006874B1
:10C98000747053657276657247657452657175652A
:10C99000737400726573706F6E64546F4874747052
:10C9A000526571756573740068747470436F6E6E50
:10C9B00065637400687474704973436F6E6E656369
:10C9C0007465640068747470526571756573740081
:10C9D00068747470526573706F6E7365007765620A
:10C9E000536F636B6574537461727400776562533F
:10C9F0006F636B65744C6173744576656E74007714
:10CA00006562536F636B657453656E64546F436CFA
:10CA100069656E74004D515454436F6E6E65637456
:10CA2000004D5154544973436F6E6E656374656471
:10CA3000004D515454446973636F6E6E65637400A6
:10CA40004D5154544C6173744576656E74004D516C
:10CA50005454507562004D515454537562004D51F9
:10CA60005454556E7375620004000000030000000A
:10CA70000A0000000700000006000000000000009F
:10CA80000008080800080A4A4000000A5FEA5FEA56
:10CA90000ED92ED36E19324489330C924C924D0824
:10CAA0000800000004880808040804848488000A38
:10CAB000448A4000048EC480000000048800000EF8
:10CAC000C000000000080001224488100C9252525D
:10CAD0004C048C84848E1C824C901E1EC244924C4A
:10CAE00006CA525FE21FF01EC13E02448ED12E1FC5
:10CAF000E24488100ED12ED12E0ED12EC48800080B
:10CB000000080000048004880244880482000EC0EB
:10CB10000EC008048244880ED126C0040ED135B35D
:10CB20006C0C925ED2521C925C925C0ED010100E75
:10CB30001C9252525C1ED01C901E1ED01C90100ED7
:10CB4000D013712E12525ED2521C8808081C1FE2AC
:10CB500042524C1254981492101010101E113B7532
:10CB6000B131113935B3710C9252524C1C925C9018
:10CB7000100C92524C861C925C92510ED00C825C2E
:10CB80001FE4848484125252524C1131312A4411D0
:10CB90003135BB7112524C9252112A4484841EC406
:10CBA00088101E0EC808080E10080482410EC242EA
:10CBB000424E048A400000000000001F080480006C
:10CBC00000000ED2524F10101C925C000ED0100EBE
:10CBD00002424ED24E0C925C900E06C81C88080E83
:10CBE000D24EC24C10101C92520800080808024095
:10CBF00002424C10149814920808080806001B758D
:10CC0000B131001C925252000C92524C001C925CAA
:10CC100090000ED24EC2000ED010100006C804982C
:10CC200008080EC807001252524F0011312A440062
:10CC3000113135BB00124C8C9200112A4498001E11
:10CC4000C4881E06C48C8486080808080818080CC6
:10CC5000881800000C836000000000000100000044
:10CC600002000000030000000400000005000000B6
:10CC70000600000007000000080000000900000096
:10CC80000A0000000B0000000C0000000D00000076
:10CC90000E0000000F000000100000001200000055
:10CCA0001400000016000000180000001A00000028
:10CCB0001C0000001E0000002000000023000000F7
:10CCC00026000000290000002C0000002F000000BA
:10CCD00032000000360000003A0000003E00000074
:10CCE00042000000460000004B0000005000000021
:10CCF000550000005A0000006100000068000000BC
:10CD00006F000000760000007D000000840000003D
:10CD10008B0000009200000099000000A0000000BD
:10CD2000A7000000AE000000B5000000BC0000003D
:10CD3000C3000000CA000000D1000000D8000000BD
:10CD4000DF000000E6000000ED000000F40000003D
:10CD5000FB000000FF0000000000000002000000D7
:10CD6000040000000100000003000000D0CD00001E
:10CD7000CD440000DBCD0000954A0000E5CD000069
:10CD800095460000F2CD000009480000F9CD0000F2
:10CD90005548000002CE0000A54800000ECE00005D
:10CDA000994700001FCE00009D4900002CCE0000D6
:10CDB00021470000150000001600000017000000C9
:10CDC0001800000019000000646973706C6179003C
:10CDD0006C696768744C6576656C006D6244697354
:10CDE000706C6179006D62446973706C61794F6633
:10CDF00066006D62506C6F74006D62556E706C6F82
:10CE000074006D62447261775368617065006D6291
:10CE10005368617065466F724C6574746572006E1C
:10CE2000656F506978656C53656E64006E656F5010
:10CE30006978656C53657450696E004E6F74206537
:10CE40006E6F75676820726F6F6D206576656E20F6
:10CE5000616674657220636F6D70616374696F6E73
:10CE600000436F6D70616374656420466C61736824
:10CE700020636F64652073746F72650A2564206295
:10CE800079746573207573656420282564252529C8
:10CE9000206F6620256400426164207265636F72B2
:10CEA0006420666F756E6420647572696E672069B0
:10CEB0006E697469616C697A6174696F6E0025646A
:10CEC0002025642025642028256420776F726473F0
:10CED00029002564207265636F7264732C202564B9
:10CEE00020776F7264732C206D617849442025642B
:10CEF0002C20636F6D70616374696F6E206379635A
:10CF00006C657320256400526573746F72656420CC
:10CF10002564207363726970747300537461727452
:10CF2000656400726164696F00000000C1CF000099
:10CF30007D520000CECF000015550000DECF00006E
:10CF4000A9540000ECCF000075560000F7CF000098
:10CF50009552000007D00000195300001BD00000BC
:10CF6000FD5200002AD000005158000036D00000C9
:10CF7000CD5700003FD00000715700004AD000009C
:10CF8000C156000055D00000F95600005ED00000E8
:10CF90002957000067D00000A552000076D000009D
:10CFA000D95200007FD00000B552000025303878FB
:10CFB000006E6F6E65006F746865720070616972F3
:10CFC0000064697361626C65526164696F006D65CC
:10CFD0007373616765526563656976656400706146
:10CFE000636B657452656365697665007061636B38
:10CFF000657453656E64007265636569766564493E
:10D000006E74656765720072656365697665644D07
:10D0100065737361676554797065007265636569EE
:10D02000766564537472696E670073656E64496EE9
:10D0300074656765720073656E6450616972007330
:10D04000656E64537472696E6700736574436861DA
:10D050006E6E656C0073657447726F7570007365F2
:10D0600074506F776572007369676E616C53747288
:10D07000656E677468006465766963654944006C31
:10D080006173744D657373616765494400556E6BD8
:10D090006E6F776E207072696D6974697665205B5A
:10D0A00025733A25735D0000000000009630077775
:10D0B0002C610EEEBA51099919C46D078FF46A708C
:10D0C00035A563E9A395649E3288DB0EA4B8DC79AC
:10D0D0001EE9D5E088D9D2972B4CB609BD7CB17E2C
:10D0E000072DB8E7911DBF906410B71DF220B06AFC
:10D0F0004871B9F3DE41BE847DD4DA1AEBE4DD6D0C
:10D1000051B5D4F4C785D38356986C13C0A86B640B
:10D110007AF962FDECC9658A4F5C0114D96C06632B
:10D12000633D0FFAF50D088DC8206E3B5E10694C0B
:10D13000E44160D5727167A2D1E4033C47D4044B4B
:10D14000FD850DD26BB50AA5FAA8B5356C98B2422B
:10D15000D6C9BBDB40F9BCACE36CD832755CDF45AB
:10D16000CF0DD6DC593DD1ABAC30D9263A00DE51DB
:10D170008051D7C81661D0BFB5F4B42123C4B356CB
:10D180009995BACF0FA5BDB89EB802280888055F4B
:10D19000B2D90CC624E90BB1877C6F2F114C6858AB
:10D1A000AB1D61C13D2D66B69041DC760671DB0199
:10D1B000BC20D2982A10D5EF8985B1711FB5B6066B
:10D1C000A5E4BF9F33D4B8E8A2C9077834F9000FAB
:10D1D0008EA8099618980EE1BB0D6A7F2D3D6D084B
:10D1E000976C6491015C63E6F4516B6B62616C1C3B
:10D1F000D83065854E0062F2ED95066C7BA5011B6B
:10D20000C1F4088257C40FF5C6D9B06550E9B7120A
:10D21000EAB8BE8B7C88B9FCDF1DDD62492DDA15CA
:10D22000F37CD38C654CD4FB5861B24DCE51B53AEA
:10D230007400BCA3E230BBD441A5DF4AD795D83DEA
:10D240006DC4D1A4FBF4D6D36AE96943FCD96E342A
:10D25000468867ADD0B860DA732D0444E51D03330A
:10D260005F4C0AAAC97C0DDD3C710550AA4102271A
:10D2700010100BBE86200CC925B56857B3856F20EA
:10D2800009D466B99FE461CE0EF9DE5E98C9D9294A
:10D290002298D0B0B4A8D7C7173DB359810DB42E8A
:10D2A0003B5CBDB7AD6CBAC02083B8EDB6B3BF9AD6
:10D2B0000CE2B6039AD2B1743947D5EAAF77D29D62
:10D2C0001526DB048316DC73120B63E3843B649442
:10D2D0003E6A6D0DA85A6A7A0BCF0EE49DFF099342
:10D2E00027AE000AB19E077D44930FF0D2A30887B2
:10D2F00068F2011EFEC206695D5762F7CB67658062
:10D3000071366C19E7066B6E761BD4FEE02BD38961
:10D310005A7ADA10CC4ADD676FDFB9F9F9EFBE8EC1
:10D3200043BEB717D58EB060E8A3D6D67E93D1A101
:10D33000C4C2D83852F2DF4FF167BBD16757BCA6E1
:10D34000DD06B53F4B36B248DA2B0DD84C1B0AAF81
:10D35000F64A0336607A0441C3EF60DF55DF67A801
:10D36000EF8E6E3179BE69468CB361CB1A8366BC91
:10D37000A0D26F2536E2685295770CCC03470BBBE1
:10D38000B91602222F260555BE3BBAC5280BBDB2E1
:10D39000925AB42B046AB35CA7FFD7C231CFD0B581
:10D3A0008B9ED92C1DAEDE5BB0C2649B26F263EC73
:10D3B0009CA36A750A936D02A906099C3F360EEB81
:10D3C0008567077213570005824ABF95147AB8E241
:10D3D000AE2BB17B381BB60C9B8ED2920DBED5E521
:10D3E000B7EFDC7C21DFDB0BD4D2D38642E2D4F171
:10D3F000F8B3DD686E83DA1FCD16BE815B26B9F601
:10D40000E177B06F7747B718E65A0888706A0FFF60
:10D41000CA3B06665C0B0111FF9E658F69AE62F820
:10D42000D3FF6B6145CF6C1678E20AA0EED20DD720
:10D430005483044EC2B30339612667A7F71660D040
:10D440004D476949DB776E3E4A6AD1AEDC5AD6D980
:10D45000660BDF40F03BD83753AEBCA9C59EBBDEA0
:10D460007FCFB247E9FFB5301CF2BDBD8AC2BACA50
:10D470003093B353A6A3B4240536D0BA9306D7CDC0
:10D480002957DE54BF67D9232E7A66B3B84A61C4E0
:10D49000021B685D942B6F2A37BE0BB4A18E0CC3A0
:10D4A0001BDF055A8DEF022D416C6C207461736B8C
:10D4B000732073746F7070656400763135350020A9
:10D4C0002573202573004D656D6F727920636C653F
:10D4D00061726564004E6F206672656520746173C9
:10D4E0006B20656E747269657300000064D500007E
:10D4F0002971000071D50000416900007DD5000050
:10D50000F970000083D500000971000089D5000082
:10D51000197100008FD50000D16F0000A5D5000063
:10D5200025720000B3D5000071690000BDD5000070
:10D53000B5720000C5D50000A56D0000CED5000075
:10D54000716B0000DAD50000796A0000E3D50000B5
:10D55000C16A0000EBD50000C56C000073656E73F6
:10D560006F727300616363656C65726174696F6E7D
:10D570000074656D70657261747572650074696CB4
:10D5800074580074696C74590074696C745A00732F
:10D590006574416363656C65726F6D657465725225
:10D5A000616E6765006D61676E6574696346696584
:10D5B0006C6400746F7563685265616400693263FE
:10D5C00052656164006932635772697465007370F3
:10D5D0006945786368616E67650073706953657447
:10D5E00075700072656164444854006D6963726FC0
:10D5F00070686F6E65000000C1C3000039750000DF
:10D60000C6C30000357600002FD600005976000012
:10D61000E9C30000BD74000034D60000D9760000D4
:10D620003AD600009173000073657269616C0072F4
:10D630006561640077726974650077726974654228
:10D640007974657300000000C4D60000757700008F
:10D65000D2D6000085770000DFD600007977000081
:10D66000E8D6000089770000F2D600008D77000030
:10D67000FBD600009177000000D7000095770000EE
:10D6800005D700009977000011D700009D770000B2
:10D6900018D70000A177000021D70000A57700006F
:10D6A00026D70000A977000031D70000AD77000031
:10D6B0003BD700007D77000045D700008177000050
:10D6C00074667400656E61626C65446973706C6148
:10D6D00079007365744261636B6C69676874006795
:10D6E000657457696474680067657448656967683C
:10D6F0007400736574506978656C006C696E6500C0
:10D700007265637400726F756E64656452656374EC
:10D7100000636972636C6500747269616E676C6541
:10D72000007465787400746674546F75636865641A
:10D7300000746674546F7563685800746674546F2F
:10D740007563685900746674546F756368507265C8
:10D750007373757265007661727300007CD7000088
:10D76000157C000086D70000F57B00008FD70000F5
:10D77000D17B00009BD70000617B00007661724581
:10D780007869737473007661724E616D65640073BD
:10D7900065745661724E616D6564007661724E61AA
:10D7A0006D65466F72496E6465780057656C636F8E
:10D7B0006D6520746F204D6963726F426C6F636B8F
:10D7C000732100705F73706920213D204E554C4CD1
:10D7D000002F686F6D652F6769742F2E706C6174F0
:10D7E000666F726D696F2F7061636B616765732F10
:10D7F0006672616D65776F726B2D61726475696EAB
:10D800006F6E6F726469636E7266352F6C696272D7
:10D8100061726965732F5350492F5350492E6370BD
:10D820007000535049436C6173733A3A5350494303
:10D830006C617373284E52465F5350495F54797040
:10D84000652A2C2075696E74385F742C2075696E9A
:10D8500074385F742C2075696E74385F7429000009
:10D860000000000000000000E97D0000A17D000034
:10D87000D77D0000DD7D0000E37D0000D57D000048
:10D880000200000003000000040000001F00000070
:10D890001C0000000E000000250000000B0000002E
:10D8A0000A000000090000001E0000001700000030
:10D8B0000C00000011000000010000000D0000003D
:10D8C00022000000FFFFFFFFFFFFFFFF1A00000024
:10D8D0002000000015000000160000000F000000EE
:10D8E00018000000130000002400000000000000E9
:10D8F00014000000050000001000000008000000F7
:10D9000019000000280000000600000000000000D0
:10D9100000000000CB830000E58A00004184000085
:10D920004D84000047840000C9830000C1830000CB
:10D9300055840000E5830000BD83000000C0014065
:10D94000001002400020024000D002400000000011
:10D95000000000000000304300000000000030C361
:10D960007371727400000000FB21F93FFB21094034
:10D970007CD91240FB2119407A6A1F407CD9224091
:10D98000BBFD2540FB2129403A462C407A6A2F40B6
:10D990005C4731407CD932409C6B3440BBFD354004
:10D9A000DB8F3740FB2139401BB43A403A463C40BC
:10D9B0005AD83D407A6A3F404C7E40405C474140E7
:10D9C0006C1042407CD942408CA243409C6B444046
:10D9D000AC344540BBFD4540CBC64640DB8F47409D
:10D9E000EB584840FB21494083F9A200444E6E00A9
:10D9F000FC291500D1572700DD34F50062DBC0009B
:10DA00003C999500419043006351FE00BBDEAB00A2
:10DA1000B761C5003A6E2400D24D42004906E000CD
:10DA200009EA2E001C92D100EB1DFE0029B11C005A
:10DA3000E83EA700F535820044BB2E009CE9840037
:10DA4000B4267000417E5F00D691390053833900BF
:10DA50009CF439008B5F840028F9BD00F81F3B005F
:10DA6000DEFF97000F980500112FEF000A5A8B0078
:10DA70006D1F6D00CF7E360009CB2700464FB700E3
:10DA80009E663F002DEA5F00BA277500E5EBC700F0
:10DA90003D7BF100F739070092528A00FB6BEA00E8
:10DAA0001FB15F00085D8D00300356007BFC46000F
:10DAB000F0AB6B0020BCCF0036F49A00E3A91D0048
:10DAC0005E619100081BE60085996500A0145F0067
:10DAD0008D40680080D8FF0027734D000606310096
:10DAE000CA561500C9A873007BE260006B8CC000A9
:10DAF00000000040FB21F93F000000002D44743E6F
:10DB0000000000809846F83C0000006051CC783B53
:10DB100000000080831BF0390000004020257A3887
:10DB2000000000802282E336000000001DF369350A
:10DB300002000000030000000400000006000000D6
:10DB40002C2066756E6374696F6E3A200061737382
:10DB5000657274696F6E2022257322206661696C7C
:10DB600065643A2066696C6520222573222C206C3E
:10DB7000696E65202564257325730A006400002002
:10DB8000232D302B2000686C4C00656667454647A6
:10DB90000030313233343536373839414243444529
:10DBA0004600303132333435363738396162636498
:10DBB000656600000000000000000000000000009A
:10DBC0000000000000000000000000000000000055
:10DBD0000000000000000000000000000000000045
:10DBE0000000000000000000000000000000000035
:10DBF0000000000000000000000000000000000025
:10DC00000000000000000000000000000000000014
:10DC100000000000504F53495800002020202020D1
:10DC200020202020282828282820202020202020CC
:10DC300020202020202020202020208810101010BC
:10DC40001010101010101010101010040404040410
:10DC5000040404040410101010101010414141413C
:10DC60004141010101010101010101010101010124
:10DC70000101010101011010101010104242424236
:10DC800042420202020202020202020202020202F4
:10DC90000202020202021010101020000000000018
:10DCA0000000000000000000000000000000000074
:10DCB0000000000000000000000000000000000064
:10DCC0000000000000000000000000000000000054
:10DCD0000000000000000000000000000000000044
:10DCE0000000000000000000000000000000000034
:10DCF0000000000000000000000000000000000024
:10DD00000000000000000000000000000000000013
:10DD10000000000000000000000000000000000003
:08DD20002025FF7F0100000037
:10DD2800FFFFFFFFE803000001000000E803DC0537
:10DD3800DC05DC05DC050000FFFFFFFFFFFFFFFF40
:10DD48001800000019FCFFFFFFFFFFFF02000000A2
:10DD580040420F00FFFF01FF030000000090D003C6
:10DD6800FFFFFFFFFFFFFFFFFFFFFFFFFFFFFFFFBB
:10DD78000A00000001000000080000000100000087
:10DD88006400002000000000D4DB0000F4DB000089
:10DD9800B4DB0000000000000000000000000000EC
:10DDA800000000000000000000000000000000006B
:10DDB800000000000000000000000000000000005B
:10DDC800000000000000000000000000000000004B
:10DDD800000000000000000000000000000000003B
:10DDE80000000000430000000000000000000000E8
:10DDF800000000000000000000000000000000001B
:10DE080000000000430000000000000000000000C7
:10DE180000000000000000000000000000000000FA
:10DE280000000000430000000000000000000000A7
:10DE380000000000000000000000000000000000DA
:10DE48000000000043000000000000000000000087
:10DE580000000000000000000000000000000000BA
:10DE68000000000043000000000000000000000067
:10DE7800000000000000000000000000000000009A
:10DE88000000000043000000000000000000000047
:10DE9800000000000000000000000000000000007A
:10DEA8000000000043000000000000000000000027
:10DEB800000000000000000000000000000000005A
:10DEC800000000008BC0000051BA000000000000F4
:10DED8001ADC0000D4C20000F9C70000F9C700002E
:10DEE800F9C70000F9C70000F9C70000F9C700002A
:10DEF800F9C70000F9C70000F9C70000FFFFFFFFDE
:10DF0800FFFFFFFFFFFFFFFFFFFF0000010041537E
:10DF18004349490000000000000000000000000024
:10DF28000000000000000000000000000000415355
:10DF38004349490000000000000000000000000004
:10DF480000000000000000000000000000000000C9
:10DF5800250200006D7D0000C98100005586000083
:04DF680001020000B2
:0400000300008285F2
:00000001FF
